:1000000008200300850F0200490E02004D0E020079
:100010009D0F0200A10F0200A50F020000000000CA
:10002000000000000000000000000000A90F020016
:10003000AD0F020000000000DDB800006BBA010047
:100040000000000000000000B10F0200010E0200DD
:1000500085FB01000000000000000000000000001F
:1000600000000000000000008D0F020000000000F2
:100070000000000000000000EDE9000000000000AA
:10008000F5EA000037EB0000D10C0200D10C0200B1
:10009000050C02000000000000000000000000004D
:1000A000F8B500224FF41261DFF8600B02F0E0F9BE
:1000B000DFF85C4B0022102104F1200002F0D8F997
:1000C000DFF8505B0022182105F10C0002F0D0F996
:1000D0000022082104F1300002F0CAF900220821B0
:1000E00004F1380002F0C4F9002020646064A064C8
:1000F000E0646862A862E862DFF81C6B7063B0635A
:10010000F0632863306470646863A863E863012067
:1001100028640020B064F0644FF0FF306864A86485
:100120000020E864306520657065F06530667066B3
:10013000B066B06202462821304602F099F90020EC
:1001400070600220308100203060DFF8D07A0246F3
:100150000C21384602F08CF9DFF8C40A7860DFF829
:10016000C40A386001203872002028702865688031
:10017000A880E8806065F066A060A065F0626865B0
:10018000A8656066A066E066706730676866286686
:10019000E86501202867E866A8660020E867A86788
:1001A0006867062030860020F067B0672067DFF8B8
:1001B000DC0DE065002020660120A081962068818A
:1001C000062070860C20E0810020B06502464021A8
:1001D00007F10C0002F04CF900220621204602F043
:1001E00047F90022102104F1100002F041F900202B
:1001F000E0616067F1BD10B584B0DFF8204A0C22E1
:10020000214600A802F072F9FFF74AFF0C2200A96C
:10021000204602F06BF91FBD2DE9F0472DED0C8B48
:1002200090B00024254600A821460A460B460EC081
:10023000302102F093F99FEDA98ADFF8D46996ED99
:100240001B0AD6ED140AC6ED1B0ADFF8CC7997ED30
:10025000149A86ED149ADFF8BC8998ED131AB8EE5B
:10026000411ADFED9F1AC1EE819AC7ED149AD8F8B2
:100270004420D8F83490A9EB0200FA30FA21B0FB00
:10028000F1F1FA2303FB110080B2002800F0228470
:100290004C2803DAD8F84010012906D12046F8622C
:1002A0000220A8F8080000F015BCD7F84CA0BAF15D
:1002B000040F24D3F4EE490AF1EE10FA1FD5B4EE80
:1002C000699AF1EE10FA1AD59FED861A20EE811A7E
:1002D000B4EE691AF1EE10FA11D59FED831AF4EE1F
:1002E000419AF1EE10FA0ADB87ED149AC6ED140A72
:1002F00086ED1B0A0320A8F8080000F025BC97ED46
:100300000DAA87ED0EAAD7ED10AAC7ED11AA0146D6
:1003100000EE101AB8EE400AD8ED0B8AC8EE800A3B
:1003200098ED0C1A81EE001A21467963396420E0B9
:10033000521C92B2FA2A00D12246DFF8D03803EBE1
:100340008203D3ED231A71EEE01AD3F8743402EE6F
:10035000103A32EE412AD7ED0D2A41EEA12AC7ED1F
:100360000D2AD7ED101A42EE021AC7ED101A491CD9
:1003700089B28142DCDBD7ED0D0A80EE80BA87EDD1
:100380000DBAD7ED100A80EE80CA87ED10CAD6EDFF
:100390001ABA98ED160AD8ED150A70EEC0CAF5EE35
:1003A00040CAF1EE10FA02DDC6ED1ACA03E030EEE3
:1003B000600A86ED1A0A00F0ADFF012802D120463E
:1003C000F86287E3BAF1000F0BD1B88D052802DB84
:1003D00005462046B885F88D052802DB45192046DC
:1003E000F8851AFA85F0002827D1B6EE00DA3CEE3F
:1003F0002A0A20EE0D0ADFEDA10AB4EE600AF1EE42
:1004000010FA11D43BEE0A0A20EE0D0ADFED9C0A29
:10041000B4EE600AF1EE10FA06D4B3EE040AF4EE7C
:1004200040CAF1EE10FA08D5B88D401CB885C8F85E
:1004300048900620A8F808004CE3B88D002802D0A8
:1004400045192046B8851AFA85F000281BD1B7EE69
:10045000000AF4EE409AF1EE10FA03D50720A8F84E
:10046000080037E39FED870AF4EE409AF1EE10FAA8
:1004700006DBF88D401CF8850820A8F8080029E361
:100480002046F88503E0F88D45192046F885284672
:1004900080B200F0E3FF012808D187ED149AC7ED80
:1004A00010AAC6ED1ABA87ED0DAA13E39FED760ADE
:1004B000F4EE409AF1EE10FA02DBDFF8380C386502
:1004C0002046B885BAF1000F10D1386D786587EDF8
:1004D0000FBAB06E706600F0B5FE40E0000000009C
:1004E00000007A446666E63F01004040B6EE00DA5E
:1004F00000F0A8FE012816D197ED140AF0EE000ACC
:1005000020EE200A87ED140A6BEE0D0AC7ED0D0AE6
:100510002CEE0D1A87ED101AC7ED0E0A87ED111A91
:1005200086ED140A6D1C97ED140AD6ED140A30EE10
:10053000200A20EE0D0A87ED150A97ED0D0AD7ED7A
:100540000E0A30EE200A20EE0D0A87ED0F0A96ED16
:100550001A0A3BEE800A20EE0D0A86ED190A98F879
:100560000100012840F0AB82D8F80C00009000A8F0
:10057000D8F810104160D8F814108160214617E0B7
:1005800000AB03EB820393ED010A50F822C000EEAA
:1005900090CAB4EE600AF1EE10FA05D500EB820CB9
:1005A0008CED000AC3ED010A521C022AE8DB491C4B
:1005B000022901DA2246F8E79DED000AB5EE400A6D
:1005C000F1EE10FA2AD5B5EE400AF1EE10FA01DC90
:1005D000B1EE400AD0ED020A30EE800A80ED020A48
:1005E0009DED000AB5EE400AF1EE10FA01DCB1EE25
:1005F000400AD0ED010A30EE800A80ED010A9DED3F
:10060000000AB5EE400AF1EE10FA01DCB1EE400A44
:10061000DDED000A30EE800A8DED000A90ED010A52
:10062000D0ED020A30EEC01ADDED000A30EE600AAD
:10063000B4EE401AF1EE10FA05D5F0EE410AB0EE34
:10064000401AB0EE600AD6ED0C0AC6ED0D0A31EE86
:10065000400A80EE010A9FED0D1A20EE010A86ED98
:100660000C0AB06BF063F4EE400AF1EE10FA0FD50D
:1006700070EE600AC6ED0E0A0EE000BF00001643E1
:100680000000A042666616400100A0400000C8427B
:1006900070EEC00AC6ED0E0A386F796F081800EBCD
:1006A000D070401002EE100A86ED102AC6ED118AB5
:1006B000D7ED100AC6ED120AD7ED141ADFF8500C68
:1006C000C0EDC41A96ED131A31EE611AD6ED132A55
:1006D00072EEE12A21EE221A00F5447181ED011A31
:1006E000C6ED131AD7ED1B1AC1ED021AD8F818106F
:1006F000039103A9C1ED011AC1ED020AC1ED038AFC
:10070000C1ED041AC1ED058AC1ED061AB8EEC22A80
:1007100081ED072AC1ED081A81ED090AC1ED0A1A17
:1007200081ED0B1ADDED032A9FEDD03A62EE832AAC
:100730009FEDCF3A41EE832A9FEDCE3A20EE833AE9
:10074000DFEDCD3A08EEA33ADFEDCC3A61EEA33A05
:100750009FEDCB4A48EE843A9FEDCA4A21EE844A87
:10076000DFEDC94A02EE244ADFEDC84A61EEA44A31
:100770009FEDC75A40EE054A9FEDC65A21EE855AB5
:10078000DFEDC55A01EE255AF8EE085AF4EE652A57
:10079000F1EE10FA00F19381DFEDC05AB4EE653A44
:1007A000F1EE10FA00F18B81DFEDBD5AF4EE653AFF
:1007B000F1EE10FA00F18381DFEDBA5AB4EE654A2A
:1007C000F1EE10FA00F17B819FEDB76AF4EE464A34
:1007D000F1EE10FA00F173819FEDDE6AB4EE465A35
:1007E000F1EE10FA00F16B81DFEDDB6AF4EE662AC0
:1007F000F1EE10FAC0F26381DFEDD82AB4EE623A6E
:10080000F1EE10FAC0F25B81F4EE653AF1EE10FA07
:10081000C0F25581B4EE464AF1EE10FAC0F24F81B3
:10082000F4EE654AF1EE10FAC0F24981DFEDCC2A10
:10083000B4EE625AF1EE10FAC0F24181DFEDC92A3E
:100840009DED033AB4EE623AF1EE10FA01D5CDED2A
:10085000032ADDED032A9FEDC43AF4EE432AF1EEBC
:1008600010FA02DBDFF8E82B0392DFEDD52AF4EE75
:10087000621AF1EE10FA01D5C1ED012A9FEDD13ACD
:10088000DFEDBA3A91ED014AB4EE634AF1EE10FAA7
:1008900001DB81ED013A9FEDB64AF4EE440AF1EE38
:1008A00010FA01D581ED024AD1ED020A9FEDB14A5D
:1008B000F4EE440AF1EE10FA02DBDFF8982B8A60BE
:1008C000DFEDC10AF4EE608AF1EE10FA01D5C1ED58
:1008D000030A9FEDBE4AD1ED034AF4EE444AF1EE1D
:1008E00010FA02DBDFF8702BCA60F4EE621AF1EE48
:1008F00010FA01D5C1ED042AD1ED044AF4EE634AA1
:10090000F1EE10FA01DB81ED043AF4EE608AF1EECB
:1009100010FA01D5C1ED050AD1ED050AF4EE440A3D
:10092000F1EE10FA02DBDFF8302B4A61F4EE621AC6
:10093000F1EE10FA01D5C1ED062AD1ED060AF4EE6A
:10094000630AF1EE10FA01DB81ED063AF1EE000ADE
:10095000B4EE602AF1EE10FA02D54FF08142CA617E
:10096000D1ED070A9FEDA32AF4EE420AF1EE10FA48
:1009700002DBDFF84C2CCA61F4EE621AF1EE10FAD9
:1009800001D5C1ED082AD1ED080AF4EE630AF1EEB3
:1009900010FA01DB81ED083ADFED970AB4EE600A48
:1009A000F1EE10FA01D5C1ED090A91ED090ADFED6A
:1009B000930AB4EE600AF1EE10FA02DBDFF8442C81
:1009C0004A62F4EE621AF1EE10FA01D5C1ED0A2A7C
:1009D00091ED0A0AB4EE630AF1EE10FA01DB81ED43
:1009E0000A3AB5EE401AF1EE10FA01D52246CA6273
:1009F00091ED0B0ADFED820AB4EE600AF1EE10FA17
:100A000002DBDFF8042CCA62214612E01B1FD3ED83
:100A1000000A92ED031AF4EE410AF1EE10FA01D544
:100A20009FED780AB8EEC00AD2ED020A00EE208AE5
:100A3000491C31293ADA9FED740A0B011A18D2F8D1
:100A400004C0BCF1010F0DF10C0C1B580CEB83031F
:100A5000DCD11B1FD3ED000A92ED031AF4EE410A1C
:100A6000F1EE10FADEDB9FED670ADBE7168733BD98
:100A7000B0568DBD03275BB9E23C9CB9983115BED9
:100A8000BF49D3B97061FDBD55C128BC36CB05BE89
:100A90003D7FDABBDDED0ABEE4BE353E6666A6BF2D
:100AA0003333F3BFCDCC4CBFCDCC8CBFB5EE408A39
:100AB000F1EE10FA03DD0F20A8F808000AE097ED28
:100AC000150A284680B200F0AFF800F055F8044649
:100AD000C8F84890C8F844900020C8F84C00C8F8FE
:100AE0002C00C8F83000C8F840000246102106F17A
:100AF000200001F0BDFC00220C2108F10C0001F0E7
:100B000031FDDFF88804F06500203066F8880028A1
:100B10001AD1F86F00280CD0B86CF968401A398ED9
:100B2000B0EB510F02DB002038810DE0012038814D
:100B30000AE0B88DF98D11FA80F0032802DB01205C
:100B4000388101E002203881204610B0BDEC0C8BCA
:100B5000BDE8F087333333BFCDCC0CC09A9919BFB1
:100B6000CDCC4CBE5017C93FC9AC454216E66840D3
:100B70007D90A341A2F2924438B50025DFF81C4CC9
:100B80000120E06700F01EFD2060E06C218E8842AD
:100B900014D3A06CE060208DA080608DE080A06DFB
:100BA0006061E06DA061206EE061606E2062A06E09
:100BB00060620120A0672846E0670125284632BD13
:100BC000A9F56E3E15E66840BA9F17443564EC44BB
:100BD0001148C16881640021C16441600221018122
:100BE00000218162C1690166416A81660021C16795
:100BF00070470000010058427B4D4F3D47FFC74200
:100C0000BEBA984101000000FFFFFFFF88690300A2
:100C1000FC600300FC5F03007C600300A8BB0300D2
:100C200000002F43000070422DE9F84F2DED048B9A
:100C300082B08346002213461046DFF8604BE56C15
:100C400005F10F0101F00F01EE1D06F007060096F9
:100C5000DFF8506B06EB810787ED030ABBF1000F4D
:100C600018D0074614E0A1F1010CACEB070C0CF115
:100C7000100C4FEAEC0E0CEB1E7E4FEA2E1EBCEB66
:100C80000E1C03D406EB8C0C8CED030A7F1C3FB2C8
:100C90005F45E8DB102D02D2294609B200E00F21A2
:100CA0009FEDBB8ADFEDBA0A9FEDBA1A07461BE03B
:100CB00006EB810CDCED031AF5EE401AF1EE10FAAA
:100CC00010DD38EE218AF4EE610AF1EE10FA01D55A
:100CD000F0EE610AF4EE411AF1EE10FA01D5B0EE31
:100CE000611A7F1C491E09B20029E1D53FB239467D
:100CF00003290BDB78EE600A70EEC10A891E01EE53
:100D0000101AB8EEC11A80EE818A07E0012905DBCE
:100D100000EE907AF8EEE00A88EE208AB5EE408A7E
:100D2000F1EE10FA01D0002F01D1B0EE408A84ED2F
:100D3000168A9FED990AB4EE408AF1EE10FA02D5B8
:100D4000B0EE408A08E09FED950AB4EE408AF1EEDD
:100D500010FA01DBB1EE028AB0EE040AB4EE408A6A
:100D6000F1EE10FA08D494ED1B0AF0EE080AB4EE86
:100D7000600AF1EE10FA02D50321218501E0042179
:100D80002185A76C07F00709DFF8208A09EB080E18
:100D9000218D8EF8B818BBF1000F0BD0A7F1010C14
:100DA0000CF0070CC44407F0070AC2449AF8B8A82C
:100DB0008CF8B8A84FF0080C10E0BAF1040F00D17D
:100DC000401CA9F101090FFA89F9B9F1000F01D509
:100DD00009F10809ACF1010C0FFA8CFCBCF1010F10
:100DE00016DB0FFA89F909EB080A9AF9B8A8BAF1E3
:100DF000030F01D15B1C03E0BAF1040F00D1521CB8
:100E0000BCF1060FDDDBBAF1030FD6D1401ED8E7E7
:100E1000B4F82AC092B29BB29A4207D3934202D24C
:100E2000042060850DE000B2002802D50320608513
:100E300007E0012802DB0420608502E09EF9B80883
:100E40006085B4F82A90B9F1040F01D1104600E092
:100E50001846CC4509D000202081E088002820D108
:100E6000042D1ED3012020811BE012FA83F2012AF7
:100E700015DB052A10DB00EE102AB8EEC00AF6EEEC
:100E8000080A20EE200A00EE900AF8EE600AF4EE5E
:100E9000400AF1EE10FA02D50120208101E0022083
:100EA000208149B2B0EE480A304600F025F9DFED66
:100EB000900AB4EE600AF1EE10FA01D5B0EE600AC5
:100EC00084ED170A584600F1010A00EE90AAF8EEE8
:100ED000E08AD4ED180A48EE800AC4ED180A9FEDA6
:100EE000CE9A20EE080A20EE090A009908EB81014B
:100EF00001F65C0181ED000ABBF1000F1AD04FF042
:100F0000000C15E00099491EA1EB0C0108318A1074
:100F100001EB5272D210B1EBC20105D408EB810192
:100F200001F65C0181ED000A0CF1010C0FFA8CFC5A
:100F30008445E7DB082D02D2284600B203E00720F3
:100F400001E0401E00B20028FBD584ED190A494695
:100F500049B2304600F048F968EE090AB7EE001AC7
:100F6000C1EE200A20EE800AD4ED1A0A48EE800A6B
:100F7000C4ED1A0A0AEB0700A0640AEB0500E0645E
:100F800002B0BDEC048BBDE8F18F000000007A4494
:100F9000000000000000C8426666A63F01009040C5
:100FA00049B2032944D1DFED9D0AB4EE600AF1EEA7
:100FB00010FA01DBB0EE600A9FED991ADFED990A95
:100FC00040EE010A90ED011A9FED970AB4EE401A27
:100FD000F1EE10FA43DADFED951AB4EE611AF1EE94
:100FE00010FA74DBB4EE401AF1EE10FA6FD59FEDF3
:100FF000900A31EE000ADFED8F1A60EE211A9FEDA4
:101000008E0A9FED8E2A01EE002A22EE200A20EEA3
:10101000210A9FEDB72ADFEDB72A41EE022A62EEE0
:10102000A00AB7EE001A31EE611A00EE810A56E00E
:10103000DFED830A60EE200A60EE800A9FEDAE1AB3
:1010400040EE410A9FEDAD0A70EE800A90ED011A64
:101050009FED750AB4EE401AF1EE10FA0ADB90ED3E
:10106000010A9FED751ADFED751A40EE011A21EEA7
:10107000A00A34E0DFED6D1AB4EE611AF1EE10FA59
:1010800025DBB4EE401AF1EE10FA20D59FED680A88
:1010900031EE000ADFED671A60EE211A9FED660A55
:1010A0009FED662A01EE002A22EE200A20EE210A98
:1010B0009FED8F2ADFED8F2A41EE022A62EEA00A11
:1010C000B7EE001A31EE611A00EE810A07E090EDEA
:1010D000010A20EE800ADFED8A0A20EE200A007A5B
:1010E000022803D1DFEDD10A20EE200A704700006C
:1010F000CDCC4C3E0000A04010B52DED028BB0EEE3
:10110000408A0C46DFED7F8A49B2FFF749FF64B29F
:10111000042C31D1DFED7C0AB4EE608AF1EE10FAD6
:1011200016DBB1EE021AB4EE418AF1EE10FA0FD5D9
:10113000DFED760A78EE200AB1EE041A60EE810A3D
:10114000FCEEE00A10EE900AC01D08EE900A3DE0A9
:10115000B4EE608AF1EE10FA03D5072008EE900A8B
:1011600034E0F1EE020AB4EE608AF1EE10FA2DDB03
:10117000122008EE900A29E0F7EE080AB4EE608A21
:10118000F1EE10FA11DBDFEDAA0AB4EE608AF1EE9F
:1011900010FA0AD5FFEE080A78EE200AB1EE041A1A
:1011A00060EE810AFCEEE08A10E0F7EE080AB4EE89
:1011B000608AF1EE10FA09D4DFED9D0AB4EE608A80
:1011C000F1EE10FA02DB062008EE900ADFF8FC0CC4
:1011D00018EE901A00EB8100D0ED000A20EE200AF4
:1011E000BDEC028B10BD0000F0EE0C0A49B20429E0
:1011F00004D19FED901A40EE010A03E09FED8E1A94
:1012000040EE010A9FED8D0A20EE800AD0ED000A23
:1012100020EE200A70470000000070429A991940A1
:101220006ADEF13D8638163F00002A43000016436F
:10123000000016C3CDCC4C3D4260E53A6666263FC1
:101240002575C23E0020DFF8541591ED140AF7EE23
:10125000040AB4EE600AF1EE10FA47DADFF8702CF7
:10126000D288042A42DAD1ED150A9FED751A60EE94
:10127000810AB4EE600AF1EE10FA03D5022A01DB0E
:10128000012012E0DFF84C1C91ED0B0ADFED6D0A36
:10129000B4EE600AF1EE10FA07DBDFED6B0AB4EE94
:1012A000600AF1EE10FA00D5012001281ED1DFF806
:1012B000241C91ED170AD1ED180A70EEC00A9FEDBB
:1012C000631AF4EE410AF1EE10FA07DBF7EE080AB2
:1012D000B4EE600AF1EE10FA00D50020DFEDC50A89
:1012E000B4EE600AF1EE10FA00D50020704700005D
:1012F00052491D3BB81E053F7593E83F2497534064
:10130000C1C0C03B0000000066660640666606C0BD
:101310005C5503000021DFF88424538D032B1FDA72
:1013200092ED140ADFEDA50AB4EE600AF1EE10FAB0
:1013300016DB92ED0D0AF2EE040AB4EE600AF1EE4D
:1013400010FA0DD592ED100ADFEDAB0AB4EE600A8B
:10135000F1EE10FA04D50421DFF8743B1981012164
:1013600092ED100AF6EE000A92ED111A30EE011A13
:1013700021EE201AF3EE0E1AB4EE611AF1EE10FA15
:101380001CD492ED0D1AD2ED0E1A71EE211A61EEF7
:10139000A01AB2EE042AF4EE421AF1EE10FA0DD4BD
:1013A000F3EE041AB4EE610AF1EE10FA06D4B1EECF
:1013B000040AB4EE401AF1EE10FA04D50521DFF864
:1013C000103B1981012192ED140A9FED8C1AB4EEA5
:1013D000410AF1EE10FA27DBDFF8F82A92ED0A0A4B
:1013E00092ED0B1A80EE010A9FED851AB4EE410AC8
:1013F000F1EE10FA18DB00EE100AB8EE400A20EE0B
:10140000200AD2ED080AF4EE400AF1EE10FA0BD5EC
:10141000D2ED090AF4EE400AF1EE10FA04D50E20DE
:10142000DFF8AC1A08810121084670473333733F57
:101430009A993940CDCC4C3ECDCCCC3D0AD7A33B7C
:101440003333333F010020420000C8420100C03F57
:10145000C8AC4542A1F292443464EC4401460020F9
:10146000CE4AD36C13FA81F102291AD392ED140AF1
:10147000DFED8F0AB4EE600AF1EE10FA11DB92EDA7
:10148000110AD2ED100A80EE200ADFED8A0AB4EECE
:10149000600AF1EE10FA04DB0920DFF8343A188113
:1014A000012002291CD39FED840AD2ED110A92ED8E
:1014B000101AC0EE810AF4EE400AF1EE10FA0FDBCA
:1014C000D2ED0E0A92ED0D1AC0EE810AF4EE400A3A
:1014D000F1EE10FA04DB0A20DFF8F439188101205C
:1014E000002913D0DFF8EC1991ED190ADFEDA50AF8
:1014F00020EE200AD1ED1A0AF4EE400AF1EE10FABD
:1015000004D50B20DFF8C8190881012092ED140AD8
:10151000DFED9D0AB4EE600AF1EE10FA08DA92ED02
:10152000150ADFED9A0AB4EE600AF1EE10FA1EDB3E
:1015300092ED100ADFED960AB4EE600AF1EE10FAB1
:101540000DD492ED0D0ADFED930AB4EE600AF1EED0
:1015500010FA04D4DFF87819C988022907DB518D05
:10156000032904DB0C20DFF868190881012092EDC3
:101570000F0ADFED870AB4EE600AF1EE10FA08D424
:1015800092ED1B0AF1EE040AB4EE600AF1EE10FAD5
:1015900012D5116F526F511800EE101ABAEEEF0A01
:1015A000DFED7D0AB4EE600AF1EE10FA04DB0D20E7
:1015B000DFF81C190881012070470000010000407D
:1015C00000005842002075498A6C12F1640F0FD256
:1015D0009FED730AD1ED180AF4EE400AF1EE10FA0D
:1015E00006DAD1ED1A0AF4EE400AF1EE10FA00DB49
:1015F0000120704785EB113F000020420100404070
:101600003433333F46FFC742BDBA984110B4014658
:101610000020DFF8C028654BD3F8144900EE104ACB
:10162000D1ED000AB4EE600AF1EE10FA08D1147898
:10163000641C1470E4B2FE2C04DB3224147001E04C
:101640000446147003F6141393ED010AD1ED010A58
:10165000B4EE600AF1EE10FA08D15478641C5470AC
:10166000E4B2FE2C04DB3224547001E004465470D2
:1016700093ED020AD1ED020AB4EE600AF1EE10FA1F
:1016800008D19178491C9170C9B2FE2904DB32213E
:10169000917001E0014691701178322905DA517894
:1016A000322902DA9178322900DB012010BC704720
:1016B000010060400100A04001007041014600208F
:1016C00091ED000AB5EE400AF1EE10FA01DCB1EE40
:1016D000400ADFF80028DFED340AB4EE600AF1EECC
:1016E00010FA08DBD3785B1CD370DBB2FE2B04DB73
:1016F0003223D37001E00346D37091ED010AB5EEB9
:10170000400AF1EE10FA01DCB1EE400AB4EE600AD4
:10171000F1EE10FA08DB13795B1C1371DBB2FE2BC0
:1017200004DB3223137101E00346137191ED020AC9
:10173000B5EE400AF1EE10FA01DCB1EE400AB4EE6B
:10174000600AF1EE10FA08DB5179491C5171C9B2F7
:10175000FE2904DB3221517101E001465171D1783B
:10176000322905DA1179322902DA5179322900DB7E
:1017700001207047DFF89C0CC0697047DFF8940CBB
:10178000006970479A99993E01009040010080409D
:101790000000C8430000164301008C427C60030037
:1017A0008096184BA8BB030035336B418869030052
:1017B0002DE9F84F2DED068B86B0814688464FF017
:1017C000000A9FEDD88ADFEDD78A9FEDD69ADFED2C
:1017D000D59ADFF8444CE088ADF81000A088ADF849
:1017E00002002089ADF800005046019005464846A9
:1017F000FFF70CFF03904846FFF760FF0290DFF809
:10180000D06628467065B0653081B06EDFF80C7C1C
:10181000D7F8141900EE101AD9ED000A30EEC01AEC
:1018200001EE900AF8EEE11A21EE211AB5EE401A07
:10183000F1EE10FA1BD596ED1D1A70EE411AF5EE79
:10184000401AF1EE10FA01DC71EE401A9FEDB61A63
:10185000F4EE411AF1EE10FA05DB216F491C216705
:10186000F16D491CF16586ED1D0A4042B06607F630
:10187000141090ED010AF16E99ED011A31EE401A43
:1018800001EE901AF8EEE11A21EE211AB5EE401A97
:10189000F1EE10FA1BD596ED1E1A70EE411AF5EE18
:1018A000401AF1EE10FA01DC71EE401A9FED9E1A1B
:1018B000F4EE411AF1EE10FA05DB226F521C22679A
:1018C000326E521C326686ED1E0A4942F16690ED78
:1018D000020A306F99ED021A31EE401A01EE900AB9
:1018E000F8EEE11A21EE211AB5EE401AF1EE10FAE7
:1018F0001BD596ED1F1A70EE411AF5EE401AF1EE67
:1019000010FA01DC71EE401A9FED871AF4EE411ACD
:10191000F1EE10FA05DB216F491C2167716E491C3D
:10192000716686ED1F0A404230673078052805D180
:1019300001203064284630707080B080F06C4044E4
:10194000F064706B716C884201D101203064B06B1F
:1019500000EB400107EB810B0BF6C000C0ED000A65
:10196000D9F804104160D9F8081081604146484612
:1019700000F0B2FA2061DFF85C850398012802D0FC
:101980000298012836D19FED670ADBF8C00800EE07
:10199000900A60EEA00ADBF8C40801EE100A21EEFE
:1019A000011ADBF8C80801EE900A61EEA11A98F856
:1019B0000000322805DA98F80300322801DA30EE08
:1019C000800A98F80100322805DA98F804003228D5
:1019D00001DA30EE010A98F80200322805DA98F8A8
:1019E0000500322801DA30EE210A00F025FDB0EEC4
:1019F00040AA37E00BF50C60D0ED020A90ED011A19
:101A0000DBF8C00800EE100A20EE000A01EE010A21
:101A100000EEA00A00F010FDB0EE40AAD9ED010AD8
:101A200099ED000A20EE000A00EEA00A00F004FD85
:101A3000F0EE408AD9ED020A99ED010A20EE000A83
:101A400000EEA00A00F0F8FCB0EE409AD9ED020AD0
:101A500099ED000A20EE000A00EEA00A00F0ECFC6E
:101A6000F0EE409AF06B002824D128460CE007EBFA
:101A7000800181ED15AA07EB8002C2ED008A81ED9D
:101A8000079AC1ED0E9A401C0728F0DBF068B061A0
:101A90003069F06170693062B1EE0C0A68EE800A5C
:101AA000C6ED030A69EE000AC6ED040A29EE800AB3
:101AB00086ED050AB06B07EB800181ED15AA07E002
:101AC00007EB8A0090ED150A38EE008A0AF1010A48
:101AD000BAF1070FF4DB86ED098A96ED090A706BFF
:101AE00007EB800080ED230AD6ED0B0A70EE800A2A
:101AF000C6ED0B0AF268B2613269F2617269326254
:101B0000B26B07EB8202C2ED008A81ED079AC1ED4C
:101B10000E9A2A46DFED030A9FED021ADFED011A45
:101B200013E000BF00000000CECC4C3E07EB820368
:101B300093ED002A70EE820A93ED072A31EE021A25
:101B400093ED0E2A71EE821A521C072AEEDBC6EDC7
:101B5000030A86ED041AC6ED051AD1ED1C0A70EED3
:101B6000600A00F27442C2ED000A81ED1C0AD6ED53
:101B70000C0AD0F8742401EE102A70EE810AC6ED2A
:101B80000C0AD9ED000AF5EE400AF1EE10FA01DC7C
:101B9000F1EE600A9FEDCB1AF4EE410AF1EE10FA75
:101BA0001BDAD9ED010AF5EE400AF1EE10FA01DC7C
:101BB000F1EE600AF4EE410AF1EE10FA0DDAD9ED19
:101BC000020AF5EE400AF1EE10FA01DCF1EE600ACD
:101BD000F4EE410AF1EE10FA08DB0122C8F81C20ED
:101BE000D8F8102042F00102C8F81020B4EE41AA43
:101BF000F1EE10FA04DAB5EE40AAF1EE10FA08D5CB
:101C00000122C8F81C20D8F8102042F00202C8F8BF
:101C10001020B5EE400AF1EE10FA08D50122C8F8FE
:101C20001C20D8F8102042F00402C8F810209FEDC4
:101C3000A60AD1ED1C0AF4EE400AF1EE10FA08DB18
:101C40000121C8F81C10D8F8101041F00801C8F89C
:101C50001010D0ED230AF4EE400AF1EE10FA08DB82
:101C60000121C8F81C10D8F8101041F01001C8F874
:101C70001010D0F8741400EE101AD8ED050AF4EE26
:101C8000400AF1EE10FA10D1D8F81810491CC8F823
:101C90001810FB290CDB0121C8F81C10D8F8101013
:101CA00041F02001C8F8101002E02946C8F81810C9
:101CB00088ED050AD8F81C10012901D12846FCE05E
:101CC00007F6141199EC030A81EC030AD8F8701096
:101CD000012906D101203064284630707080B08020
:101CE0007CE0316D491C31653278012A01D0032A2C
:101CF00037D102292AD2628D042A27DAE16C002921
:101D00006CD196ED0A0ADFEDD70AB4EE600AF1EE67
:101D100010FA08D5D0F8741401EE101AB4EE601A57
:101D2000F1EE10FA0FDAF9EE0C0AB4EE600AF1EEF9
:101D300010FA53DBD0F8740400EE100AB4EE600A17
:101D4000F1EE10FA4AD50120306447E0272908D384
:101D50007288002A03D011FA82F14B2901D30121A4
:101D60003164D0F8740400EE900A96ED0A0A00F08F
:101D70007BF9D8F87400401CC8F87400FB2805DB18
:101D80000120307030647080B08030653078012878
:101D900024D17088002821D0B18800291ED00322C8
:101DA00011FA80F03D2801DB01203064608D0428A9
:101DB00000DB0222F088824201D2012030642846F2
:101DC00070663066F065FEF727FA0190206F606755
:101DD00028462067B080F080C8F87400706BB16C42
:101DE000401AFA304FF0FA084146B0FBF1F108FB17
:101DF00011007189884201D100F037FA706BB16C23
:101E0000401AFA304146B0FBF1F108FB110064289A
:101E100001D100F06BFAE088BDF81010814204D1C6
:101E2000BDF80210A288914200D00125002812D0EE
:101E3000706BB16C401AFA304146B0FBF1F108FB0F
:101E40001101322902D10120208114E04B2912D145
:101E5000002020810FE0A08800280CD0706BB16CAE
:101E6000401AFA304146B0FBF1F108FB11007D2821
:101E700001D101202081BDF800002189884200D0D5
:101E80000125706B07EB8001D1F87414B162401C1E
:101E90007063FA2801D100207063B06B401CB063FE
:101EA000072801D10020B063F06B401CF06301985B
:101EB0002843401E8041C043C00F06B0BDEC068BD6
:101EC000BDE8F28FC4F51C430C578944D46103006C
:101ED000FC5F0300FC60030010B4DFF8402590EDC8
:101EE000000AD2F8143900EE903A30EE600A02F699
:101EF0001413D0ED010A93ED011A70EEC10A90EDB2
:101F0000021AD3ED021A31EE611AB5EE400AF1EE73
:101F100010FA02DDF0EE401A01E0F1EE401AF5EEA3
:101F2000400AF1EE10FA02DDB0EE602A01E0B1EEF7
:101F3000602AB5EE401AF1EE10FA02DDF0EE412A09
:101F400001E0F1EE412A71EE821A71EEA21AB5EEAD
:101F5000400AF1EE10FA01DCB1EE400ADFF8B404F9
:101F600090ED082A32EE000A80ED080AF5EE400AEC
:101F7000F1EE10FA01DCF1EE600A90ED090A30EEA4
:101F8000200A80ED090AB5EE401AF1EE10FA01DCE4
:101F9000B1EE411A90ED0A0A30EE010A80ED0A0A0C
:101FA00090ED0B0A30EE210A80ED0B0ADFF8703459
:101FB000DB6B002B12D1002306E002EB840404F655
:101FC0007C04C4ED001A5B1C9BB21C460F2CF4DB96
:101FD000B2EE0E0A21EE800A80ED150A038902EBAB
:101FE0008302D2F87C4800EE104A31EEC00AD0EDF0
:101FF000150A30EE200A80ED150A02F67C02C2EDC9
:10200000001AF2EE0E0A80EE200ADFF80C2482EDB0
:102010001B0AD0ED170AB4EE600AF1EE10FA01D5F2
:1020200080ED170AD0ED180AF4EE400AF1EE10FA2E
:1020300001D580ED180ADFEDAB0AB4EE600AF1EECF
:1020400010FA03D5826D8918816501E00021816550
:10205000591C018189B20F2901D100210181806DB4
:1020600010BC70470100E0409FED9F1ADFF8A80305
:10207000408D042801DBB0EE001ADFF8A403B5EEB2
:10208000400AF1EE10FA07DBF5EE400AF1EE10FA25
:1020900002D5C188491CC1800178002905D00229D8
:1020A00060D02DD3032976D0B0E0F1EE0C1A31EEDA
:1020B000211AB4EE401AF1EE10FA0BDBB4EE601AFE
:1020C000F1EE10FA06D5016D1029C0F08F800021C5
:1020D00001658BE0416BDFF8442302EB8101D1F80D
:1020E000741401EE901ADFF83C1391ED010AF4EE3E
:1020F000401AF1EE10FA40F18980C1ED011A85E035
:10210000416BDFF8182302EB8101D1F8741401EE62
:10211000901ADFF8101391ED002AB4EE612AF1EE67
:1021200010FA01D5C1ED001AF7EE001AB4EE610AFB
:10213000F1EE10FA6ADBB7EE000AF4EE400AF1EEB7
:1021400010FA63D5016D418000210165B9EE0C0ADA
:1021500030EE410AF4EE400AF1EE10FA10D40221FA
:10216000017053E0F9EE0C1A31EEC11AB4EE410AD7
:10217000F1EE10FA4ADBF4EE410AF1EE10FA45D521
:1021800003210170A549426B01EB8201D1F874145F
:10219000A44A51603AE0416BA04A02EB8101D1F8B8
:1021A000741401EE901A9F4991ED012AF4EE421A3F
:1021B000F1EE10FA01D5C1ED011ADFED831AB4EE8C
:1021C000610AF1EE10FA21D5F4EE610AF1EE10FA8F
:1021D0001CDB016D818000210165B1EE0C0A31EE3E
:1021E000000AB4EE600AF1EE10FA0ED5012101707A
:1021F0008C490A6842654A688265884A436B02EBEB
:102200008302D2F874240A6000E0017000787047FD
:1022100000280CD0C168804AD160916490ED070A13
:1022200082ED070A406A506282ED180A9066704794
:10223000002803D07849282200F058B970470028B8
:1022400006D0794942684A6002680A60007A0872DA
:10225000704780B5002801D1002002BD54220146FC
:10226000724800F043F9012002BD10B56A4C608D40
:10227000218D002904D0002802D00020208106E012
:10228000084302D00120208101E0022020810020AB
:10229000E06420626061A0802085E0626065A065E6
:1022A00002464021624800F0E3F8E06F012801D1C6
:1022B000FEF78EFC57484189002909D0628E8A4278
:1022C00001D2218600E02286002141810846A067D4
:1022D000A06F012801D1608E20860020A06710BD6C
:1022E00000000000EC51383E0000000010B54A4CE0
:1022F000608D218D002904D0002802D0002020818B
:1023000006E0084302D00120208101E00220208164
:102310000020206260616085E08002460821454817
:1023200000F0A6F80020E062E06F012801D1FEF77E
:102330004FFCA06F012801D1608E208610BD80B5B2
:10234000012034490867FFF7D1FFFFF78EFFBDE892
:10235000014003E000202F49086770472D48C089DD
:102360002D49098E814200D200E070472A49CA6C8B
:102370000B8E9A4203D20886002088677047254951
:10238000488170472448C16C002904D1818DC08DDB
:1023900010FA81F0704700207047014600200029A4
:1023A00002D0012901D0704702E01B48C06C704781
:1023B0001948018EC26C891A828D891AC08D081A3B
:1023C00000D5002070470000FEFF7FBF38B50446EF
:1023D0001348104D1049012C06D106224A860C22C2
:1023E000EA819622428105E007224A860F22EA818D
:1023F00064224281A889A04209D0088E082803DA05
:10240000488EFFF7B3FF02E0E889FFF7AFFFAC812A
:1024100031BD0000FC6003007C600300886903009C
:10242000FC5F030058C20300A8BB0300D461030093
:10243000B4BB03004072030081B08DED000A009828
:10244000401000F1FE500090DDED000AC0EE200AC1
:102450009DED001A70EE810ACDED000AB5EE001A6E
:10246000DDED001A80EE210A00EE810A01B070470E
:1024700062F30F2262F31F4200B500BF13009646BD
:102480009446103928BFA0E80C50FAD85FEA417C86
:1024900028BF0CC048BF40F8042BC90728BF20F84C
:1024A000022B48BF00F8012B00BD50F8041B61B19E
:1024B00050F8042BD30744BFA9F101039A18002355
:1024C000091F42F8043BFAD1EFE7704762B38B076C
:1024D00008D0521E11F8013B00F8013B00F02480A7
:1024E0008B07F6D1830740F0208000BF103A07D356
:1024F00030B4B1E83810103AA0E83810F9D230BC46
:10250000530724BFB1E80810A0E8081044BF51F8F1
:10251000043B40F8043BD20724BF31F8022B20F8DB
:10252000022B44BF0B7803707047083A07D3B1E819
:102530000810083A40F8043B40F804CBF7D25307A0
:10254000E4E78268521C8260426832B10268531C20
:10255000036011704168491E416070470022FFF717
:102560008BBF000062F30F2262F31F42401810F08D
:10257000030308D0C91A1FD3DB0748BF00F8012D99
:1025800028BF20F8022D130030B414461546103928
:1025900028BF20E93C00FAD8490728BF20E90C00F1
:1025A00048BF40F8042D890028BF20F8022D48BFFD
:1025B00000F8012D30BC7047C91818BF00F8012D74
:1025C000CB0728BF00F8012D7047000010B50FF2AF
:1025D000740001F081FBDFF8844C0020A073208799
:1025E000E06502464021DFF8980DFFF741FF012228
:1025F0003C21AA2001F02CFE00206074E07302460A
:1026000004F18001012002F085FB002805D00FF2C3
:10261000440001F061FB032010BD002204F18C0195
:10262000BC2002F077FB002805D00FF2340001F047
:1026300053FB032010BDBC2002F08FFC606500201E
:1026400010BD000050443A53746172743230303916
:102650003134000050443A45525241434300000097
:1026600050443A45525256480000000010B5DFF879
:10267000EC4B002204F18001012002F0A7FB0028AE
:1026800005D00FF22C0001F027FB032010BD002223
:1026900004F18C01BC2002F099FB002805D00FF258
:1026A000200001F019FB032010BD002010BD000028
:1026B00050443A4552524143434F464600000000C1
:1026C00050443A45525256484F4646002DE9F84F7D
:1026D0002DED028BA4B003F00FF8DFF8C42C00231B
:1026E00003F026F806460F46DFF8704BD4E91001D8
:1026F000A6EB00080EA81421FFF730FF0FF27810A8
:1027000090ED008A03F020F9451EAD41ED0F0EA9B2
:10271000012003F018FC207AA84200D02572832003
:1027200002F0D8FD0546B8F1140000D54042032858
:1027300015DBA16F491CA167322291FBF2F2322313
:1027400003FB1211002901D00B2808DBCDE900673B
:10275000D4E9102341460FF2241001F0BDFA606F56
:1027600040446067E06E804500DC4046E066206FD4
:10277000404500DA4046206701950EA984B06846BE
:102780001422FFF7B3FE0FBCB0EE480A01F0D1FBF4
:10279000A06D2818A065A06E401CA06641F2717162
:1027A000884259DBD4E91201A6EB000B206D416A87
:1027B000002901D0012500E0002590F828A0606DD7
:1027C000002802D14FF0FF3801E090F9288003F093
:1027D000BBF8814613A84021FFF7C0FE0FF2B402F8
:1027E000D2E90001CDE90C010CA803F013F913A8FC
:1027F00001F0EAFCE16F481CE06716980B9094F931
:102800000D000A9094F90C000990A06D089094F9BD
:1028100009000790CDF818800595CDF810A0CDF8E7
:102820000C90CDF808B0BDF9340001909DF932004C
:1028300000909DF931309DF930200FF2600001F0D9
:102840004BFAC4E912670020A066606742F210707C
:10285000E06600202067A06794F9080000F0E0FA25
:10286000002801D000F0D7F8C4E91067002024B098
:10287000BDEC028BBDE8F28F00007A4450443A531D
:10288000544552522825642920256C6C6420256CFF
:102890006C640A00000000000000000050443A2070
:1028A0005B25755D25643A25643A25643A256420E4
:1028B000747325642C6C636425642C7265662874BB
:1028C00025642C6525642C76256429202564202523
:1028D000642C25642C25642C25640A0010B5DFF8CF
:1028E0007C4994F9000000283AD494F90B0094F93B
:1028F0000110814228D1617B0818E07240B23D2866
:1029000001DB3C38E07294F90B100FF2700001F01B
:10291000E3F90020A065DFF8C00C90F90100014642
:1029200011F1010F01D1012010BD94F90120511ABC
:10293000012901DB101A00E0801A40B2012801DBF6
:10294000012010BD002010BDDFF8900C90F901208F
:10295000914203D0D4E90023C0E90023002010BD38
:10296000A06DDFF80C1D884205DB0FF2180001F0A6
:10297000B3F9012010BD002010BD000050443A4EB4
:102980005425640050443A4E6F54696D6500000050
:1029900010B40020DFF8C41802E04B7B9A18CA720A
:1029A00091F90B20002811D44878801A40B20128F0
:1029B000F3DA00280AD0030000D55B4291F90D40FC
:1029C0009C42EDDA101BC8720020E9E73C2A02DBCA
:1029D000A2F13C00C87210BC704780B5DFF87C08DB
:1029E0000021C17301214172002181724FF0FF313A
:1029F00001700F210173142141730021817301873C
:102A0000C1658174016641660A4624211430FFF7CE
:102A10002FFD002002BD30B5A5B00AA85821FFF750
:102A20009DFD00A82821FFF799FD20A81421FFF79C
:102A300095FD0AA800F024FEDFF8384C9DF8290027
:102A400020709DF82900C02806D113A9C88DA4F8CC
:102A50005E00086B206694E0000633D49DF82A00DF
:102A60008DF8800020A89DF82B1041700021817006
:102A70009DF82C10C170BDF833100A0A0271417123
:102A80000DF133018A788271C978C1719DF83710D0
:102A900001729DF8381041729DF82D1081729DF8D9
:102AA0002E10C1729DF82F1001739DF830104173E4
:102AB0000E2220A9601CFFF709FD0F20A4F85E007C
:102AC00024665EE0DDF82A10080C8DF8000000A8EE
:102AD0000A0A42708170DDF82E100A0CC2700A0AD0
:102AE00002714171DDF832100A0C82710A0AC2715A
:102AF0000172DDF836100A0C42720A0A8272C17243
:102B000013990A0C02730A0A4273817313A90A7992
:102B1000C2734A790274CA88130A8DF8113082741C
:102B2000097A8DF81310DDF83A100A0C8DF814208C
:102B30000A0A8DF815208175DDF83E100A0C8DF813
:102B400017200A0A8DF818208DF81910DDF84210A8
:102B50000A0C82760A0A8DF81B208DF81C10DDF80D
:102B600046100A0C8DF81D200A0A82778DF81F1076
:102B7000202200A9601CFFF7A9FC2120A4F85E0018
:102B80002466B4F85E20D01CDFF8D016096D4882A8
:102B9000DFF8E85A0120287068700320A870216EC1
:102BA000E81CFFF793FC2946832003F0DFF825B0EB
:102BB00030BD38B5DFF8A4364FF46164C1EB0115C0
:102BC000AD0014FB005414194FF47A756C43DC61AA
:102BD0005B7C009313460A4601460FF20C0001F09D
:102BE0007BF831BD0000000050443A425425643A5D
:102BF00025643A25642C282564290000F8B52DEDBC
:102C0000028B9EB0DFF87867314684B06846402278
:102C1000FFF76CFC0FBC00F0E3FC10EE100A03F0B1
:102C2000FBF941EC100B9FED7C8BDFF83046256AF9
:102C300053EC102B51EC180B03F016FA03F0E6FAE4
:102C400015FA80F020624FF6FF75A84200D3256286
:102C5000314684B068464022FFF748FC0FBC00F0C4
:102C600073FC10EE100A03F0D7F941EC100B676A01
:102C700053EC102B51EC180B03F0F6F903F0C6FAE5
:102C800017FA80F06062A84200D3656200200D90C0
:102C900002200C90314684B068464022FFF726FCA3
:102CA0000FBC00F0DDFAE18A4018E08280B2FF2814
:102CB00001DBFF20E08200200D9003200C903146C4
:102CC00084B068464022FFF711FC0FBC00F0C8FA40
:102CD000A16A4018A062A84200D3A56200200D900E
:102CE00006200C90314684B068464022FFF7FEFB78
:102CF0000FBC00F0B5FA218B4018208380B2FF286A
:102D000001DBFF20208300200D9007200C9031462E
:102D100084B068464022FFF7E9FB0FBC00F0A0FA40
:102D2000618B4018608380B2FF2801DBFF20608345
:102D300000200D9008200C90314684B06846402257
:102D4000FFF7D4FB0FBC00F08BFAE16A4018E06299
:102D5000A84200D3E56200200D9009200C90314676
:102D600084B068464022FFF7C1FB0FBC00F078FA40
:102D7000216B40182063A84200D325630EA801F000
:102D800023FA276E1C9803F047F90022DFF85C3D18
:102D900003F06AF903F03AFA57FA80F02066616EA0
:102DA000491C6166B0FBF1F0207500200D900120F8
:102DB0000C90314684B068464022FFF797FB0FBC69
:102DC00000F04EFA616B40186063A84200D365635F
:102DD000207C00F030FB1EB0BDEC028BF1BDDFF8B3
:102DE0007C04C18A002914D1816A002911D1018B88
:102DF00000290ED1418B00290BD1C16A002908D1CD
:102E0000016B002905D1406B401E8041C043C00FBB
:102E1000704701207047000000000000000059408A
:102E20002DE9F04F9FB0064600250EA801F0CCF921
:102E3000DFF82844E07B3146884204D0012E79D166
:102E4000284601F0D1FB28460D9001200C90DFF8B8
:102E5000301584B068464022FFF748FB0FBC00F0F5
:102E6000FFF907469DED1C0ADFF81405D0ED0E0AA8
:102E700030EE600A10EE100A03F0CEF82A46DFF8B2
:102E80006C3C03F0F1F803F0C1F981461FFA89F9AF
:102E9000DFF8EC044088BDF83A100A1AD2B2099261
:102EA000DFF8DC24D268119B9A4208D1884206D10F
:102EB000DFF8CC04C088BDF83E1088420ED000A8D0
:102EC00029460A460B460EC0119800901C980190A6
:102ED0001D98029000A9A42002F048FF002E3FD1C7
:102EE000002F03D1099850EA090000D001250020E5
:102EF000A0654FF0FF302070D4E90001DFF8DC2638
:102F0000C2E90001DFF8FC2CC2E90001DFF8C826A5
:102F1000C2E90001207BE072E07B002800F0AE8077
:102F20000020E073607C002800F0A8800120A074DD
:102F30000546A3E0002E11D1206D90F82810406ABC
:102F4000002801D0012200E02A46119B0FF2BC208C
:102F500000F0C2FE012001F047FB74E7284652E171
:102F60000FF2C022D2E90001CDE9050105A802F067
:102F700051FD94F9012094F900104FF47A704FF448
:102F800061684FF03C0B11FB08F312FB0B3394F913
:102F900002C043FA8CF3B4F904C000FB03C3BDF9CB
:102FA00018C09DF816A08DF801A09DF901A0CDF8DC
:102FB00020A09DF815A08DF800A09DF900A0CDF8E7
:102FC0001CA09DF914E01EFB08F81AFB0B88DDF825
:102FD00020A0D04400FB08C0F046414509D09DF92F
:102FE0000080424505D094F902809DF901A0D045AA
:102FF00001D1984210D2CDF810C0089803900798DC
:103000000290CDF804E0B4F90400009094F9023085
:103010000FF60C4000F060FE00F0AEF9002819D069
:10302000DDE90501C4E900012846A072D4E90001E8
:10303000DFF8A825C2E900011198009094F9023048
:1030400094F9012094F900100FF6F03000F044FEDE
:10305000FFF79EFCDDE90501C4E90001FFF73EFC36
:1030600000280BD0D4E90001DFF86C25C2E900018B
:10307000607C002801D00120A0740125012E07D119
:10308000E07B3146884203D0002000F041FAE6732D
:10309000012E56D1002F54D0DFF8688B207C617C44
:1030A00008430AD101206074D4E90001C8E9020193
:1030B000A27861782078FFF77CFD94F9010098F9F7
:1030C0000910401A411E222901D2012005E010F109
:1030D000230F01DA012000E0002001282AD1FFF7A8
:1030E0007EFE002826D0207C401C2074C0B215280B
:1030F00009D10FF6643000F0EFFD0120A074142018
:103100002074012516E00020206660660246242116
:1031100004F11400FFF7ACF9607C401C6074A278E5
:1031200061782078FFF745FD0622214608F1080066
:10313000FFF7DCF9FFF762FD40220EA99048FFF788
:10314000D5F9A07B012828D1208F002801D10125A5
:103150001CE0E16D814215D2002F03D1099850EA9D
:10316000090000D00125DFF89C8A98F9020094F943
:10317000022090420AD0481CE065D4E90001C8E969
:10318000000103E00020A0732087E065012E04D138
:10319000607C002801D00120A0742846012801D1BC
:1031A0000021A165216D496A00292BD10021A1656B
:1031B000012826D10FF6AC20D0E90023CDE9042365
:1031C00004A802F027FC022000F0A2F9119CDFF80D
:1031D000348AD8F81000201A0B2812D31B9802F05A
:1031E0001BFFCDE9020100949DF912309DF91120D9
:1031F0009DF910100FF6742000F06EFD1198C8F8BC
:103200001000002528461FB0BDE8F08F50443A6CEE
:1032100063646F6E2063256420652564202825641F
:1032200029000000000000000000000080B5002020
:10323000DFF8B819886500F002F8002002BD00B57B
:1032400091B000A800F0C0FF402200A9DFF8A0095B
:10325000FFF74CF9012011B000BD0000B05E030083
:103260000FB410B590B000249DF98C0001280BD14B
:1032700001F060F81599884202D3441AE4B271E073
:103280008038441AE4B26DE000A800F09DFF9DF97B
:103290008800401E082865D8DFE800F02905111DC8
:1032A0002935414D590004981699884201D3441A92
:1032B00058E0DFF854291018401A441C52E00598D1
:1032C0001799884201D3441A4CE0DFF83C291018C2
:1032D000401A441C46E006981899884201D3441AC3
:1032E00040E0DFF824291018401A441C3AE0039803
:1032F0001599884201D3441A34E0DFF80C291018DC
:10330000401A441C2EE007981999884201D3441AA8
:1033100028E0DFF8F4281018401A441C22E008982E
:103320001A99884201D3441A1CE0DFF8DC281018EF
:10333000401A441C16E009981B99884201D3441A8C
:1033400010E0DFF8C4281018401A441C0AE00A985C
:103350001C99884201D3441A04E0DFF8AC28101805
:10336000401A441C204610B010BC5DF814FB01202C
:10337000DFF8781888727047DFF87008807A704735
:10338000E0BD030000F029BFDFF86018792802DBF8
:103390007820088700E008870120887370470000C4
:1033A00040420F0010B5040001D1012402E0072CB7
:1033B00000DB062421460FF6D00000F08DFC641ED1
:1033C000052C2DD8DFE804F0030A11181F26DFF8BA
:1033D0001C08372101733C21417321E0DFF80C0800
:1033E000192101731E2141731AE0DFF800080F2133
:1033F00001731421417313E0DFF8F0070A21017310
:103400000F2141730CE0DFF8E407072101730C2161
:10341000417305E0DFF8D407052101730A214173E8
:10342000DFF8C807017BC172BDE81040FFF7B0BAF2
:10343000DFF8A007704700EB80018800821CDFF8EE
:103440009407DFF8A817CB691B0E92B21354521CD5
:10345000CB691B0C92B21354521CCB691B0A92B25B
:103460001354521CCB6992B21354521C0B6A1B0AA0
:1034700092B21354521C0B6A92B21354521C4B6AF0
:103480001B0A92B21354521C4B6A92B21354521C30
:10349000CB8A92B21354521C8B6A1B0A92B21354F9
:1034A000521C8B6A92B21354521C0B8B92B213545F
:1034B000521C4B8B92B21354521CCB6A1B0A92B211
:1034C0001354521CCB6A92B21354521C0B6B1B0A3E
:1034D00092B21354521C0B6B92B21354521C0B7DBC
:1034E00092B21354521C4B6B1B0A92B21354521CCF
:1034F0004B6B92B21354501C4887704710B5DFF8DD
:10350000EC46618F0FF2887000F0E6FB608F10BD13
:1035100010B5DFF8D846012807DB627C002A04D00A
:1035200001460FF27C7000F0D7FB0022242104F149
:103530001400FEF79DFF002020740120608700200A
:1035400060742066606610BD0FB400B591B000A82D
:1035500000F03AFE9DED0B0ADDED1D0AB4EE600AA7
:10356000F1EE10FA02DB30EE600A05E09FED421A40
:1035700071EE600A30EE800A10EE100A02F04CFD87
:10358000DFF85426DFF8543602F06CFE02F0DEFE5F
:1035900002F042FD0022DFF8483602F065FD02F03D
:1035A00035FE00EE100AB8EEC00A10EE100A02F066
:1035B00033FDDFF82426DFF82C3602F055FDDFF866
:1035C0002826DFF8483602F04DFE02F0BFFE00EE7E
:1035D000100A11B05DF814FB50C2030048C203008A
:1035E0000FB400B591B000A800F0EEFD9DED0D0AFE
:1035F000DDED1F0AB4EE600AF1EE10FA02DB30EEE8
:10360000600A05E09FED1C1A71EE600A30EE800A38
:1036100010EE100A02F000FDDFF8BC25DFF8BC3523
:1036200002F020FE02F092FE02F0F6FC0022DFF82B
:10363000B03502F019FD02F0E9FD00EE100AB8EE17
:10364000C00A10EE100A02F0E7FCDFF88C25DFF864
:10365000943502F009FDDFF89025DFF8B03502F06F
:1036600001FE02F073FE00EE100A11B05DF814FBCB
:1036700040771B0074BA030000247449C4A80300F7
:1036800070B52DED068B9EB004460EA800F09CFD93
:10369000DFF85855A87B012804D1288F002801D1D4
:1036A0000020A873A87C012817D1687C002814D0BA
:1036B000C0216170DFF81C15C0220A70487004F147
:1036C0002406FFF71BFFF085FFF7B2FE30630120F1
:1036D000FFF71EFF0020A874A4E19FEDD48B9FED9F
:1036E000D59BDFF80C5500200D9001200C90294649
:1036F00084B068464022FEF7F9FE0FBCFFF7B0FD2C
:103700000A2880F0BE80002060700D9002200C908E
:10371000294684B068464022FEF7E8FE0FBCFFF75A
:103720009FFD61780843607000200D9003200C908D
:10373000294684B068464022FEF7D8FE0FBCFFF74A
:103740008FFDA07000200D9004200C90294684B0BD
:1037500068464022FEF7CAFE0FBCFFF781FDE0700D
:1037600000200D9005200C90294684B06846402228
:10377000FEF7BCFE0FBCFFF773FD2071294684B035
:1037800068464022FEF7B2FE0FBCFFF729FF10EE9D
:10379000100A02F041FC41EC100B53EC102B51ECE1
:1037A000190B02F061FC02F031FDA4F80B0004F1EA
:1037B0000B061C9802F030FC53EC182B02F054FC62
:1037C00002F024FDB070BDF83A00F070294684B0D4
:1037D00068464022FEF78AFE0FBCFFF7B5FE10EEEA
:1037E000100A02F019FC41EC1A0B53EC1A2B51ECA5
:1037F000190B02F039FC02F009FDE0731D9802F08C
:103800000BFC53EC182B02F02FFC02F0FFFC207491
:1038100000200D9006200C90294684B06846402276
:10382000FEF764FE0FBCFFF71BFD607100200D90DA
:1038300007200C90294684B068464022FEF756FEC9
:103840000FBCFFF70DFDA07100200D9008200C901B
:10385000294684B068464022FEF748FE0FBCFFF7B9
:10386000FFFCE07100200D9009200C90294684B0E7
:1038700068464022FEF73AFE0FBCFFF7F1FC2072CB
:10388000CEE08020607000200D9002200C90294630
:1038900084B068464022FEF729FE0FBCFFF7E0FC2B
:1038A000C4F8020000200D9003200C90294684B03B
:1038B00068464022FEF71AFE0FBCFFF7D1FCC4F8A1
:1038C000060000200D9004200C90294684B0684624
:1038D0004022FEF70BFE0FBCFFF7C2FCC4F80A0043
:1038E00000200D9005200C90294684B068464022A7
:1038F000FEF7FCFD0FBCFFF7B3FCC4F80E00294631
:1039000084B068464022FEF7F1FD0FBCFFF768FE69
:1039100010EE100A02F080FB41EC100B53EC102B60
:1039200051EC190B02F0A0FB02F086FC606204F17E
:1039300024061C9802F070FB53EC182B02F094FB49
:1039400002F064FC3071BDF83A007071294684B011
:1039500068464022FEF7CAFD0FBCFFF7F5FD10EEEA
:10396000100A02F059FB41EC1A0BA24AA24B02F0DA
:1039700035FD06D8A14AA24B02F048FD01D29FEDC9
:10398000A4AB53EC1A2B51EC180B02F06DFB02F0B8
:103990003DFCF0801D9802F03FFB53EC182B02F029
:1039A00063FB02F033FC307200200D9006200C9077
:1039B000294684B068464022FEF798FD0FBCFFF709
:1039C0004FFCC4F8120000200D9007200C902946EF
:1039D00084B068464022FEF789FD0FBCFFF740FC2B
:1039E000C4F8160000200D9008200C90294684B0E1
:1039F00068464022FEF77AFD0FBCFFF731FCC4F8A1
:103A00001A0000200D9009200C90294684B06846C9
:103A10004022FEF76BFD0FBCFFF722FCC4F81E002E
:103A2000FFF70DFC1EB0BDEC068B70BD0000000062
:103A300000002440000000000000594010B596B07E
:103A400004460020002C05D10FF26C2000F044F950
:103A5000002048E004F15001497801293CD101A837
:103A60005421FEF77BFD0020ADF8000013E000EECE
:103A7000102AB8EE400ADFED680A20EE200A01A8FD
:103A8000BDF8001000EB810080ED000ABDF80000D9
:103A9000401CADF80000BDF80000142816DABDF88F
:103AA000000054F82020A2F52F70B0F5167FDED963
:103AB000BDF800100FF2102000F00EF901A8BDF8BB
:103AC00000104FF07E5240F82120DFE701201590D2
:103AD00001A800F08BFD05E0022903D194F8500005
:103AE0000120C046C0B216B010BD00000000244046
:103AF00080B5112802D11078FFF746FC002002BDE6
:103B000010B596B01446102826D0142811D01528C8
:103B100014D0162817D017281AD0292806D03D28E7
:103B200043D1002C41D0FFF781FB3EE0FFF71FFCA3
:103B30003BE021780020FFF725FC36E021780120CA
:103B4000FFF720FC31E021780220FFF71BFC2CE07E
:103B50002078FFF727FC28E000A85421FEF7FEFCA0
:103B6000207814A94870012817D100200FE004EB39
:103B700080014A788B781B0403EB0262CB7802EB5E
:103B800003220979511800AA42F82010401C142879
:103B9000EDDB00A8FFF752FF07E0022805D16078AF
:103BA0008DF8500000A8FFF749FF002016B010BDA7
:103BB0000E4908659831C16183210170142181602B
:103BC00001210173018200214182144941610020D9
:103BD000704700008CAA03007B14AE47E17A743F63
:103BE00000005940E17A843F2D431CEBB05E030096
:103BF000E0BD0300B81E85EB51B89E3F9A99999994
:103C00009999B93F1CC0030080969800E2361A3F8C
:103C10009A9999999999B93F6F12833AC4A8030068
:103C200050443A2025643A25643A25642E25643EA2
:103C300025643A25643A25642E25640050443A549C
:103C4000696D654E6F7469202564202564202564A4
:103C5000202825642900000050443A425446554C1F
:103C60004C000000000000000000000050443A2515
:103C7000643A25643A25642065783020282564203C
:103C8000252E32662900000050443A555425640020
:103C900050443A4241544C454E4754482025640014
:103CA00050443A436C6561726261746368282564AC
:103CB0002C636E742564290050443A5346205054B6
:103CC0005233206E756C6C0050443A534645525244
:103CD0005B25642C25645D000EB470B5C1B004464C
:103CE00000A84FF48071FEF739FC45AB22464FF433
:103CF000807100A802F0A2FB00A802F0BDFB441CEA
:103D0000002000A9611801F8010C644D2878401CBE
:103D10002870802080F3118800BF00BF6878401CA5
:103D200068705F4E317808462218FA2A0DDA5D4A2B
:103D30008018002902D00A2100F8011C224600A99F
:103D4000FEF7C4FB3078201830706878401E687029
:103D5000C0B2002802D1002080F3118802F0C8FC14
:103D600041B070BC5DF810FB4D480078002801D0D0
:103D7000801C00E00020C0B2704738B5484C227863
:103D8000002A10D000280ED0032101704270454D4A
:103D90002946801CFEF79AFB0022FA212846FEF7EE
:103DA00067FB0020207031BDF0B595B004A80FF27C
:103DB000FC010CC90CC0922002F04EFD040004D19D
:103DC0000FF2F000FFF788FF65E000229221FEF776
:103DD000C9FB002517E000208DF802009DF80200C5
:103DE000002803D0C868019008690290306A002852
:103DF00001D0C0680390102200A904EB0510801CBC
:103E0000FEF764FB6D1C072D16DA04A82F5C3846FC
:103E100001F0A3F80600F5D000A81021FEF79EFBE4
:103E20008DF8007006F12000017A8DF801104168CC
:103E30000029D0D00120CFE70CA82021FEF78EFB6F
:103E4000194800680C9002F0B8FD0D9001F078FD63
:103E50008DF838000DF13A0001F0DCFD10A801F0FA
:103E6000B8FD20220CA904F17200FEF72FFB06A872
:103E70000FF24C011422FEF739FB9220ADF81B0023
:103E80003120207007206070214606A802F0B4FDA2
:103E9000204602F0F9FC15B0F0BD0000C06303003D
:103EA000AAC2030088B30300980F020001020405B0
:103EB00008108300524349206661696C00000000CD
:103EC00005000000000000000000000000000000ED
:103ED0000000000038B5DFF8A80A00880146102964
:103EE00008DA002806D0DFF89C4A04EB810041681C
:103EF000491C4160DFF88C4A2068401C2060B0F506
:103F0000617F15DB01250AE004EB85004268002A89
:103F100004D029460FF68C20FFF7DEFE6D1C102D15
:103F2000F2DB00224021201DFEF7A2FA00202060D3
:103F300031BD0FB42DE9F0472DED028B88B0DFF8CD
:103F4000484AB4F876A004F108050A27B5F91E001E
:103F500010FB07F0B5F92010A0EB010804F5BA76C4
:103F6000304603F0A1FC94F8740117FB00F7BFB2D0
:103F70002A2F18D10FFA88F8B8F1000F13D5B068BE
:103F800000280DD10120FEF708FA8046FEF7D7F988
:103F90000120B060424639460FF61420FFF79CFE20
:103FA0000120706023E0B068012807D1FEF7D2F944
:103FB0000020B0600FF61020FFF78EFE7068282FEB
:103FC0000DDB002806D1D4F8802039460FF60420F6
:103FD000FFF782FE01207060FEF7C0F907E00128BC
:103FE00003D10FF61020FFF777FE002070601298C3
:103FF00004909DED138A8DED058ADDED148ACDEDDB
:10400000068ADDF85C8004A890EC030A404600F0C4
:104010008AFCDFF8787995ED030ADDED120AB4EE3B
:10402000600AF1EE10FA30D195ED040AB4EE480AB8
:10403000F1EE10FA29D195ED050AB4EE680AF1EE19
:1040400010FA22D1F86900F10109C7F81C90B9F102
:10405000150F02D30020F8611FE0B9F1020F1CD345
:10406000686901F0D9FFCDE90201286901F0D4FFA8
:10407000CDE90001E86801F0CFFF02460B46494652
:104080000FF67C10FFF728FE07E00498E86005981B
:104090002861069868610020F861414604A8FDF790
:1040A00087FB804604F12000FEF7C2F8A8690128CA
:1040B00014D1F868401CF860FCF79DF804F120006A
:1040C000FEF7B6F8282204F1200104F14800FEF7BB
:1040D0000DFA0FF64010FFF7FFFD18E0FDF74AFB61
:1040E000012812D13869401C3861FDF747FB78611F
:1040F000FCF781F804F12000FEF78AF87A69396943
:104100000FF61810FFF7E8FD01E000F021F9B8699B
:10411000401CB861B0F5617F08DBFB687A693969DA
:104120000FF60810FFF7D8FD0020B861FFF7D2FEA8
:10413000BAF1000F40D0B4F8760000283CD1287ABC
:10414000DFF84C1894ED020ABDEEC00A10EE102AFA
:104150004FF47A735A4301FB002095ED010ABDEE3E
:10416000C00A10EE101A081841007A68BA603B685D
:104170007B60D4F8800038607869029038690190DB
:10418000386800900FF6B800FFF7A6FD04F180052F
:10419000B068039070680290286A01F03DFFCDE995
:1041A0000001A86A01F038FF02460B46D4F88010DF
:1041B0000FF6AC00FFF790FD404608B0BDEC028B57
:1041C000BDE8F0075DF814FB002805D0DFF8B8174C
:1041D000096F4022FEF78AB9704738B50C460500D2
:1041E0000BD1DFF8A40700EE104AB8EE400A80EDCC
:1041F000030A0830FEF723F815E0012D0BD1DFF894
:10420000880700EE104AB8EE400A80ED020A083036
:10421000FEF715F807E0022D05D1DFF86C070474EE
:104220000830FEF70CF80D2010FB04F229460FF6BB
:104230005000FFF751FD42F27470044640F2EF70F7
:10424000224601460FF64800BDE83840FFF744BD5E
:104250002DE9F8432DED028B84B007468846914640
:104260000FF63C00FFF738FD42F27470044640F24E
:10427000EF70224601460FF61800FFF72DFDDFF81C
:10428000084700224FF4C0712046FEF7F1F804F110
:10429000080504F1B406AE6600EE107AB8EE408A66
:1042A00085ED018A00EE108AB8EE400A84ED020A1C
:1042B00085F80890F2EE0A8A48460D2111FB00F0BD
:1042C000029020EE280A10EE100A01F0A5FECDE9BA
:1042D000000128EE280A10EE100A01F09DFE0246A9
:1042E0000B460FF2C870FFF7F7FCFBF7D9FE284624
:1042F000FDF7A5FF0020606704F174010220C8806B
:1043000028223046FEF7F2F80120607104F5BA70F9
:1043100003F0CAFA0020C4F87C01C4F87801024610
:104320003C2104F5C07004B0BDEC028BBDE8F8433D
:10433000FEF79EB810B590B0FEF724F8044600A82A
:10434000FFF742FF0398001910B010BD00000000F5
:104350002DE9F041DFF83046251DA86A616D8842DD
:1043600004D16A8CB4F84E309A4279D0B0EB01088F
:1043700002D5DFF82006804404F1540695ED100ABA
:10438000D6ED060A30EE600AB5EE400AF1EE10FAFC
:1043900003D5DFED940A30EE200AD5ED0E0A96ED36
:1043A000041A70EEC10AF5EE400AF1EE10FA03D5D8
:1043B0009FED8C1A70EE810A6878012802D00228DD
:1043C00027D02DE004F1F40739469FEDCA1A404684
:1043D00000F052F8207940442071C0B206281FDB5B
:1043E00004F5807004F174019FEDC21AD0ED0A0A41
:1043F00090ED080AD4F8000100F03EF82079401C46
:104400002071002240213846FEF732F80220687001
:1044100006E004F174019FEDB71A404600F02CF855
:10442000688C002809D10022402104F1F400FEF735
:104430001FF80020207101206870282204F120015B
:1044400004F14800FEF752F804F17400F06104F141
:10445000B407402204F174013846FEF747F8F761CB
:10446000A88CB4F8BA10884204D004F15406F08441
:10447000A4F8BA00BDE8F081F8B52DED028BF0EE9E
:10448000408AB0EE608AB0EE410A0C46DFF8F8547C
:10449000EE8CAF8CA68000F038F894ED0B0A30EE6D
:1044A000280A84ED0B0A00F075F884ED0B0A66808B
:1044B0002780A86B206394ED0D0A30EE080A84ED86
:1044C0000D0A00F047F884ED0D0A95ED100ADFEDB6
:1044D0008A0A20EE200A84ED0E0ADFED880AB4EE87
:1044E000600AF1EE10FA02DBDFF8AC04A063686B3F
:1044F000E0636088002801D10020E063286BA060A1
:10450000288DE080BDEC028BF1BD38B505460C4628
:10451000E0682818E06000F05CF8E060608803283C
:1045200002D0042807D00DE020692818206100F08F
:1045300050F8206131BD60692818606100F049F8C9
:10454000606131BD20692818206100F042F82061C7
:1045500031BD000080B52DED028BB0EE408A9FED9D
:10456000B10AB4EE408AF1EE10FA0DDB9FEDAE0A0F
:1045700038EE008A18EE100A01F04EFD02460B4696
:104580000FF23450FFF7A8FBB0EE480ABDEC028BE7
:1045900001BD000080B52DED028BB0EE408A9FED8D
:1045A000A10AB4EE408AF1EE10FA0DDB18EE100A03
:1045B00001F032FD02460B460FF20850FFF78CFB6C
:1045C0009FED990A38EE008AB0EE480ABDEC028BE6
:1045D00001BDDFF8C013884202D3DFF8C01308180A
:1045E0007047000000247449FDF7F0BEFDF731BEAE
:1045F0002DE9F8432DED048B8AB00446B0EE408AD5
:10460000F0EE608AB0EE419ADF4D05F5C27696ED88
:104610000B0AF0EE480AB4EE600AF1EE10FA05D18A
:10462000D5F884012018C5F8840102E00020C5F8FF
:104630008401F0EE689A96ED0C0AB4EE690AF1EE88
:1046400010FA03D170682018706001E000207060DB
:10465000B0EE490AD6ED0D0AF4EE400AF1EE10FA7A
:1046600003D1B0682018B06001E00020B060D6F837
:104670000480D5F8849140F6B837B94504DAB845D6
:1046800002DAB068B8422EDB10EE100A01F0C4FC6A
:10469000CDE90801B068069019EE900A01F0BCFC63
:1046A000CDE90401CDF80880B0EE480A10EE100AFA
:1046B00001F0B2FCCDE900014A4621460FF210405C
:1046C000FFF70AFBD5F88401B84202DB0020C5F8E9
:1046D00084017068B84201DB00207060B068B842A5
:1046E00001DB0020B0600AB0BDEC048BBDE8F183B3
:1046F00000000000000000008FC2753D0100C841AD
:104700002DE9F8432DED048B8AB00446B0EE408AC3
:10471000F0EE608AB0EE419AB5EE400AF1EE10FA82
:1047200001DCB1EE400A984DDFED940AB4EE600A68
:10473000F1EE10FA05DBD5F890012018C5F89001CC
:1047400002E00020C5F89001F0EE689AF5EE409A7C
:10475000F1EE10FA02DDB0EE690A01E0B1EE690A8D
:1047600005F5C876B4EE600AF1EE10FA03DB706866
:104770002018706001E000207060B0EE490AB5EECC
:10478000400AF1EE10FA01DCB1EE401AB4EE601A04
:10479000F1EE10FA03DBB0682018B06001E00020F1
:1047A000B060D6F80480D5F8909140F6B837B94596
:1047B00004DAB84502DAB068B8422EDB10EE100A0F
:1047C00001F02AFCCDE90801B068069019EE900AC4
:1047D00001F022FCCDE90401CDF80880B0EE480AD2
:1047E00010EE100A01F018FCCDE900014A462146FE
:1047F0000FF20030FFF770FAD5F89001B84202DBF3
:104800000020C5F890017068B84201DB002070609C
:10481000B068B84201DB0020B0600AB0BDEC048B88
:10482000BDE8F18301247449002474C970B52DEDED
:10483000088B8AB00646B0EE408AF0EE608AB0EE91
:10484000419AF0EE499AB0EE68AA20EE000A0AEE0C
:104850000A0A09EEA90AFDF7EFFD4B4CD4F89C01BA
:1048600004F5CE75002805D10021E9604C49A96006
:1048700000212961D5ED030AF4EE400AF1EE10FAA9
:1048800001D585ED030AD5ED020AB4EE600AF1EE1A
:1048900010FA01D585ED020AD5ED040A70EE80AA62
:1048A000C5ED04AA6968491C0BEE101A85ED01BA22
:1048B0003018C4F89C0147F2315188422FDB19EEC1
:1048C000900A01F0A9FBCDE908011AEE100A01F0E7
:1048D000A3FBCDE90601B0EE480A10EE100A01F084
:1048E0009BFBCDE90401E86801F096FBCDE90201EC
:1048F000A86801F091FBCDE90001B8EECB0A8AEE81
:10490000800A10EE100A01F087FB02460B460FF2F8
:104910000820FFF7E1F900206860C4F89C010AB0A4
:10492000BDEC088B70BD70B52DED048B0446B0EE68
:10493000408AF0EE608AB0EE419A134DB5F8766089
:10494000FFF756FEB0EE491AF0EE680AB0EE480ADC
:104950002046FFF7D5FEB0EE491AF0EE680AB0EE39
:10496000480A2046FFF762FF05F5D87080EC038AFD
:10497000A5F88061BDEC048B70BD000035336B4140
:1049800004600300D4BC030050AC030050C003001B
:1049900040420F00819698000000C841806967FF7F
:1049A00000007A4450443A462564282564290000D2
:1049B00050443A42504F4E205648282564292053EF
:1049C000746570282564290050443A42504F464689
:1049D0000000000050443A53746570436E74557083
:1049E00020564828256429205354455028256429F9
:1049F0000000000050443A45584954564800000011
:104A000050443A4E41435B25645D2025662025666F
:104A10002025660050443A4F4652000050443A5216
:104A2000432825642C2564290000000050443A5294
:104A3000432825642C2564292C4F46282564290009
:104A400050443A53532825642C25643E25643E2562
:104A500064292C52432825642C2564290A0000006F
:104A600050443A532825642C252E32662C252E32AC
:104A700066292C562825642C2564290A000000008C
:104A800050443A50555428256420256429000000DC
:104A900050443A5052497625642C4D7625640000E6
:104AA00050443A31345345503230000050443A2596
:104AB000662025662025640050443A446973744F8B
:104AC0006625660050443A43616C4F4625660000F7
:104AD00050443A45532825643A25642C252E3266E5
:104AE0002F25642C252E32662F25642C252E326628
:104AF0002900000050443A45462825643A25642C94
:104B0000252E32662F25642C252E32662F25642C07
:104B1000252E32662900000050443A4E43252E329D
:104B2000662C252E32662C252E32662F78252E32C5
:104B3000662C79252E32662C7A252E32660A0000E4
:104B40002DE9F04100242546DFF80C791EE0052010
:104B500000F0F8FC0020F16909688847002804D0BB
:104B60002046441CC0B20228F1DBE4B2032C0BDB6C
:104B70000020317847F82100307857F82000C8F835
:104B80000400304601F080FE6D1C0024192D18DA57
:104B90002C2001F061FE064622462C21FDF768FC20
:104BA000DFF8B888304658F835108847307847F82D
:104BB000206008EBC508307857F82000C8F80400DA
:104BC000C8E72046BDE8F081002200E0521C92B206
:104BD0008A4204D2135CFF2BF8D0012070470020DA
:104BE000704702B51346372119705870022200A988
:104BF000981CFDF76BFC01BD02B510460121017048
:104C0000022200A9401CFDF761FC01BD008A0228B8
:104C100001DB012070470020704770B588B0064660
:104C200002A80FF69C011422FDF760FCDFF82808AB
:104C300050F82600458A281D01F00EFE0446224643
:104C400001213046FFF7CDFF211D304601F07BF9F1
:104C5000281DADF80B002846A0F1080189B2201DDF
:104C6000FFF7B2FF00280DD000F0BDFECDE9000136
:104C7000082200A928190838FDF728FC214602A8B7
:104C800001F0BAFE204601F0FFFD08B070BD10B57E
:104C90000C46C17801290ED100216160FFF7B6FFF3
:104CA000002805D0A068002802D000F0EDFE00E04A
:104CB0000020A06010BD8068002804D000F0E4FE51
:104CC000A060606010BD606800F0DEFE6060A06003
:104CD00010BD10B400216FF00042104611E0DFF863
:104CE0007C4704EBC3035B68002B09D01C6A002CD3
:104CF00006D0DB78002B03D1E368984200DD18462C
:104D0000491C49B20B46192BE9DB904200D1002027
:104D100010BC70472DE9F04184B004461546264684
:104D2000DFF8340750F8267008788DF800004868DE
:104D3000019088680290002F01D1032043E000A970
:104D40003846FFF7A4FF00A907F1200002F048FF52
:104D500007F11C0898F80C0001280BD1204601F03F
:104D60001FF907F1100002F0B5FF0020F96949684A
:104D700088470DE09DF80000002809D107F11000D8
:104D800002F0A8FF3879012802D12046FFF745FF3D
:104D90002A4600213D20FB691B699847F8780028C6
:104DA00002D1022001F013FED8F80800002801D03B
:104DB000012300E0002398F80C2031460FF2A86090
:104DC000FEF78AFF002004B0BDE8F081FEB506467C
:104DD0001446DFF8840650F8265008788DF8000055
:104DE0004868019088680290002D19D09DF8000055
:104DF00000280AD105F11C07B868002810D0C06847
:104E00000190B8680069029003E000A92846FFF706
:104E10003EFF00A905F1200002F002FF002801D0AA
:104E20000320FEBDEB6905F11C07387B002803D188
:104E30000020D968884704E0224600213E201B69F3
:104E40009847022001F0C3FDB868002801D0012373
:104E500000E000233A7B31460FF21860FEF73CFF7A
:104E60000020FEBD30B587B00546DFF8EC0550F8F0
:104E7000254008788DF80C004868049088680590F3
:104E800010788DF800005068019090680290002C16
:104E900003D008781178884201D0032030E003A9BC
:104EA0002046FFF7F4FE00A92046FFF7F0FE049825
:104EB0000199884205D105980299884201D10020C4
:104EC0001EE000A904F1200002F0AAFE002801D093
:104ED000032015E003A904F1200002F081FE002266
:104EE00011463F20E3691B699847022001F06FFDDE
:104EF000049B019A29460FF28850FEF7EDFE002030
:104F000007B030BD10B50C4611461A46DFF84835DB
:104F100053F82030002B01D1012010BD2046DB6961
:104F20001B699847002010BD10B50C4611461A4663
:104F3000DFF8243553F82030002B01D1012010BDBB
:104F4000192C04D1012100F06CF9002010BD20467D
:104F5000DB695B699847002010BD0146CE2901DA64
:104F6000002801D100207047DFF8EC0450F8210040
:104F7000704710B582B000218DF80010082804D0C9
:104F800010281CD0202830D013BD00AA01214020B9
:104F9000DFF8C4345B68DB695B6998479DF8000003
:104FA000800703D50021012002F041FF9DF8000099
:104FB000400732D50021022002F039FF13BD00AABC
:104FC00001214020DFF890345B68DB695B6998471A
:104FD0009DF80000000703D50021032002F027FF01
:104FE0000021042002F023FF13BDDFF86C04046AE3
:104FF00000F0F9FCE2699268904700280DD1606AE0
:10500000002806D00069002803D10021082000F004
:1050100008F90021084602F00AFF13BD10B5044646
:10502000206AA268002A07D1002810D04269521ACB
:10503000012A05DB4068F7E74069401A012806DAD3
:1050400000F0D1FCE2699268BDE81040104710BD45
:105050002DE9F84304460D4604F1100002F0B2FEBB
:10506000064604F1100002F0B4FE074620782B2813
:1050700002DA4FF0040801E04FF00308002F42D09D
:1050800040F2012008EB0601814203DB2046BDE827
:10509000F2438AE0B5F8031016FA81F2DFF8BC9308
:1050A00008EB020181420DDB0FF2E0310FF2F0302C
:1050B000FEF712FE09F1C801284601F09DFC002010
:1050C000A5F80300B5F80300484400F1C8022078B1
:1050D0002B2803DA3946FFF784FD02E03146FFF75B
:1050E0008BFD3A4604F11001B5F8030018FA80F080
:1050F0004844C83002F01EFEB5F8030008EB060174
:105100000818A5F80300BDE8F18338B50446154634
:10511000606A00280FD08069401A01280BDA00F07D
:105120000FFC012802D1207B002804D0294620460C
:10513000BDE834408CE731BD70B586B000A80FF2F1
:1051400094311422FDF7D2F901F037FC0446002512
:105150001CE0DFF8081301EBC0004668002E14D0F5
:1051600096F82800002810D0F07800280DD12146AC
:105170003046FFF753FF00AA21463046FFF7C5FF30
:10518000214606F1200002F068FD6D1CEDB22846B4
:105190001928DEDBBDF80300002803D0B04900A8C1
:1051A00001F02AFC002006B070BD2DE9F04385B067
:1051B000044600A80FF230311422FDF797F9257844
:1051C0004FF4FE70618A90FBF1F6B6B204F1100064
:1051D00002F0FFFD0746DFF88C9219E0B8464A4618
:1051E00041462846FFF7FDFC424604F1100109F153
:1051F000040002F09FFD608A00FB08F0001DADF87E
:105200000300494600A801F0F7FBA7EB0807BFB26F
:10521000002F03D0B742E1DBB046E0E705B0BDE8C0
:10522000F08330B587B004460D468B4850F8240013
:10523000FFF7BBFF002D13D001A80FF2C0211422ED
:10524000FDF754F900A80FF2C8210A6802608DF832
:1052500002400320ADF8070000A901A801F0CCFB33
:1052600007B030BD30B583B000A80FF24C210CC997
:105270000CC000240FE0784800A9615C50F8215070
:10528000002D07D02846FFF7C1FC002802D0284691
:10529000FFF78BFF641C052CEDDB37BD6E4951F821
:1052A0002000002804D0406A002801D00120704767
:1052B00000207047684951F82000002802D14FF0C3
:1052C000FF30704790F82810481E8041C043C00F3F
:1052D00040B27047604951F82000002804D0006AAD
:1052E000002801D0C0687047002070472DE9F041C8
:1052F0000446012510E0584850F8250000280AD03F
:10530000D4E90067012000212A4602F0FDFD304368
:105310003943C4E900016D1C2B2DECDB04F10806B8
:1053200081271EE04C4850F82700002818D0A7F12C
:105330008002501102EB90604FEAA0185FFA88F8E3
:1053400006EBC800D0E9004501200021A2EB88123D
:1053500002F0DAFD2043294306EBC802C2E900014E
:105360007F1CCE2FDEDBBDE8F0812DE9F04186B059
:1053700007460C4600A80FF29C111422FDF7B6F860
:105380004FF4F37001F068FA050019D121E03E46B0
:105390002C2010FB06F81FFA88F808F10200ADF87F
:1053A0000300412028706E7042462146A81CFDF77C
:1053B0008DF8294600A801F01FFB4444BF1BFFB233
:1053C000002F03D00C2FE2DB0B26E1E7284601F08B
:1053D0005BFA06B0BDE8F08138B5044601250CE063
:1053E0001D4850F82530002B06D0224600214820C9
:1053F000DB695B6998472C346D1C2B2DF0DB31BDCC
:1054000070B500240120144A00E0401CC0B20146DF
:105410002B2906DA52F821100029F6D0641CE4B2D8
:10542000F3E720462C2111FB00F5ADB2284601F030
:1054300013FA06000FD000222946FDF793F83046F4
:10544000FFF7CAFF31462046FFF78FFF3046BDE821
:10545000704001F019BA70BD109D03007858030028
:1054600040590300ECA4030023612025642C25642B
:105470002C25640023722025642C25642C256400CF
:1054800023632025642C25643E25640061727261CB
:105490006E67655F646174615F7061636B65740002
:1054A00025733A2074785F646174612069732066A3
:1054B000756C6C2825642900010E06120800000096
:1054C00005000000000000000000000000000000D7
:1054D00000000000050000000000000000000000C7
:1054E00000000000000000000500000000000000B7
:1054F00000000000000000000000000005000000A7
:10550000000000000000000000000000000000009B
:105510000501000005000000000000000000000080
:10552000000000000000000010B5DFF8B8410022C4
:1055300008212046FCF79CFF204610BDDFF8A4019F
:105540007047000038B5044602F02CFD4FF47A7223
:105550006243841851EBE27500BF00BF00BF00BF7B
:1055600000BF02F01FFDA942F6D301D8A042F3D339
:1055700031BD80B5FFF7D8FF02F018FEBDE801404D
:10558000BCE080B5084600F0E7F9584802F0E3FEB9
:10559000002805D00FF27810BDE80240FEF79CBB52
:1055A00001BD0023524A4021504802F033BFFB2383
:1055B0000FF26C1202F0F9BEF8B50C4615461E4605
:1055C000052749480178491C0170002003F01EF8A6
:1055D000002806D133462A462146002003F019F858
:1055E000074601F085F83846C0B2F2BDF8B50C4662
:1055F00015461E4605273C480178491C01700020CD
:1056000003F004F8002806D133462A46214600203C
:1056100003F001F8074601F06BF83846C0B2F2BD5E
:1056200002280ED005280CD006280ED008280AD053
:105630000E2806D01D2806D0222802D0C02802D06D
:1056400005E00420704707207047092070470020BC
:1056500070472DE9F8430C4615461E46052740B213
:10566000FFF7DEFF804615F8019B1F480178491CB3
:1056700001702049404603F098F8002808D10095B1
:10568000731EDBB24A466108404603F0A4F80746A1
:1056900001F02EF83846C0B2BDE8F2832DE9F041A2
:1056A00082B00C4615461E46052740B2FFF7B8FFEC
:1056B00080460D480178491C01700E49404603F0B0
:1056C00074F8002807D10096089B2A4661084046D6
:1056D00003F06CF8074601F00BF83846C0B2BDE89D
:1056E000F681000040C20300C063030060BD0300F8
:1056F00083650000801A060002F03CBC80B5FFF70D
:105700001DFF01210170C1704171817101BD000057
:105710004D534720426F782046756C6C00000000A6
:1057200073746172745F74785F73747265616D0015
:105730001B4213D1094236D12AB18446B0FBF2F0A4
:1057400002FB10C2704703F0BDB8FCD30022002357
:1057500070470B000200002100207047904271EB5F
:10576000030CF6D370B5B1FA81F4B3FA83F52C1BB0
:10577000A340C4F1200532FA05F63343A2405FF09E
:105780000046E64002E05B085FEA3202841A71EBF1
:10579000030524BF204629467641F4D302000B00BE
:1057A0003000002170BD012ACFD970B5140C20D073
:1057B000B1FA81F4B2FA82F5C4F120046419B4F1AB
:1057C0002006D6D3B2405FF00044F440002502E04A
:1057D00052085FEA3303C61A71EB020E24BF30464B
:1057E000714664416D41F3D302000B002000290093
:1057F00070BD0C46B1FBF2F102FB11452D0445EAE8
:105800001045B5FBF2F402FB145580B240EA0545A1
:10581000B5FBF2F002FB105240EA044070BD0000FC
:1058200000B585B000A80FF208511422FCF75EFE07
:1058300000A802F090FD002803D00FF2BC40FEF754
:105840004BFA05B000BD80B50020DFF88014487128
:105850008DF8000000A9082002F0E9FA0FF2A44038
:10586000FEF73AFA01BD10B5DFF860444FF47A72E2
:10587000DFF85C1404F1240003F069F84FF42F7290
:10588000DFF8581404F1380003F061F8002010BD6F
:105890007047DFF84C04704710B586B0044601A885
:1058A0001421FCF75BFEFFF7F4FF00900D22214668
:1058B00001A8FCF70BFE0420ADF8070000A901A821
:1058C00001F09AF806B010BD10B58CB0044606A8D9
:1058D0001421FCF743FE00A81821FCF73FFE0D221F
:1058E000214606A8FCF7F2FD00A8FFF7FFFC1820F0
:1058F000ADF81B0000A906A801F07EF80CB010BDA1
:1059000010B5DFF8C84360702078012808D16078AE
:10591000082805D1FFF7A6FC0FF2F43003F080F859
:105920006078042802D10120207003E0082801D10A
:1059300000202070611C0720BDE8104002F077BAFB
:10594000DFF8880300787047DFF88003C07870477D
:10595000DFF878034079704770B5040038D0DFF87D
:105960006C53D5E90401002901D100280DD0D4F8E9
:105970000520D4F80930101A63EB0101D54A012340
:10598000994202D824D3904222D3D64E3078401C7C
:105990003070802080F3118800BF00BF7078401CF9
:1059A0007070FFF7A9FED4F80520D4F80930C5E9D6
:1059B0000423C5E906017078401E7070C0B200284B
:1059C00002D1002080F31188BDE8704000F090BE45
:1059D00070BDBE49D1E90423C0E90023D1E9062303
:1059E000C0E90223704738B5FFF786FEB74AD2E90F
:1059F000044520186941D2E90645001BA94134BD80
:105A0000B24902780A7242784A728078887200201D
:105A1000888170470622B449FCF758BD10B504468A
:105A200000F0CBFFA9490A6A002A01D0A21A00E0BF
:105A30000246B2F57A7F00D3024688891018888121
:105A400000B2B0F57A7F05DBA0F57A708881887A9C
:105A5000401C887291F90A003C2804DB3C388872AB
:105A6000487A401C487291F909003C2804DB3C3814
:105A70004872087A401C087291F90800182801DB66
:105A8000002008720C6210BD80B50A2801DA0520DA
:105A900002BDA12801DBA02002BD0A2190FBF1F08C
:105AA00002F0D0FF41EC100B02F0E4FF51EC100BC0
:105AB00000F0ACFB02F0C6FF41EC110B9FED8B0B2D
:105AC00003F023FA51EC100B00F0A0FB00EB800177
:105AD000480002BD00B587B002A80FF26821142269
:105AE000FCF704FD00A800210A4606C0FFF726FDCA
:105AF00001788DF8001000A9C2784A7042798DF8BB
:105B000002208079C87001208DF804000520ADF8CE
:105B10000B0002A800F070FF07B000BD30B59FB0C9
:105B200005A86421FCF71AFD00A80FF22C2114220D
:105B3000FCF7DCFC0024FF22642105A8FCF798FC9C
:105B4000012517E02846C0B2FFF707FA002810D059
:105B50002946491E012906D9C91E022903D9091F50
:105B600001D01A3905D105A964B26554408A401C98
:105B700004196D1C092DE5DB64B2ADF8034005A9DD
:105B800000A800F039FF00201FB030BD38B5044632
:105B9000A0780146491F1CD0491E1DD0491E01296D
:105BA00027D9891E01292CD9203907D00F390AD0CD
:105BB000491E4AD0491E01292CD94BE0D4F80D00CA
:105BC000FFF71EFF46E0B4F80300C0B2FFF798FEEF
:105BD00040E0414802F0C7FEA078052801D101202D
:105BE00000E00020394DE870E91C062002F01FF9A2
:105BF00030E0072801D1012000E00020334908717E
:105C000028E0324D092802D10020A87022E00120AE
:105C1000A8701FE02D4D3A280ED136A0FEF75CF893
:105C20000120687105F1380002F0C8FED4F80D10AB
:105C3000082002F0FCF80DE00FF2EC00FEF74CF843
:105C400005F1380002F08FFE04E0D4F80D100120B9
:105C500003F023FCA0781438032801D915380FD19C
:105C60008320FFF77AF903000AD0D4F80D20B4F8A6
:105C70000310A078DB691B6901B0BDE8304018470C
:105C800031BD80B581780C2908D018290FD01B2987
:105C900007D02C290ED031290FD001BDBDE802401C
:105CA000FAE5FFF711FEBDE80140FFF7A9BBBDE82B
:105CB00001400FE7BDE8014030E7044800780028C4
:105CC00003D1BDE80140FEF76FB801BD40BC030041
:105CD0002168000000F2052A64BC03004768000048
:105CE0004CEA4001C063030048BC03000000000010
:105CF000000000404D4F4E00736B697020524349C5
:105D0000000000004D4F46462043422100000000A5
:105D100023212120617020737461746520636861A0
:105D20006E6765210A0000004D4F464600000000E6
:105D300004FF31000000000000000000000000002F
:105D40000000000004FF1800000000000000000038
:105D5000000000000000000004FF2C000000000014
:105D60000000000000000000000000002DE9F041EC
:105D700080460C46FFF7F1F80546002700F01DFEAF
:105D80000646B8F1010F1AD0B8F1040F47D0B8F1A8
:105D9000050F74D0B8F1080F00F08080B8F1250F1E
:105DA00000F0A580B8F1A10F00F09480B8F1A40F25
:105DB00000F09680B8F1BB0F00F0AD80AFE003F0CB
:105DC00090FCDFF83482B4F9000000EE900AF8EE9F
:105DD000E00A20EE800A88ED000A03F082FCB4F9A4
:105DE000020000EE900AF8EEE00A20EE800A88ED4C
:105DF000010A03F076FCB4F9040000EE900AF8EE14
:105E0000E00A20EE800A88ED020A2088A8F80C003B
:105E10006088A8F80E00A088A8F810007FE003F0C2
:105E20008DFDDFF8D481B4F9000000EE900AF8EEA1
:105E3000E00A20EE800A88ED050A03F07FFDB4F940
:105E4000020000EE900AF8EEE00A20EE800A88EDEB
:105E5000060A03F073FDB4F9040000EE900AF8EEB0
:105E6000E00A20EE800A88ED070A2088A8F82000C2
:105E70006088A8F82200A088A8F824004FE0DFF886
:105E80007881D8F834002168884200D101271C228B
:105E9000214608F13400FCF719FB40E0DFF8588197
:105EA00098F850002178884200D10127012221462C
:105EB00008F15000FCF70AFB0222611C08F15200B5
:105EC000FCF704FB022204F10B0108F15400FCF77B
:105ED000FDFA24E00C2221464848FCF7F7FA1EE0C0
:105EE00001270C2221464648FCF7F0FA17E0DFF8BC
:105EF0000881D8F858002168884205D1D8F85C009C
:105F00006168884200D101270822214608F1580023
:105F1000FCF7DCFA03E0E078374981F86C00002DEB
:105F20000FD0002F0DD1686A00280AD04069801B6D
:105F3000012806DA214605F11000BDE8F04101F024
:105F4000CDBEBDE8F08102460846012A0CD0042AE5
:105F50000ED0052A10D0082A12D0A12A14D0A42AC3
:105F600016D0BB2A18D0704714222349FCF7AEBACA
:105F700014222449FCF7AABA1C222349FCF7A6BA2A
:105F800006222249FCF7A2BA0C221C49FCF79EBA51
:105F90000C221B49FCF79ABA01221D49FCF796BA5C
:105FA00001280AD004280DD0052810D0082818D0C0
:105FB000252811D0BB2819D07047FF2214210E4884
:105FC000FCF756BAFF2214210E48FCF751BAFF2203
:105FD0001C210D48FCF74CBAFF2208210D48FCF7A4
:105FE00047BAFF2206210948FCF742BAFF220121E5
:105FF0000748FCF73DBA000098B90300C0B9030098
:10600000F8B90300ACB90300CCB90300E8B9030048
:1060100004BA0300F0B903005FF0FF0C1CEAD05192
:1060200014BF614506E0C110400721F0E04101F1D5
:106030006051704779B900F0004100020AD0B0FA0F
:1060400080FC00FA0CF001F16051A1EB0C5101EB66
:10605000D0214005704741020CBF40F4E0016FF0D1
:106060000001002070470000B0B581EA030C0CF07D
:10607000004C40F2FF7515EA11541DBF15EA135785
:10608000AC42AF4239E0E41923EA455343F48013AC
:10609000C90241F0004141EA505EC7021100A7FB6E
:1060A000020200284FF00000EEFB01204FF000013B
:1060B000E3FB072118BF42F00102401800214941CB
:1060C000E3FB0E01A4F580640F0302D252004041AD
:1060D000494154F101046CDD470872F1004250F16E
:1060E000000051EB0451A1F580115CBF41EA0C01A5
:1060F000B0BD4CEA05510020B0BD05EA1357AC42D3
:1061000014BFAF4241E050EA410E1CBF52EA430EB9
:1061100002E061460020B0BD24423C441BD15FEA4E
:10612000070EF6D0090302BF01460020AEF1140E9F
:10613000B1FA81F7AEEB070401FA07FE0C37C7F19D
:10614000200100FA07F7C8404EEA000E23EA455343
:1061500043F48013A2E733F00043B3FA83F704BF9C
:10616000B2FA82FE77440B3FE41BB7F1200E2FBF3B
:1061700002FA0EF3BB40C7F1200E22FA0EFE38BF22
:1061800043EA0E03BA40641C82E750EA410E14BF92
:1061900052EA430E6FF000014FF4001717EB430F64
:1061A0008ABF194617EB410FB5E74CEA05510020AD
:1061B000B0BDD4F10104B4F120070FDAC4F1200717
:1061C000520828BF42F0010210FA07F501FA07F75A
:1061D000E1BF2A43E0403843E1400FE0352C98DC32
:1061E000C7F1200452EA400220FA07F218BF42F039
:1061F000010231FA07F0A1400A43002172F1004286
:1062000050F1000051EB0C01B0BD0000F446400D10
:1062100040EAC120490006D200F014F8004248BF0D
:106220006FF00040604700F00DF84FF000418842E9
:106230008CBF084640426047400D40EAC1204900FB
:1062400080F00D8040F00040490DA1F58061491CAF
:1062500005D4D1F11F0154BFC840C01770474FF09B
:106260000000704770B44FF0004591EA030C44BF42
:106270006B4003F0A7BB00BF841A71EB030603D287
:10628000001BB141121973414FF4001C1CEB410F6C
:1062900034BF7CEB430443E00C0DA4EB1356352EC6
:1062A00050DC45EAC323DB0A45EAC121C912B6F135
:1062B00020050DDD63FA05F6EB4086EA0305124280
:1062C00018BF45F00105C01851F100010CD213E0D0
:1062D00062FA06F5F2405540F3415A40B340F340AC
:1062E0005A408018594107D349085FEA30005FEAF5
:1062F000350528BF45F0010501F58011420875F10B
:10630000004250F1000041EB045170BC4FF4001CFE
:106310001CEB410F38BF70470020090D090570477D
:106320001CEB410F10D252EA43060BD0BCEB410FDD
:1063300005D80C0DAB43661E342EB5DD02E0AB4331
:106340008018594170BC704770BC70474FEAF17CAF
:10635000BCF1E04C2CBFBCF5001F11E05FEA4C0C17
:1063600034BFBCF17F5F2EE05FEA9C0C4FEA0C1C4F
:106370004FEA3C0CC10071F100414CEB507070478A
:10638000C90241EA5051C00218BF41F0010141F079
:1063900000414FEA6C50C0F10900212810D240EAB8
:1063A000CC7CCCF1200C11FA0CF070F10040CCF157
:1063B000200C21FA0CF00CF0004C40EB0C00704764
:1063C0004FEACC707047490011F5001F04D84FEA1E
:1063D000CC10FF30C0057047C81770474FF4001C41
:1063E0001CEB410F94BF1CEB430F09E041EA030C87
:1063F00050EA4C0C52EA0C0C03D28B4208BF82428A
:10640000704714BF99429042704700004FF4001C3F
:106410001CEB410F94BF1CEB430F09E041EA030C56
:1064200050EA4C0C52EA0C0C03D2994208BF90423D
:10643000704714BF8B4282427047000008B584B099
:106440000023029311B90093019302E00090481ECB
:10645000019004AB00A907487844183003F068FBAA
:10646000009911B1009A00211170002858BF0298BC
:1064700005B000BDCFC0FFFF00F10103810704D0CC
:1064800010F8011B89B18107FAD10268B2F101311C
:10649000914311F0803F04BF50F8042FF6E710F845
:1064A000011B11B110F8011BFBE7C01A7047000077
:1064B00030B4802080F3118800BF00BFDFF8941350
:1064C000886800220A7182F3118800281CBF0268C4
:1064D000002A33D0436954699C422FD100E0224600
:1064E0001468A4B165699D4211D12246146874B143
:1064F00065699D420BD12246146844B165699D428D
:1065000005D12246146814B165699D42E7D0802305
:1065100083F3118800BF00BF03680C69844208BF81
:106520000B61016A0B60196202621168016001B1BE
:106530000862106092F8290082F82800002080F399
:10654000118830BC704730B5DFF808430020607117
:1065500081B0206AE16900F18040606208001CBFE0
:1065600020468847002080F31188E56808E0E86845
:10657000616A411A48BF6062002080F311882D686B
:1065800005B3802080F3118800BF00BF206920B1CF
:10659000686921694969884219D3287C4007EBD58D
:1065A000E868216A401A0128E1DA284600F0BCF8C0
:1065B000802080F3118800BF00BF287C0028D6D13E
:1065C00001B030BD802080F3118800BF00BF01B052
:1065D00030BD000070B5DFF87C4200206070012003
:1065E0002070E06B68B1802080F3118800BF00BF8D
:1065F000E06B8047002080F31188E063606384F8DB
:106600003800A06800281CBFC16A002904D00968AE
:106610000A001CBF4068884794F8310040B1A06868
:1066200094F8301080F82810207908B1FFF740FF67
:10663000206948B304E028682061002080F31188B5
:10664000802080F3118800BF00BF25690DB32E7C28
:10665000FEB170070ED5E868216A411A012905DAF2
:10666000284600F061F8287C20B90DE0616A411AE3
:1066700048BF606206F0FB001028DCD1A868806883
:106680004068007C0028D6D1802080F3118800BFAC
:1066900000BF607950B9206900B32069007C0028F0
:1066A000206909D080688068406805E0FFF74BFFEB
:1066B00060790028FAD1EEE7A060A068C16A21B134
:1066C00049680A001CBF40688847A06890F8280005
:1066D00084F8300084F83100204670BD84F8310021
:1066E00084F83000A060207080F31188204670BDCF
:1066F00010B5584C2078401E2070C0B298B9606820
:1067000088B1802080F3118800BF00BF606830B17D
:1067100001202070204604F02CF9002020706078C1
:1067200008B980F3118810BD30B581B08168494C3B
:1067300041B1226AC2600A68496802B151600A60C8
:1067400000218160017C11F00301017426D12169CF
:1067500091B92061207838B901202070204604F0DA
:1067600008F90020207001E0012060716078A8B96C
:1067700080F3118801B030BD42694B699342E8D380
:106780008142E7D09A4209D103461B68002BEDD025
:106790005D69AA42EAD18B42F7D1DAE701B030BD98
:1067A00030B52C4C227881B04169521C227004F122
:1067B0000C0200E01A461368A3B15D69A94211D228
:1067C0001A46136873B15D69A9420BD21A46136861
:1067D00043B15D69A94205D21A46136813B15D69D8
:1067E000A942E7D303600262106043B118625A699C
:1067F0008A420CBF90F82910002180F82810017CF3
:1068000051B9802181F3118800BF00BFFFF78CFFD1
:10681000607808B980F3118801B0BDE8304067E7BF
:1068200030B50C4C2578681C207081B0204604F0EF
:10683000A0F86078257008B980F3118801B030BDE8
:1068400000B581B004F0C8F802480121017001B020
:1068500000BD0000C063030030B5134D0446287826
:1068600081B020B9281D04F0F1F801202870281DFE
:1068700004F005F9204604F0E4FF0446281D04F066
:1068800024F9204601B030BD30B50446064D81B034
:10689000281D04F0F4F8204605F033F9281D01B056
:1068A000BDE8304004F011B9C4C0030080B5FEF764
:1068B00023FF009000A800F083F8042000F087F880
:1068C000444802F050F801BD70B5424C2046C06803
:1068D000C0460546FEF7FDF90646B54212D03146E0
:1068E0002846C046C0463146204605F097FB002E9C
:1068F000204603D0BDE8704002F035B8BDE87040D6
:1069000002F05CB870BD10B582B000200090FEF7B8
:10691000BFFF0021022002F0C0FD23E00098FFF736
:106920007DF82D480178491C0170FEF705FCFFF742
:10693000DFFE00A9294805F07FFB0028EED02007E4
:1069400002D50820FEF715FBE00602D51020FEF761
:1069500010FBA00602D52020FEF70BFBA00701D5F7
:10696000FFF7B2FF3E2005F085FB04466007E0D448
:10697000E5E710B584B0174C04F114030822042194
:1069800004F1680005F098FB022002904FF40060CB
:10699000019004F180000090114B50220FF24C0145
:1069A00004F1340005F094FB4FF47A720D4920464F
:1069B00004B0BDE8104001F0CABF0648C068704787
:1069C00080B50146054805F0B5FB40B202BD064959
:1069D00005F0CEBBA47B0300C06303000C7C030066
:1069E00007790000AD780000D87B030073656E73F3
:1069F0006F725F7461736B002DE9F04705460E46B8
:106A0000B5F80370334C2078401C2070802080F350
:106A1000118800BF00BF6078401C6070287805288E
:106A200003D1FDF7A1F9804601E04FF0000808EB23
:106A3000070000F10D0A5046FFF70EFF8146B9F13D
:106A4000000F11D151460FF2940001F0E9FF607878
:106A5000401E6070C0B2002802D1002080F311886F
:106A6000BDE8F047FFF744BEB5F803004044A5F881
:106A700003000D2229464846FBF728FD3A463146D9
:106A800009F10D00FBF722FDB8F1000F04D007EB70
:106A900009000D30FDF771F9B5F8030000F10D01A3
:106AA00089B24846FEF783FD6078401E6070C0B230
:106AB000002802D1002080F31188FFF719FEB9F1F8
:106AC000000F04D04846BDE8F047FFF7DDBEBDE843
:106AD000F0870000C0630300FEF763BD7478627541
:106AE00066666572206973206E6F7420616C6C6FCE
:106AF00063617465642825642921210A000000006F
:106B00002DE9F043002300E05B1C032B4ADA00244C
:106B100033E005F1070EAEEB060E4FF007089EFBC3
:106B2000F8F8C8EBC808AEEB080E5FFA8EFE0FF659
:106B30006468C3EBC30908EBC90808EB8609D9ED03
:106B4000070A07EB000909EB8E0999ED3F1A60EE81
:106B5000810A08EB860898ED001A0CEB8E0EDEED2C
:106B6000001A41EE610A30EE800A761C072ED0DB57
:106B70000CEB850585ED000A641C032CC4DAC4EB1C
:106B8000C405AF00542515FB030507EB050C0D46A6
:106B9000002A03D100264CF82560EDE79FED440A5A
:106BA0000026E3E7BDE8F083D2B218B400230CE07E
:106BB00094ED031A21EE001AF7EE001A71EEC01AD6
:106BC00001EEA01A84ED001A5B1C032B0ADA51F8BF
:106BD000234000EE904A002A00EB8304E8D1C4ED84
:106BE000000AF1E70C2201460C3018BCFBF77EBC12
:106BF00038B504460D4600200AE0C0EBC00204EBA5
:106C0000820202EB810155F82020C1F8FC20401CD3
:106C100004F5F27292F902100328EEDB5278C9B241
:106C20002046FFF76DFF94F8E4219FED220A2946E4
:106C300004F5A870BDE83840B6E70000F8B5044692
:106C400094F9E651EDB2002617E0542212FB0642F9
:106C500011FB002151F8251000EE901A00EEA00A59
:106C6000401C1C210328F0DB11FB064000EB8507CC
:106C700005F09CFA87ED5D0A761C032E03DA9FED82
:106C80000C0A0020EDE704EB850000F5C87191EDDA
:106C9000070AB5EE400AF1EE10FA06D0D0ED640A0C
:106CA00080EE800A81ED0E0AF1BD00208863F1BDFF
:106CB00000000000A4707D3F10B5044604F5A870E4
:106CC000D0ED020A90ED011A94ED540A20EE000A6C
:106CD00001EE010A00EEA00A05F068FA002002E0C9
:106CE00000228A61401C03280FDA04EB800202F5BF
:106CF000A871B5EE400AF1EE10FAF1D0D2ED540AC7
:106D0000C0EE800AC1ED060AECE710BDD0ED000A26
:106D100070EE800AC0ED000AD0ED010A40EE000AD4
:106D2000C0ED010A89B2531E994215D100EE102A16
:106D3000B8EE400AD0ED000AC0EE800AC0ED000AAD
:106D4000D0ED010A80EE800A80ED010AD0ED000A44
:106D500000EEE00A80ED020A70472DE9F84F044684
:106D60000D4694F9E601C0B200902E88322096FBC1
:106D7000F0F0322101FB1067B5F878804FF0000980
:106D80002AE004EB890A09EB490005EB800B4FF47C
:106D9000FA7231460BF140009AED5A0AFFF7B6FF3E
:106DA00040F2DC5241460BF190009AED5A0AFFF78F
:106DB000ADFF3222394689B20BF11C00C9EBC90381
:106DC00004EB8303DDF800C003EB8C0393ED3F0A73
:106DD000FFF79CFF09F10109B9F1030FD1DBBDE811
:106DE000F18F8A1D072392FBF3F3C3EBC303D21A7F
:106DF00050F8222000EE102A00EB8100D0ED000AAE
:106E000030EEC00AB0EEC00A704730B40A46002126
:106E1000931D072493FBF4F4C4EBC4041B1BDBB2E7
:106E2000541D072594FBF5F5C5EBC505641BE4B2BD
:106E300050F8233000EE103A50F8222000EE902A4D
:106E4000F4EE400AF1EE10FA0AD500EB840292ED5E
:106E5000001AB4EE401AF1EE10FA01D501210EE04D
:106E6000B4EE600AF1EE10FA09D500EB8400D0ED23
:106E7000000AB4EE600AF1EE10FA00D501210846CE
:106E800030BC70472DE9FE4306460C4696F8E651A5
:106E90002088002800F08A8000273CE0C7EBC7006C
:106EA00006EB8009294609F15400FFF79AFF08EB29
:106EB000870080ED000AD4ED030A30EE800A84EDED
:106EC000030A09F1A80829464046FFF78AFFD4EDD6
:106ED000050A30EE800A84ED050A294609F15400BE
:106EE000FFF793FF00EE100AB8EE400AD4ED040A53
:106EF00030EE200A84ED040A29464046FFF785FF5C
:106F000000EE100AB8EE400AD4ED060A30EE200A70
:106F100084ED060A7F1C0DF10008032FBEDB002064
:106F20000AE094ED010A08EB8001D1ED000A30EE91
:106F3000200A84ED010A401C0228F2DB94ED020ACB
:106F4000D8ED020A30EE200A84ED020A294606F541
:106F5000C870FFF746FFD4ED030A30EE800A84EDD7
:106F6000030A294606F5D670FFF73BFFD4ED050A64
:106F700030EE800A84ED050A06F5E47629463046AF
:106F8000FFF72FFFD4ED1B0A30EE800A84ED1B0AB9
:106F900029463046FFF739FF00EE100AB8EE400AE6
:106FA000D4ED1A0A30EE200A84ED1A0ABDE8F78300
:106FB0000A8890F9E631DBB200EB830090ED5D0AC0
:106FC0003220034692FBF3F300FB1323002B04D182
:106FD00081ED020A81ED030A7047D1ED020AF4EE59
:106FE000400AF1EE10FA02D581ED020A08E0D1ED77
:106FF000030AB4EE600AF1EE10FA01D581ED030A3E
:10700000521C034692FBF3F300FB132000281BD114
:1070100091ED020AD1ED030A30EE600AD1ED040AC7
:1070200070EE800AC1ED040A022B0BDBD1ED010AE0
:1070300070EE600AF0EEE00A91ED051A71EE200A9A
:10704000C1ED050A81ED010A088840F2DB52904249
:1070500009D191ED040AF3EE0E0A80EE200A81EDCB
:10706000040A012088707047F8B52DED048B84B0B8
:107070000C460021642749E0C1EBC10200EB82020B
:1070800090F9E63152F8232000EE102A00AA02EB14
:10709000810282ED000A04EB810202F2B445D5EDD3
:1070A000030A70EE800AC5ED030A4FF4C87313FBA0
:1070B000014394F8B06403EB860696ED001A70EE77
:1070C000C10AC5ED030AD2F8B45400EE905A70EE2E
:1070D000800A02F2B445C5ED000A94F8B054323586
:1070E0003E4695FBF6F607FB165503EB850595ED39
:1070F000001A70EEC10A02F2B442C2ED000A94F81E
:10710000B02403EB820282ED000A491C0329B3DBA1
:1071100094F8D804002816D100200EE004EB80017A
:10712000D1F8B42400EE102ADFED850A80EE200AA3
:1071300001F2CC4181ED000A401C0328EEDB012066
:1071400084F8D80458E004F5966090ED040ADFED69
:107150007D0A80EE200A8DED000A90ED050A80EE92
:10716000200A8DED010A90ED060A80EE200A8DEDD1
:10717000020A9FED758A9FED740ADFED738A002085
:1071800011E004EB8001D1F8CC1400EE901A00A9B4
:1071900051F8201001EE101A00EE818A00EEA00ACC
:1071A00041EE018A401C0328EBDB04F0FFFFB0EE48
:1071B000409AB0EE680A04F0F9FF29EE000AB5EE35
:1071C000400AF1EE10FA01D088EE008AB0EE480ACB
:1071D00004F0FAFFDFEDC80A20EE200AF3EE0E0AF3
:1071E000B4EE600AF1EE10FA03DB002084F8D80454
:1071F00002E0012084F8D80494F8B004401C84F81C
:10720000B004C0B2642802D1002084F8B00404B0F5
:10721000BDEC048BF1BD000070B52DED048B06466E
:10722000301D90ED018A7068FEF7F6FE41EC190BF7
:1072300018EE100AFEF7F0FE02460B4614461D46F5
:1072400053EC192BDFF8F406DFF8F416FEF70CFF09
:1072500022462B46FFF7DAF81CD253EC192BDFF845
:10726000E406DFF8E416FEF7FFFE02460B4614467E
:107270001D469FEDDD0A38EE000A10EE100AFEF7FB
:10728000CBFE22462B46FFF7C1F803D2012086F839
:10729000740002E0002086F87400BDEC048B70BD21
:1072A00070B504460D461646FFF7C8FC2046FFF7AA
:1072B00003FD29462046FFF750FD29462046FFF7EB
:1072C000E1FD05F178012046FFF772FE31462046C8
:1072D000BDE87040C8E6000038B52DED028B90ED9A
:1072E000050A90ED038AFBEE040A9FED841A08EE6E
:1072F000201AB4EE401AF1EE10FA1DD510EE100A65
:10730000FEF78AFE02460B4614461D4618EE100A8A
:10731000FEF782FEDFF83426DFF83436FEF7A4FEEF
:107320000022DFF83036FEF79DFF22462B46FFF79E
:107330006DF801D2012000E00020BDEC028B32BDCF
:10734000000048420000C842000000002DE9F04162
:107350002DED028B804600200CE098ED190A01EB20
:10736000410208EB8201D1ED120A30EE200A88EDCD
:10737000190A401CC0B201460329EEDB98ED1A0A37
:10738000D8ED1B0A9FED8F1ADFED8F1A40EE011A20
:10739000F4EE610AF1EE10FA15DB9FED8C1ADFEDC9
:1073A0008C1A40EE011AF4EE610AF1EE10FA0ADBD3
:1073B0009FED881ADFED881A40EE011AF4EE610A9B
:1073C000F1EE10FA4DDA9FED850AF4EE400AF1EE87
:1073D00010FA46D49FED828BD8F81400FEF71CFEFD
:1073E00004460D46D8F80C00FEF716FE53EC182B99
:1073F000FEF738FF02460B462046294604F016FFEA
:107400000022DFF85435FEF72FFEDFF85025DFF8B5
:107410005035FEF727FF02460B4616461F46D8F8A2
:107420001800FEF7F9FD04460D46D8F81000FEF7E7
:10743000F3FD53EC182BFEF715FF02460B462046D2
:10744000294604F0F3FE32463B46FEF7DFFF08D341
:1074500098ED190ADFEDCC0AB4EE600AF1EE10FAED
:1074600001DB002000E00120BDEC028BBDE8F081D3
:107470002DE9F041804698ED1A0ADFEDA10A80EE71
:10748000200AD8ED1B0A9FED9E1AC0EE810A20EE5D
:10749000200A10EE100AFEF7BFFD02460B46164604
:1074A0001F46D8F80C00FEF7B7FD0022DFF8B43411
:1074B000FEF7DAFD04460D46D8F81400FEF7ACFDE1
:1074C000DFF8A424DFF8A434FEF7CCFE02460B4616
:1074D0002046294604F0AAFEDFF86824DFF890343D
:1074E000FEF7C0FE32463B46FEF778FF01D801208A
:1074F00000E00020BDE8F081ED2E65420000FA4377
:1075000038B52DED048B05460C4600200CE095EDBA
:107510000F0A01EB410205EB8201D1ED080A30EEC2
:10752000200A85ED0F0A401CC0B201460329EEDB9C
:107530006869FEF771FD41EC180B2869FEF76CFDD8
:1075400041EC190B53EC182BDFF82804DFF8281452
:10755000FEF78AFD02460B4651EC190BFEF756FF6B
:107560002CD253EC182BDFF81404DFF81414FEF7B8
:107570007BFD53EC192BFEF749FF1FD253EC182B60
:10758000DFF80004DFF80014FEF76EFDDFF8CC230F
:10759000DFF8F833FEF766FE53EC192BFEF736FFE3
:1075A0000CD295ED0F0ADFEDC40AB4EE600AF1EEDD
:1075B00010FA03D5002C01D1012000E00020BDEC21
:1075C000048B32BD00C028C500854F49000048C467
:1075D00000E87D480000C8C200C82F4701806D4503
:1075E0008DEDB5A0F7C6B03E0000CDC338B5054659
:1075F0000C460020A070607095F87A00002806D034
:1076000095F8741005F17800FFF77AFFA07095F8EF
:107610007400002813D12846FFF75EFE00280CD125
:107620002846FFF793FE002807D12846FFF720FFE2
:10763000401E8041C043C00F00E0012060706078B0
:10764000002805D1A178481E8041C043C00F00E04A
:107650000120207031BD70B400220378447B2418CF
:10766000E370437B144610E05B1CDBB20A2593FBFE
:10767000F5F505EB8506A3EB4603DBB21D18ED78A7
:10768000661C16FB052292B2641C0A2CECDB04205B
:1076900008702D2A02DB022048700BE0222A02DB50
:1076A0000120487006E00F2A02DB0020487001E04C
:1076B0000020087070BC704710B504469FED9C0A0E
:1076C000002008E000EB400104EB8101D1ED090A44
:1076D00000EEA00A401C0328F4DB04F067FD84EDF3
:1076E0001C0ADFED940AB4EE600AF1EE10FA05D53B
:1076F000002211460846BDE81040B3E010BD00006E
:1077000000401C4670B50C4604F59B65E97BAA7BDE
:10771000121992F8E124891AE973A97B091990EDED
:107720001C0ADFED850AB4EE600AF1EE10FA03DB05
:10773000012081F8E10402E0002081F8E104E87B07
:10774000A97B091991F8E1140818E873904E0022FA
:10775000242106F50170FAF78BFE96F89A070428A3
:1077600010D196F89B0700280CD0E87B022803DA9A
:1077700094F8D804002805D1002204210220BDE895
:1077800070406FE070BD0000CDCC4C3E30B591B084
:107790007F4C04F5F2718878401C88704A78002A82
:1077A0000BD194F8E421002A02D1012284F8E421CB
:1077B00040B2072801D101224A7040B2072290FB53
:1077C000F2F2C2EBC202801A88708888401C88805E
:1077D000B4F86012491CA4F8601280B2322190FB08
:1077E000F1F1322202FB110131290BD194F88617F5
:1077F000491CC9B2052291FBF2F202EB8202891AFE
:1078000084F88617B0F5FA7F24D104F51875402264
:10781000294600A8FAF76AFE0022B82104F5F470A0
:10782000FAF726FEBDF8000040F2DC51884204D091
:10783000402200A92846FAF759FE04F28670C17C5E
:10784000491CC9B20A2291FBF2F202EB8203A1EBBE
:107850004301C17411B030BD002240F29C714C480C
:10786000FAF706BE2DE9F04106460C461546484F8C
:1078700097F8990709300A2190FBF1F101EB810299
:10788000A0EB420800220A2107F28F70FAF76AFE85
:107890005FFA88F808EB070080F88F6707F29970A5
:1078A00044708570BDE8F081002803D03849B1F8F4
:1078B0009A170180704700009A99993EF8B5344CA8
:1078C00001462046FFF794F904F5F47504F528768F
:1078D000324629462046FFF7E3FCB4F8E80140F2BF
:1078E000F31188420DD12846FFF796FC04F28C77FD
:1078F00039462846FFF77AFE04F29A713846FFF7B8
:10790000AAFEB4F8E801322190FBF1F1322202FB29
:107910001100312808D12846FFF7CEFE04F28C7200
:1079200031462846FFF7EEFEBDE8F1402EE70000A5
:107930000000000052499D390100C04085EB51B85C
:107940001E85F73FD7A3703D0AD71540CDCCCCCCD0
:10795000CCCC004000005440000004C09A99999992
:1079600099991B400000F8BF8DEDB5A0F7C6B03E59
:107970000AD7E33FE17A14AE47E1BA3FC976BE9F2A
:107980001A2FAD3FEC51B81E85EBA13F9999E93F05
:107990002484030000000000FDF881C0232FE34091
:1079A000DA1ED9C0F3456E40EDE88DBF0B030F3EE4
:1079B0002D8AE038A267283A8A81D23A5C560C3B7D
:1079C0008A81D23AA267283A2D8AE0380000000066
:1079D000AD9D27C0EE695740790B1FC088848C3F4E
:1079E00061738ABE9135EC3C61A1F13A0939353CAD
:1079F0004B87E23CDD04173D4B87E23C0939353CBF
:107A000061A1F13A000000001D1073BE20794C3FC7
:107A1000AE63E7BD2813F53D5676F9BB3631F43A2F
:107A200042CE113D63B55ABE5EB1083FD24136BF6A
:107A30005EB1083F63B55ABE42CE113D38B504462B
:107A4000002500E06468002C0CD0207A0A7890426F
:107A5000F8D1E0684A689042F4D120698A6890427F
:107A6000F0D1012529460FF26420FCF735F9002DED
:107A700000D10024204632BD38B504462020FEF750
:107A8000EBFE054600222021FAF7F2FC0C222146EB
:107A900005F10800FAF72AFD60686861A068A8612E
:107AA00001202877284632BDF8B500231C4601F195
:107AB0000805854A1678761C1670802686F311888C
:107AC00000BF00BF5678761C567006686F6801E0EC
:107AD00034467668002E04D0D6F80CC06745F7DA35
:107AE0000123002B0AD033680B604E603368002BF3
:107AF00001D0596000E00160316005E0002C02D047
:107B000061600C6000E001605078401E5070C0B2AF
:107B1000002802D1002080F31188FEF7E9FD002043
:107B2000F2BD10B5684C2278521C2270802282F37C
:107B3000118800BF00BF6278521C62704A680B68EF
:107B4000002B01D05A6000E002604868002801D094
:107B50000A6802600846FEF797FE6078401E607073
:107B6000C0B2002802D1002080F31188FEF7C0FDCA
:107B7000002010BD30B40268002A03D0C168D36869
:107B8000994200D04268002A28D04F490B785B1CEC
:107B90000B70802383F3118800BF00BF4B785B1C00
:107BA0004B70D36852699A1AC3689C1A92FBF3F51A
:107BB00003FB0543436103699C1A92FBF3F203FB49
:107BC000024282614878401E4870C0B2002802D14B
:107BD000002080F3118830BCFEF78ABD30BC7047AE
:107BE00070B504460D462068FFF728FF06000BD14C
:107BF0002846FFF741FF064631462046FFF754FF6F
:107C00003046FFF7B7FF02E0307F401C3077207A24
:107C1000401C2072307A002800D16660002070BDC0
:107C200010B504462068FFF709FF002801D10320A2
:107C300010BD017F491E0177217A491E2172017A08
:107C4000002901D100216160017F002903D1014693
:107C50002046FFF766FF002010BD70B51A4A137862
:107C60005B1C1370802383F3118800BF00BF53781F
:107C70005B1C5370006801E083614068002815D0E8
:107C800043695C1A83695B1A012C05DAC5686619B9
:107C900094FBF5F405FB14644461012BECDA0469F0
:107CA0001D1993FBF4F304FB1353E5E75078401ED2
:107CB0005070C0B2002802D1002080F31188FEF776
:107CC00017FD002070BD0000C06303002366632021
:107CD00025640000002141810181704738B50446C8
:107CE000002926D0002C24D0B4F90800B4F90A20C9
:107CF0001018228890FBF2F302FB130360880246FF
:107D000065689BB200FB0350FAF7E0FBB4F90A0088
:107D10002188884202DA401C608131BD09D1208966
:107D2000401C208100B2218890FBF1F201FB12007F
:107D3000208131BD2DE9F04104460D461646002D47
:107D40003ED0002C3CD0B5F9081008462A881346CE
:107D5000374607EB000C634509DB698801FB07F236
:107D60006B6801FB00312046FAF7B0FB1CE01B1AE0
:107D7000BB4201DBB04603E0A2EB01081FFA88F822
:107D8000698801FB08F26B6801FB00312046FAF7B5
:107D90009DFB6888A6EB080189B200FB01F26968C7
:107DA00000FB0840FAF792FBB5F90800381829885B
:107DB00090FBF1F201FB120028816889801B688129
:107DC000BDE8F081B0F90A10408811FB00F080B2E4
:107DD0007047B0F90A0080B270470000506002603E
:107DE0004160086070470A68F8E7486001607047C2
:107DF00001684068F9E7002007E0364901EBC0025E
:107E000041F8302011464960401C0928F5DB7047D5
:107E100010B402680B4600E01268824204D09468F5
:107E2000A342F9D1104600E0002010BC70472DE9B4
:107E3000F04104460D462646264F57F8368008E0A6
:107E4000D8F80820100002D0294620469047D8F8DC
:107E5000008007EBC6008045F2D10020BDE8F0812C
:107E600038B50C46092801DA210007D1224601461F
:107E70000FF2640000F0D4FD032032BD154901EB80
:107E8000C00521462846FFF7C3FF002806D10C2075
:107E9000FEF7E2FC84602946FFF7A5FF002032BD13
:107EA00070B504460D460B4800EBC400FFF7B0FF69
:107EB000060007D12A4621460FF2340000F0B0FD3B
:107EC000032070BDFFF794FF3046FEF7DDFC002075
:107ED00070BD00008CBC030061626E6F726D616CDE
:107EE0002072656769202825642025782900000014
:107EF00061626E6F726D616C20756E726567692864
:107F000025642C2578290000D2B2203A22BF00FA3D
:107F100002F1002070475242D041D2F1200291403C
:107F20004140D0409040414070470000012100F0A6
:107F30001F029140DFF84C21400942F820107047A1
:107F4000012100F01F029140DFF83C21400942F876
:107F50002010704780B50FF2481000F061FDDFF887
:107F60002C010021016041610161BDE8014004F084
:107F70008EBA70477CB504F096FA04460D46444E1E
:107F8000D6E900239D4208D801D3944205D2CDE919
:107F900000450FF29C1000F043FDC6E90045204665
:107FA00029467CBD80B504F07EFA4FF47A72BDE8B4
:107FB000084004F0DFBBF8B504460D4616461F46E0
:107FC00045EA040030430FD121460FF2A81000F01B
:107FD00027FD4FF4AD720FF2E4010FF2D40000F070
:107FE0001FFD0020C046C046B6F57A7F08D34FF487
:107FF0007A70B6FBF0F045194FF47A7101FB106608
:10800000B5F57A7F08D34FF47A70B5FBF0F0041918
:108010004FF47A7101FB105500F025F81B4A0698C1
:1080200010701C486421694300FB041030180021C3
:10803000C2E90201380000D01761324629462046C5
:1080400004F05BFABDE8F14002E0104800787047A8
:1080500080B5012004F05BFB01200C4988701420DE
:10806000BDE8024062E780B5002004F050FB0748FD
:1080700000218170C078002803D11420BDE802409F
:108080005EE701BD00E100E080E100E068C10300BF
:1080900060C2030040420F0000200146704700000C
:1080A0005B495D727463496E69742E2E2E0A00005E
:1080B0005B455D25732C2025640A0000443A5C571B
:1080C0006F726B73706163655C4445565C53656E9B
:1080D000736F724875625C4D4153535F50524F4A03
:1080E0004543545C50524F445C47544134584C5CB7
:1080F000525C706C6174666F726D5C6578796E6FDE
:1081000073393631305C6669726D776172655C6FA8
:10811000735C706C6174666F726D5C6578796E6F9C
:10812000735C7372635C7274635C7274632E63005D
:108130005B455D4F6F7073212C206C6173745F73AE
:10814000797374656D5F74696D655F6E73656320C7
:1081500028256C6C75292C2073797374656D5F7498
:10816000696D655F6E7365632028256C6C75290ADF
:10817000000000005B455D7274635365745469636D
:108180006B54696D652829202D207365632825644B
:108190002920697320696E76616C69640A000000A9
:1081A00080B504F018FB0D49086001BD80B500F0F2
:1081B000F1F80B4805F046FA012005F062FA05F0E7
:1081C000A3FA05F09BFB05F0A9FBFFF7C3FE0FF236
:1081D0001400BDE8024000F023BC000080690300E9
:1081E00000EA320653797374656D20626F6F7420F4
:1081F000646F6E65202121210A00000010B588B04F
:10820000044600A81421FAF7A9F905A800210A4696
:108210000B460EC00D22214600A8FAF757F904F1CB
:108220000D00CDF80D009DF80010062904DB0FF2BB
:108230004010FBF751FD63E09DF80000002801D0DD
:10824000022910D1BDF8030000280CD00422DDF86B
:108250000D1006A8FAF73AF90422DDF80D00011D09
:1082600007A8FAF733F99DF80000042848D8DFE89A
:1082700000F0030B13263700DDF80D2005A99DF84B
:108280000100FCF747FD3BE0DDF80D2005A99DF856
:108290000100FCF79BFD33E09DF80100FCF7FEFFB9
:1082A00000282DD09DF80100FCF757FE406A00F130
:1082B000080205A99DF80100FCF7D4FD20E09DF817
:1082C0000100FF2803D100A8FDF760FC18E0DDF8ED
:1082D0000D30BDF803209DF80210FCF713FE0FE0EF
:1082E0009DF80100FF2803D100A8FDF7CAFC07E0B4
:1082F000DDF80D30BDF803209DF80210FCF714FEE8
:1083000008B010BD00B591B000A84021FAF726F9D9
:1083100000A9144805F00CFB00A8FFF76FFFF7E772
:1083200010B584B0104C23461022402104F2344092
:1083300003F0C2FE022002904FF49660019004F216
:108340004C400090094B5A220FF23C0104F580602A
:1083500003F0BEFE1FBD80B50146024803F0EAFEF1
:1083600040B202BDDC760300A87203000593000052
:108370005B4552525D206F76657220434D44204D1F
:108380004158202578000000636D645F7461736B51
:108390000000000080B505F0EAFB05F0CDFC05F01B
:1083A0004AFDBDE8014005F0A7BDF8B504460D46FD
:1083B00016461F46002C0DD10FF2F00000F030FBE6
:1083C00036220FF218110FF2081000F029FB0020DE
:1083D000C046C046002D0DD10FF27C1000F020FBEE
:1083E0003B220FF2F8010FF2E80000F019FB002029
:1083F000C046C04605F0D6FD002805D13A463146B4
:108400000FF2741000F00CFB29462046BDE8F44042
:1084100005F08CBCF8B504460D4616461F46002CE8
:108420000DD10FF2701000F0FBFA49220FF2AC01EF
:108430000FF29C0000F0F4FA0020C046C046002D68
:108440000DD10FF2701000F0EBFA4E220FF28C01FA
:108450000FF27C0000F0E4FA0020C046C046300075
:108460000DD10FF2701000F0DBFA53220FF26C0105
:108470000FF25C0000F0D4FA0020C046C0463B4634
:1084800032462946204601B0BDE8F04005F048BC20
:1084900010B5044605F0BCFC012C04D02046BDE814
:1084A000104005F09ABC10BD000000005B455D6DFA
:1084B00061696C626F7857726974652829202D2074
:1084C000627566206973204E554C4C0A000000000E
:1084D0005B455D25732C2025640A0000443A5C57F7
:1084E0006F726B73706163655C4445565C53656E77
:1084F000736F724875625C4D4153535F50524F4ADF
:108500004543545C50524F445C47544134584C5C92
:10851000525C706C6174666F726D5C6578796E6FB9
:1085200073393631305C6669726D776172655C6F84
:10853000735C706C6174666F726D5C6578796E6F78
:10854000735C7372635C6D61696C626F785C6D61A2
:10855000696C626F782E63005B455D6D61696C626A
:108560006F7857726974652829202D2073697A65A0
:1085700020697320300A00005B495D6D61696C629F
:108580006F7857726974654576743A20257328258B
:1085900064290A005B455D6D61696C626F785265A4
:1085A00061642829202D20627566206973204E554C
:1085B0004C4C0A005B455D6D61696C626F78526579
:1085C00061642829202D2073697A65206973203021
:1085D0000A0000005B455D6D61696C626F785265F1
:1085E00061642829202D2063616C6C6261636B20BB
:1085F0006973204E554C4C0A0000000010B504462B
:1086000005F0B8FE01200549605410BD002105F0B9
:1086100020BF06F06AB806F0C1B8000068C20300C7
:108620000C2802D36FF400407047854A42F82010AE
:1086300006F039BA2DE9F84F04460C2C80F08980F9
:1086400006F0A4FB05467F4810F8146000EB4400D8
:108650004778304605F06DF88046384605F069F8F1
:108660008146204606F05BFA384605F089F88346D5
:10867000304605F085F88246524659460FF2C8103A
:1086800000F0CEF9BBF1010F63D0BAF1000F1AD19F
:108690004FF0000B04E00A2006F094FC0BF10A0BEB
:1086A000BBF5FA7F08D2304605F06AF88246BAF187
:1086B000000FF0D14FF0000BBBF1000F03D00FF211
:1086C000A81000F0ADF9384605F05AF88346BBF122
:1086D000000F2DD10121304605F018F80021384651
:1086E00005F014F84FF0000A01E00AF1010ABAF1AE
:1086F000640F16DA0021304605F02FF8052006F049
:108700004DFC0121304605F028F8052006F046FC16
:10871000384605F035F80128E7D10FF26C1000F06B
:108720007FF9BAF1640F03D10FF2781000F078F9F5
:108730004146304604F0EAFF4946384604F0E6FF79
:10874000204606F0B7F829462046BDE8F44F06F06B
:10875000AAB9BDE8F18FF0B587B004461D460C2CD0
:1087600001D2080602D56FF400401CE001910D9E75
:1087700003960C9805900495069201A9204606F0F0
:10878000B1FA070004D02046FFF754FF38460AE04C
:108790000E98010006D00021009133462A460F9919
:1087A00006F023FC002007B0F0BD39E71FB5069C9A
:1087B000002C01D0002B02D16FF4004009E02270A0
:1087C0000022039202920193009401232246FFF7B4
:1087D000C2FF04B010BD2DE9FF4705460E46904686
:1087E0009946DDF830A0BAF1000F02D0B9F1000FC0
:1087F00002D16FF4004020E009F101073846FEF78E
:108800002BF8040002D14FF0FF3016E04A465146E3
:10881000601CF9F75BFE84F8008000200390029052
:10882000019000903B46224631462846FFF793FFD1
:1088300005462046FEF728F8284604B0BDE8F08734
:1088400074BF0300706803005B495D534441206CB2
:10885000696E653A25642C2053434C206C696E6523
:108860003A25640A000000005B455D53434C206CD0
:10887000696E65206973207374696C6C204C4F5766
:108880002121210A000000005B495D534441206C16
:10889000696E65206973207265636F7665726564C1
:1088A0000A0000005B455D534441206C696E652001
:1088B0006973206E6F74207265636F76657265648C
:1088C0000A0000007047000030B4544982680B6A07
:1088D0009A188260012202744A692AB902604861CA
:1088E0000FF23100C8610CE001F11403846895684F
:1088F000651B012D03DB13461A68002AF7D10260BD
:10890000186048694A6A8068821A48BF486230BC69
:108910007047000010B5044610E0A0610168616175
:1089200000210174A069816081F31188A069406809
:108930008047802080F3118800BF00BF606928B1A4
:108940008168226A8A1A012AE7DB616210BD30B4AD
:10895000002300241D4638C018C01438C26082604D
:10896000416030BC704710B5802181F3118800BF91
:1089700000BF017C294CC1B104F1140100E0114693
:108980000A6892B182420ED011460A686AB18242E8
:1089900009D011460A6842B1824204D011460A68E1
:1089A0001AB18242EBD102680A60C1688160FFF7A8
:1089B0008BFF607808B980F3118810BD802181F3A6
:1089C000118800BF00BF027C14490AB30022027460
:1089D00082680B6AD21A826001F1140200E01A4622
:1089E000136893B183420ED01A4613686BB1834269
:1089F00009D01A46136843B1834204D01A4613685B
:108A00001BB18342EBD100681060486900B9C861AE
:108A1000487808B980F3118870470000C0630300EC
:108A20000EB400B582B003A90091024600AB01214B
:108A3000034878440A3001F07BF806BC5DF810FB6F
:108A400023750100010040F10980F446404200F026
:108A500005F851F000416047010000BF09D0B0FAAD
:108A600080F18840C91CC1F58461090501EBD02162
:108A70004005704780B54FF0FF3251EC100B06F007
:108A8000BDFA41EC100B01BD2DE9F8452DED088B29
:108A90000FB486B040F2FF7107989DED080B8DED85
:108AA000040BC0F30A50884208D107980024000341
:108AB00005BF069800280225012512E0012807DAE3
:108AC00006A806F04BFC012802DB0024002508E084
:108AD000079A40F2FE3161F31E520792441A4FF09A
:108AE000FF35002104A806F05AFC1A9F06460FB174
:108AF0000020388036B9DDE908230020002106F087
:108B00008DFC12D0002D13D524B2012C15D1DDE936
:108B100006230020DFF88C1306F080FC05D0012E20
:108B20000BD1DF4906F07AFC3ED10AB0CD49E8E12D
:108B3000022D04D1DDE90601E2E1012E6FDB022EF8
:108B400008BFDDE9080100F0DB81012D2AD107987B
:108B50000028099806D4002854BF9FEDD50B9FED3F
:108B6000D60BCBE100280ED456B94FF0FF3104A844
:108B700006F015FC002848BF9FEDD10B00F1BE8127
:108B80009FEDCB0BBAE156B94FF0FF3104A806F0C8
:108B900006FC002848BF9FEDB40B00F1AF819FEDAC
:108BA000C60BABE1012E11D10998002824B206D4DE
:108BB000012CACBF9FEDBE0B9FEDBF0B9EE1012CC6
:108BC000ACBF9FEDBD0B9FEDBA0B97E10998002854
:108BD00010D466B94FF0FF3104A806F0E0FB00287E
:108BE00042BF079800289FEDA00B00F187819FED01
:108BF000B20B83E106F022FC2221016066B94FF03E
:108C0000FF3104A806F0CBFB002842BF07980028DC
:108C10009FEDAB0B00F172819FEDA50B6EE1079804
:108C2000002848BF002E0CD506F008FC2121016069
:108C30000AB04FF0FF30BDEC088B6FF00041BDE88B
:108C4000F485DDE9060100220023FDF7C7FB38BFEC
:108C5000002509D381F00041CDE906014FF0FF3135
:108C600004A806F09CFB0546012C13D1DDE90601A2
:108C70007F4A804BFDF7CAFB0CD2DDE906230026B4
:108C80009FED7D8B00204FF08041FDF7EDF9CDE9A0
:108C900006011CE0DDE906239FED798B00207A496F
:108CA000FDF7E2F953EC182BFDF7DCFAFDF7AEFA0D
:108CB000A0F120063046FFF7C5FE0022734BFDF7FA
:108CC000D3F953EC182BFDF7CDFA41EC180B0FF24A
:108CD000582000EB461ADDE9060153EC182B00F092
:108CE00067FEDDE9062341EC190B51EC180BFDF78B
:108CF000B9FA02460B4651EC190B03F097FA41EC16
:108D00001A0B53EC1A2BFDF7AFF941EC1B0B8DED51
:108D1000069B06F0A5FA53EC1B2BFDF7A5F9DDE940
:108D2000062300F045FE0646884600204D4953ECD8
:108D3000182B00F03DFE00224FF08043FDF794F920
:108D400032464346FDF78EFA53EC1A2BFDF78CF9A9
:108D5000DDE90623FDF786FA41EC180B4C4A4D4B32
:108D600003F064FACDE904012046FFF76BFE41EC05
:108D7000190BDAE9000153EC192BFDF773FADDE961
:108D80000423FDF76FFACDE90401DDE90823FDF7BF
:108D90006BF90022404BCDE90201FDF737FBC0F033
:108DA000938001223D4BFDF719FB40F29180002298
:108DB0000023FDF72BFBDDE9022339BF00203849F2
:108DC00000203849FDF74EFAFDF720FA0446DDE9A8
:108DD000080153EC182BFDF747F9CDE90201DAE958
:108DE0000223DAE904019FED308BFDF73BFADDE960
:108DF0000823FDF739F953EC182BFDF735F9DDE9B8
:108E00000223FDF72FFACDE90201DAE9002351EC44
:108E1000190BFDF727FADDE90823FDF725F90646CA
:108E200088462046FFF70EFE02460B463046414676
:108E300000F0BEFD53EC182BFDF716F9DDE9022317
:108E4000FDF710FACDE902010FB13C800024009437
:108E50000022044B02A806F0F7FAA8B3012837D085
:108E600042E000BF0000F03F000000000000008072
:108E7000CD3B7F669EA0E63F000000000000F03F73
:108E8000000000000000E03F000050400000903F64
:108E9000EF39FAFE422EE63F0000E0C00000E0405D
:108EA0000000E0BF0000E03FEF39FAFE422EE63F4F
:108EB000000000000000F07F000000000000000043
:108EC000000000000000F0FF0020CDE9020007E0F4
:108ED0000020014902E000BF0000F07FCDE902015F
:108EE00006F0ACFA22210160002D1DBFDDE9020170
:108EF00081F0004141EC100B9DED020B51EC100B89
:108F00000AB0BDEC088BBDE8F48580B50020009068
:108F100053EC112B51EC100BFFF7B6FD41EC100B8D
:108F200001BD000000000000000000000000F0BFD4
:108F30000000000000000080000000000000008031
:108F40000000000000000000000000C05294EEBFCE
:108F500000000048204E51BE000000F86467BCBC11
:108F60000000000000000000000000208133EDBF81
:108F700000000080B3DB14BE000000506706A3BCF5
:108F80000000000000000000000000D0E9DCEBBFA2
:108F900000000008C39259BE00000080B0D3B8BCE6
:108FA000000000000000000000000070F98FEABF20
:108FB000000000C0A51028BE000000E8BFC0B0BC83
:108FC000000000000000000000000070284CE9BF15
:108FD00000000060134B42BE000000C03D20B8BC42
:108FE000000000000000000000000050FA10E8BF80
:108FF000000000C05FF62BBE000000905C71A7BCB3
:10900000000000000000000000000020FCDDE6BFC2
:10901000000000C0F8F154BE00000018E9F6B9BC29
:109020000000000000000000000000D0C3B2E5BF57
:1090300000000070E43254BE00000050DB06B4BCF7
:10904000000000000000000000000010EF8EE4BFF0
:1090500000000020F36252BE000000C02A879ABCC4
:109060000000000000000000000000B02272E3BF1A
:10907000000000F0E8E056BE00000028352DBDBC21
:109080000000000000000000000000000A5CE2BFD9
:10909000000000B0FA8E41BE00000040AE6FBDBCC3
:1090A000000000000000000000000000564CE1BF7E
:1090B000000000F015CD5FBE00000000141C90BC45
:1090C000000000000000000000000040BD42E0BFC2
:1090D00000000030F93457BE000000E06C1E93BC65
:1090E0000000000000000000000000E0F57DDEBF91
:1090F000000000B08A535EBE00000080DA77AABC90
:109100000000000000000000000000C09D81DCBFE6
:1091100000000000FFA226BE0000006057E2B0BCC5
:10912000000000000000000000000060F98FDABFBE
:10913000000000580A8151BE000000F05F60B8BC1A
:1091400000000000000000000000000098A8D8BF48
:10915000000000607A7F45BE000000D05433A3BCFD
:109160000000000000000000000000600FCBD6BF30
:10917000000000D091CB40BE000000406D1BA0BCA1
:109180000000000000000000000000A0FBF6D4BFBB
:1091900000000098C5CE52BE000000003A397EBCE7
:1091A0000000000000000000000000E0FE2BD3BF24
:1091B0000000004073872BBE00000000926879BC5D
:1091C000000000000000000000000040C069D1BFA6
:1091D00000000058F16353BE00000080438D7CBC4A
:1091E000000000000000000000000080D85FCFBF3A
:1091F000000000181F8354BE000000B03F42A2BC14
:1092000000000000000000000000008067FCCBBFF1
:1092100000000060FAFF53BE00000050E00DB8BC33
:1092200000000000000000000000000098A8C8BF77
:10923000000000607A7F35BE000000C0543393BC4C
:10924000000000000000000000000000DC63C5BF5B
:1092500000000058D6FF54BE00000000396490BCE6
:109260000000000000000000000000C0AD2DC2BFE3
:1092700000000080A45915BE000000E0484BABBCC4
:109280000000000000000000000000801A0BBEBFBC
:1092900000000050BF3C5ABE000000A0B364B6BC42
:1092A00000000000000000000000008004D6B7BFEE
:1092B00000000040BBCF36BE0000008076CEA8BCC8
:1092C00000000000000000000000008032BBB1BFC1
:1092D000000000402A0043BE00000028C60CBDBCB0
:1092E0000000000000000000000000009473A7BF11
:1092F000000000182B3B59BE000000C0E55DA5BC76
:10930000000000000000000000000000EE4397BFD6
:10931000000000A0E6C340BE00000020958DB5BC53
:1093200000000000000000000000000000000080BD
:10933000000000000000008000000000000000802D
:1093400000000000000000000020704730B58BB026
:10935000040001D102204BE005A80FF25C112CC9DA
:109360002CC000210A460B460EC000A81421F9F7B4
:10937000F5F81122214600A8F9F7A8F89DF8014058
:10938000082C1FD19DF8000000280BD12320FBF7EB
:1093900085FF002806D0002205A9CC20FBF7BAFCE7
:1093A000012025E09DF8000001280BD1CC20FBF71F
:1093B00081FF012806D1002205A9CC20FBF706FD7C
:1093C000012015E0232C12D19DF8000000280ED1B9
:1093D0000820FBF763FF002809D0002208A9082015
:1093E000FBF7F4FC002205A9CC20FBF793FC00203E
:1093F0000BB030BD30B58BB0050001D102204AE082
:109400000020029001902C780422691C02A8F9F730
:109410005DF80422691D01A8F9F758F821460FF2FA
:10942000A400FFF7FDFA2046FBF797FD00281DD0AA
:109430000025406A00280DD103A829460A460B469C
:109440000EC0029804900198059003A92046FBF7EE
:1094500061FC0125FCF774FA012803D10820FCF710
:109460004FFA0125002D01D0002014E006A80FF2CC
:1094700068011422F9F73AF800A80FF270010A689F
:1094800002608DF802400320ADF81B0000A906A879
:10949000FDF7B2FA02200BB030BD002803D002283D
:1094A00005D002D305E0084650E70846A2E7084683
:1094B0004AE70020704700000100000000000000A3
:1094C0000000000023234548206E6F206576656EFE
:1094D00074282564290A000005000000000000002F
:1094E0000000000000000000000000000A1A000058
:1094F00038B50C46082820D1854DE8688DF8000065
:1095000000AA012149206B691B699847207800282F
:1095100013D000EE100AB8EE400ADFED7C0A80EEB0
:10952000200A85ED040A10EE100AFCF775FD0246CC
:109530000B460FF2E810FAF7CFFB002032BD10B552
:109540000020734C00E00120002806D1A06980476C
:109550000028F8D104F1180060616369002B05D17F
:109560000FF2C410FAF7B8FB032010BD04F1080293
:10957000002147205B699847002010BD10B50446C4
:1095800064490820FEF76CFC204661494969496836
:10959000BDE81040084713B586B002A81021F8F7BF
:1095A000DDFF00A800210A4606C0594C61698968A0
:1095B0008847002801D001206AE0062202A900A8FD
:1095C000F8F794FFFCF7C4F901284ED1E0680128B0
:1095D0004BD194ED040AF7EE000A70EEC00ABDF913
:1095E000000001EE100AB8EEC11A21EE001AB4F91B
:1095F000000001EE900AF8EEE11A00EEA11ABDEEAD
:10960000C11A11EE100AADF8000000A8B0F902105E
:1096100001EE101AB8EEC11A21EE001AB4F90210C8
:1096200001EE901AF8EEE11A00EEA11ABDEEC11A91
:1096300011EE101A4180B0F9041001EE101AB8EEC4
:10964000C11A21EE000AB4F9041001EE101AB8EEA6
:10965000C11A00EE810ABDEEC00A10EE101A818018
:10966000062200A902A8F8F741FFBDF800002080FB
:1096700000A8418861808088A080082206A90DF199
:109680000E00F8F723FF02A90120FCF76FFB002072
:1096900008B010BD10B504461E490820FEF700FCB6
:1096A00020461B494969C968BDE810400847F8B51C
:1096B00004460D461646164F252C05D13178F96023
:1096C0000FF26C00FAF708FB3246294620467B6908
:1096D0001B6901B0BDE8F04018470D4B5B695B6941
:1096E00018470B4890ED020A70470B4901F1100230
:1096F000C26101220270042242700622827001229D
:1097000002820E2242824161002070470000C8425E
:10971000DC640300F1A40000C065030041434F4531
:10972000464620252E326600414343205046000025
:109730004C50462073746174757320203A20256460
:1097400000000000024601214820884B5B6A5B69EB
:10975000184770B50024854D00E0641C012C0ADA1E
:1097600004EB440005EBC006B06A80470028F4D142
:1097700006F1280068626B6A002B05D10FF2F41025
:10978000FAF7AAFA032070BD05F120020021472054
:109790005B69984705F11802022147206B6A5B69F3
:1097A0009847002070BDF8B50446FCF71CF96F4DD2
:1097B000C5E9020100222A70D5E90623002B01D158
:1097C000002A14D0D5E90467002F01D1002E0ED055
:1097D000801BB9418B420AD301D8824207D30FF2D2
:1097E0009C10FAF779FA012028700020F2BD20467B
:1097F000696A49688847002801D00120F2BD00222B
:1098000005F14001A120FBF785FA002801D00320D3
:10981000F2BD54A0FAF760FA0020F2BDD3B586B0CD
:1098200001A81021F8F79AFE504C2078002820D08B
:10983000D4E90601DDE90623D4E90467921BBB41A4
:10984000994214D801D3904211D200208DF8000023
:109850000FF23410FAF740FA0020FFF7A4FF00AA35
:1098600003214920636A1B6998470020207001206A
:1098700012E001A8616A89688847002801D00120A8
:109880000AE0082206A90DF10A00F8F71FFE01A957
:109890000420FCF76BFA002008B0D0BD38B50546AF
:1098A000324C2078002805D00FF2EC00FAF714FAB9
:1098B000002032BD002204F14001A120FBF786FA0E
:1098C000002805D12846616AC9688847002801D068
:1098D000032032BDD4E90601002901D1002803D0BC
:1098E000FCF781F8C4E904011FA0FAF7F5F900209C
:1098F00032BD1E4B5B6A5B69184780B503463D3B32
:10990000022B09D8194B1B78002B05D00FF29400BD
:10991000FAF7E2F9002002BD144B5B6A1B69BDE84F
:109920000050184710B5114C04F14C02012147209A
:10993000636A5B69984704F14C0010BD0B4890EDD9
:10994000080A70470A4901F11002C261042202703C
:10995000427006228270012202820E2242824161FE
:109960000020704747594F004759430028620300C1
:109970001066030047594F205046000047594F20BA
:10998000534B4950000000004759524F2053544157
:10999000525421210000000047594320534B4950A5
:1099A00000000000534F445220534B4950212100E6
:1099B00070B44FF0004591EA030F44BF6B40FCF7D1
:1099C0005BBC00BF841A71EB030604D26E40001B1F
:1099D000B141121973414FF4001C1CEB410F34BF0D
:1099E0007CEB430684E00C0DA4EB1356362E7DDC95
:1099F000012E43DC45EAC32343EA525312BFD2028D
:109A000092025B08240545EAC12141EA5051D2EB9C
:109A1000C020994125D407D1B0FA80F610FA06F19A
:109A200064D00020203608E0B1FA81F6B140C6F1DA
:109A3000200220FA02F21143B0404FEAF474B4EB72
:109A4000465434F001064FEA74040AD8D6F50016DD
:109A5000760D04F00044F04061FA06F25040F14007
:109A60004840C00A40EA415021F0004128BF5FEA67
:109A7000500550F1000044EBD12137E045EAC32303
:109A8000DB0A45EAC121C90AB6F120050EDD42EA2A
:109A90000242120CC5F1200603FA06F6EB4042EA38
:109AA00006056D42984161F100010DE062FA06F58C
:109AB000F240554063FA06FC82EA0C02F3405A4039
:109AC0006D42904161EB030111F4801F05D1641ECA
:109AD000620502D06D004041494121F480114308E4
:109AE00075F1004350F1000041EB045170BC704728
:109AF0001CEB410F15D223F0004352EA43060BD072
:109B00004FEA4C0CBCEB410F04D80C0D661E342EF2
:109B1000B7DDEBE7801A994150EA410608BF002102
:109B2000E4E708BF1CEB430F28BF6FF00001DDE73F
:109B30002DE9F04FA1B08246002017461D46029144
:109B40000B900DF1440B6FF000490AE017F8011B70
:109B50000298D0470290002800F0A8820B98401C81
:109B60000B90387808B90B98A2E22528EED1002096
:109B7000059006900790089009900A9001E040F047
:109B8000010017F8011F2029F9D023290DD02B2916
:109B900004D02D2906D030290AD00CE040F0020074
:109BA00080B2EEE740F00400FAE740F00800F7E783
:109BB00040F01000F4E72A290ED12968296051F8F5
:109BC000042B2960002A0D9204D5514240F0040074
:109BD0000D9180B27F1C11E000210D9109E00D99DB
:109BE000494505D001EB810302EB430130390D916A
:109BF0007F1C3A78A2F130010A29F0D339782E2956
:109C000003D04FF0FF310C911DE017F8011F2A29F6
:109C100007D1296829607F1C51F8042B29600C9218
:109C200011E000210C9109E00C99494505D001EBA8
:109C3000810302EB430130390C917F1C3A78A2F189
:109C400030010A29F0D3ADF838000FF674403978A6
:109C500005F05EFD08B117F8010B8DF83A009DF88C
:109C60003A00682802BF39786829622005D06C283C
:109C700004BF38786C2803D171208DF83A007F1C1E
:109C800011A8049017F8014BB4F125002AD01C3814
:109C900000F0CC80001F022840F2C880133800F08A
:109CA000EE80093800F0C280801E00F04F81401E17
:109CB00000F02481401E022840F2B880001F00F00E
:109CC0001D81401F00F08380401E00F0D880401EA0
:109CD00029D0C01E0CD0801E00F0D180C01E00F024
:109CE000CE803DE10120059025208DF8440043E120
:109CF0002868286050F8044B28600394DDF8308011
:109D0000B8F1000F04D52046FCF7B6FB804607E00B
:109D100042460021204605F007FD08B1A0EB0408EB
:109D2000CDF8188028E1296829604FF03C0851F8E7
:109D3000040B29600021CDE9000111A80390DDE9A1
:109D40000001049C11B908B90C9AC2B10206120FA5
:109D5000A0EB02123032D2B23A2AA8BF2732000951
:109D6000A8F1010340EA017009091A5508BF00284B
:109D7000984604D0039A08EB04039A42E6D308EB12
:109D800004000390C8F13C010C980691814209DA65
:109D9000401A08904FF6EF71BDF838000840ADF852
:109DA0003800E9E0002840F1E7809DF8380000F035
:109DB0001400102840F0E0800D98059A801A089A47
:109DC000801A401A0128C0F2D7800890D4E09DF88C
:109DD0003A0062281AD0682806D06A280CD06C286D
:109DE0001CD0712808D019E02868286050F8041B9E
:109DF00028600B980880BFE02868286050F8042B82
:109E000028600B98C117C2E90001B5E028682860F6
:109E100050F8041B28600B980870ADE02868286093
:109E200050F8041B28600B980860A5E02868C01D46
:109E300020F007022A60D2E9000108322A60CDE949
:109E40000001002903D5012005902D200CE0BDF86C
:109E50003800810703D5012005902B2004E0C007BE
:109E600004D50120059020208DF84400059911A803
:109E700008180390214600A800F0D8F97CE09DF86E
:109E80003A206C2A0DD0712A18BF6A2A09D1286895
:109E9000C01D20F007032B60D3E9000108332B60BD
:109EA00005E02968296051F8040B29600021CDE9FB
:109EB0000001682A08BF80B207D0622A08BFC0B27A
:109EC00003D0742A18BF7A2A02D10021CDE90001FB
:109ED0009DF83800000730D5DDE90001002908BFF2
:109EE00000282AD044F02000782826D130208DF890
:109EF00044008BF80140022005901EE09DF83A00D6
:109F0000294600F0D8F8CDE90001002904DA0598C7
:109F1000411C05912D210EE0BDF83800810704D5C4
:109F20000598411C05912B2105E0C00705D5059832
:109F3000411C0591202100F80B10059911A8081863
:109F40000390214600A800F0EDF815E001200590EF
:109F50002868286050F8041B28608DF844100BE036
:109F6000012005902520002C8DF8440004D0059890
:109F7000411C059100F80B400D980599401A08996D
:109F8000401A0699401A0999401A0799401A0A99E5
:109F9000A0EB01089DF8380040070FD420208DF871
:109FA0004000002408E0012310AA00A9504600F058
:109FB00070FC00287AD1641C4445F4DB059C11AE8A
:109FC0000AE016F8011B0298D047029000286DD0D5
:109FD0000B98401C0B90641E002CF2D130208DF8A1
:109FE00040000026089C08E0012310AA00A9504662
:109FF00000F04FFC002859D1761CA642F4DB069CE9
:10A00000039E0AE016F8011B0298D0470290002830
:10A010004CD00B98401C0B90641E002CF2D13020C9
:10A020008DF840000026099C07E0012310AA00A932
:10A03000504600F02EFCC8BB761CA642F5DB039808
:10A040000699079C0E1809E016F8011B0298D047E4
:10A05000029058B30B98401C0B90641E002CF3D157
:10A0600030208DF8400000260A9C07E0012310AA4A
:10A0700000A9504600F00DFCC0B9761CA642F5DBE5
:10A080009DF8380040077FF56CAD20208DF840002A
:10A09000002400E0641C4445BFF663AD012310AA10
:10A0A00000A9504600F0F5FB0028F3D04FF0FF3038
:10A0B00021B0BDE8F08F622826D068281DD06A281C
:10A0C00008D06C2827D0712804D0742823D07A288F
:10A0D0000CD020E00868C01D20F007000860D0E91F
:10A0E0000023083008601946104670470A680A6065
:10A0F00052F8040B0A60002170470A680A6052F89F
:10A10000040B0A6000B20BE00A680A6052F8040B04
:10A110000A6040B204E00A680A6052F8040B0A6060
:10A12000C11770472DE9FA4E05460A462F696F2A76
:10A1300008BF082405D041F02000782814BF0A2465
:10A1400010243C26D5E90001642A18BF692A8146FB
:10A150008A4605D1002903DAD9F100096AEB4A0AD7
:10A16000BAF1000F08BFB9F1000F0CD1286B50B93C
:10A17000082C36D195F83800000732D530203B2620
:10A1800087F83B002DE0E317484651462246FBF78F
:10A19000CFFAA4FB0023A9EB02023032D2B2A6F11F
:10A1A000010B3A2A5E4603DB9DF80030513B9A18BA
:10A1B00081465FEA010A0BF8072008BFB9F1000FDA
:10A1C00003D0E868F1198842DDD3082C09D195F84D
:10A1D0003800000705D5F05D302802D0761E30200B
:10A1E000F055C6F13C00A861F119E960296B88427D
:10A1F00008DA081A28624FF6EF71288F084028877E
:10A20000BDE8F38E00290ED595F8381001F0140141
:10A21000102908D1696B6A69891A2A6A891A081A89
:10A220000128A8BF2862BDE8F38E00002DE9F24F97
:10A2300004468EB0D4E90001CDE9020104AF9DF8D7
:10A24000380040F0200BBBF1610F0AD0206B0028D2
:10A2500048BF062004D408BFBBF1670F01D101201D
:10A2600020636168C1F30A5040F2FF7290421CD132
:10A27000080304BF2068002809D10320A0619DF8CD
:10A28000380061381A2836D30FF2486108E00320FD
:10A29000A0619DF8380061381A2829D30FF22C618B
:10A2A000E0680322F8F712F9BEE1012816DA204629
:10A2B00005F054F8012811DB00250020BBF1610FE7
:10A2C00020D1E168302201F8012B4A1CE2609DF8A0
:10A2D0003820612A0CBF782258220FE0626840F2D1
:10A2E000FE3161F31E52451A62604FF0FF30E5E720
:10A2F0000FF2D451D4E70FF2D851D1E70A70616957
:10A30000891C616110B90026002584E1BBF1610F51
:10A3100040F09780206B00284CBF2126461CDDE9C9
:10A320000201D4E900AB00220023FCF76FF836B23B
:10A330003ABF8BF00040CDE902A0CDE902AB06F1B7
:10A3400001082D1F8DF810200DF1110700E0C71D29
:10A35000B8F1010F33DBDDE9020100220023FCF735
:10A360003DF82CD21C2102A805F00AFADDE9020111
:10A37000FBF74CFFA8F10708B8F1010F814609DB94
:10A38000FEF760FB02460B46DDE90201FFF710FB1A
:10A39000CDE90201F81D072105E009F00F0200F8E0
:10A3A000012D4FEA2919B9F1010F01DB491EF4D53E
:10A3B000491E5CBF002200F8012DF9D5C7E70DF159
:10A3C0001100391AB142B8BF0E4636B230000DF155
:10A3D00011072FD4884206DA04A9411849780829C0
:10A3E000A8BF0F2100DA002104AA821800E0761E1F
:10A3F00012F80139401E8B42F9D00F2904D104A96B
:10A4000041184A78521C4A70002802D504AF761CC5
:10A410002D1D36B2701E0DD4C1190A783032D2B259
:10A420003A2A03DB9DF838303A3B9A18401E01F86F
:10A430000129F2D5206B002840F1ED80701E2063C9
:10A44000E9E0DDE9020100220023FBF7DFFF3CBF6A
:10A4500081F00041CDE902012DB247F297506843E7
:10A460004B49DFF8309190FBF1F52DB2C5F1070AA9
:10A47000BAF1010F90461CDBDDE902675FEACA70A2
:10A4800007D542464B4630463946FBF7EDFD0646BA
:10A490000F464FEA6A0A4046494642464B46FBF79A
:10A4A000E3FDBAF1000F80468946E7D1CDE90267A6
:10A4B00024E0CAF1000A0026374F14E05FEACA70B0
:10A4C00007D542464B4630463946FBF7CDFD06469A
:10A4D0000F464FEA6A0A4046494642464B46FBF75A
:10A4E000C3FD80468946BAF1000FE7D1DDE90201DC
:10A4F00032463B4601F09AFECDE90201BBF1660F00
:10A50000216BDFF898900CBF05F10A000620461871
:10A51000142EA8BF132630208DF810000DF111075E
:10A52000012E3DDBDDE90201FBF786FE07F10801A4
:10A5300004220A23B0FBF3F303EB8307A0EB4700ED
:10A54000303001F8010D0A20B3FBF0F000EB80077A
:10A55000A3EB47033033521E01F8013DE9D1083E19
:10A56000012E01F10807DBDBDDE90201FBF764FEE8
:10A57000FEF772FA02460B46DDE90201FFF718FA10
:10A5800000224B46FBF770FDCDE90201CAE700BF90
:10A59000A0860100000024400000F03F84D79741CE
:10A5A0000DF11100381A0DF1110702E0401E6D1E69
:10A5B0007F1C39783029F9D0BBF1660F02D12DB25A
:10A5C000691C04E0BBF1650F0CBF01210021226B67
:10A5D0008E1836B2B042B8BF064636B231001AD431
:10A5E000814204DAC85D3528A8BF392000DA30205E
:10A5F000CA19521E00E0761E12F80139491E834224
:10A60000F9D0392802D1C85D401CC855002902D5AF
:10A610007F1E761C6D1C2DB29DF83810009533B24C
:10A620003A46204600F003F80FB0BDE8F08F2DE960
:10A63000F043054685B01E46D5F83080012E894688
:10A64000174602DA01260FF2902749F02000BDF9E3
:10A650003040662808BF641C17D0672840F082800D
:10A6600014F1040FC0F28480444580F2818095F893
:10A670003800641C000702D44645B8BFB04624B277
:10A68000B8EB040848BF4FF0000824B2E868A96995
:10A69000012C25DA4A1C30230B54B8F1010F03DAE0
:10A6A00095F83810090702D52E211154521C18EBC9
:10A6B000040FB8BFC8F1000424B26142A044B04501
:10A6C000AA61B8BF4646696236B2EE613246AB69EE
:10A6D00039461818F7F7FAFEA8EB0600A862C1E0A1
:10A6E0000818A64218DA32463946F7F7EFFEA9698C
:10A6F0007118A01BA961B8F1010F686203DA95F81F
:10A700003800000705D5EA682E208854E869401C07
:10A71000E861C5F82880A5E022463946F7F7D6FE5D
:10A72000A8692018361BB8F1010F03DA95F8381024
:10A73000090703D5EA682E218154401CA86136B26E
:10A74000B045B8BF4646E868AB6936B23246E11953
:10A750001818F7F7BBFEA8693018A861A8EB060027
:10A7600068627FE0B9F1610F16D14FF0700918E00F
:10A77000464504DA95F83810090758BFB046B8F1D5
:10A78000010848BF4FF00008B9F1670F14BF4FF040
:10A7900045094FF0650904E0B9F1410F08BF4FF0DA
:10A7A0005009A969E86817F8013B0B544A1CB8F135
:10A7B000010F05DA95F83810090758BFAA6117D5B7
:10A7C0002E211154531CB8F1010FAB6110DB761E22
:10A7D00036B2B045B8BF464636B23246394618188A
:10A7E000F7F774FEA8693018A861A8EB0600686244
:10A7F000E868A9690F18200007F8019B03D42B20F3
:10A8000007F8010B03E02D2107F8011B6442002625
:10A810000DF1080808E00A2200A805F03DF80198AB
:10A8200008F8010B761C009C21B20129F3DA022EF4
:10A8300006DA49F02000652804BF302007F8010B34
:10A840004EB9302007F8010B07E0761E02A8305CF5
:10A85000303007F8010B012EF7DAE868A96908180B
:10A86000381AE86195F8380000F0140010280DD16E
:10A870006869A9690818696A0818E9690818A96A5D
:10A880000818696B8842BCBF081A286205B0BDE889
:10A89000F083F8B504460D4616461F46002004E036
:10A8A000E86A401CE8627F1E002047B116F8011BD1
:10A8B000A868A047A8600028F2D14FF0FF30F2BD91
:10A8C000686A6C747A4C00006E616E004E414E00F6
:10A8D000696E6600494E46003000000035488168C8
:10A8E000002904BF08B008E0EFF30982A2F12802B2
:10A8F000036882E8F84F83685A60FBF76BFE816853
:10A9000079B14A6892E8F84F036002F1280282F3B5
:10A91000098890692849814202D013F47F4F43D0BF
:10A920007047264826490968401A80F308884FF086
:10A930008071C161234981617FF0060E704701BCBF
:10A940002046DFF884E000BDFEE7204800681C498F
:10A950000968401A203820F0070080F308884FF07B
:10A9600000011448417081F3118862B600F018F8B4
:10A97000FEE703680CB44FF0000141704FF0000196
:10A9800081F311881249134A0A604FF0800181F364
:10A9900011880CBC036070470D490E4A0A6070476D
:10A9A0000B490C4A0A6070474FF0000181F311888F
:10A9B00070470000C06303008EB90000E81F030069
:10A9C000CCCC010015BC010049B90000001000000A
:10A9D00004ED00E00000001010B5EFF3108072B637
:10A9E0000A4C216841F47F01216080F31088A06E39
:10A9F00010F4700F04BFA72004F056FF4FF0007052
:10AA0000C4F81C020020C4F8140210BD20ED00E0C0
:10AA100070B504463748384E0568B5B1287A88B114
:10AA20006868A0420ED1012028723078401C307036
:10AA3000287A401E2872C0B210B9284604F048FF98
:10AA4000FBF756FEED68002DE8D170BD2B492C4A6E
:10AA50000A60002100220B468C46A0E80E10103838
:10AA6000802181F3118800BF00BF22490A68C260BB
:10AA700008602148407808B980F31188704730B5E4
:10AA80001D4D04462878401C287081B0A868217AA2
:10AA900039B9606001252572FBF72AFE284601B00E
:10AAA00030BD6168814208D01021204604F026FFA5
:10AAB000207A0028F8D1A8686060207A451C2572A9
:10AAC000FBF716FE284601B030BD0B490A78521C30
:10AAD0000A70017A491E0172C9B2002918BFFBF73A
:10AAE00007BE00B581B004F0F3FE01B05DF804EBE1
:10AAF000FBF7FEBD98C20300C063030078C20300E9
:10AB000011BA000000F5E0700268914203D3436877
:10AB10009A18914202D380680028F5D17047DFF877
:10AB20006007016891B94FF4803181604FF4805122
:10AB300041604FF0FF31C16001610421DFF844271B
:10AB40004161C2F8BC11DFF8401701600120704775
:10AB500001F1080313F0070305D001F10803C3F165
:10AB6000080303F007035918D21A8161C26042F04A
:10AB700001034B60511828234B60DFF80417096963
:10AB8000C16170472DE9F04F064601F1080010F051
:10AB9000070083B008BF884607D001F10800C0F164
:10ABA000080000F0070000EB010802F1080010F0B7
:10ABB000070006D002F10800C0F1080000F007000D
:10ABC00082181546A5EB0800A0EB030943F003002B
:10ABD00003EB080BC8F80400AB4528BF04F0ACFE3B
:10ABE0002879C00758BF04F0A7FEB9F1100F38BF8D
:10ABF00004F0A2FEB069854209D1F0684844F060D3
:10AC0000C6F818B040F00100CBF804006DE170699F
:10AC100085420BD1B0684844B060C6F814B040F02B
:10AC20000101CBF8041040F80B005EE1686800F009
:10AC30000301012940F0AD80C008C0000190C008A8
:10AC400020283AD2D5F808A0EF680090BD4208BF8E
:10AC500004F072FE554508BF04F06EFE6868009966
:10AC6000C008C000B0EBC10F18BF04F065FE00982B
:10AC700006EBC00000F128018A4507D031698A45FA
:10AC8000C0F08280DAF80C10A9427DD1574506D178
:10AC9000009A3068012191408843306076E0283086
:10ACA000874205D0306987426ED3B868A8426BD11D
:10ACB000CAF80C70C7F808A068E0EF68D5F818A0CB
:10ACC000AF420CD0A8683169884223D3C168A94239
:10ACD00004BFB968A9421DD1C760B8601CE005F186
:10ACE0001400076837B905F110000768A7B101E043
:10ACF0000846076807F114010A68002A02BF07F135
:10AD000010010A68002AF3D13169884202D3002178
:10AD1000016001E004F010FEBAF1000F36D0E869DE
:10AD200006EB800000F5987001688D4208D107603D
:10AD3000A7B9EA697068012191408843706025E0F5
:10AD40003069824508D3DAF81000A84214BFCAF867
:10AD50001470CAF8107001E004F0EEFDB7B130696C
:10AD6000874211D3C7F818A0296929B1814226BFAB
:10AD700039618F6104F0E0FD686938B1316988425A
:10AD800002D37861876101E004F0D6FD019845198E
:10AD9000814468684008400068604FEAD90549F07E
:10ADA0000100CBF8040049F80B90202D23D206EBCC
:10ADB000C50000F12807B9F1100F38BF04F0BCFD41
:10ADC000306820FA05F1C907BA4604D40121A94028
:10ADD0000843306006E0B868316988422CBF82467B
:10ADE00004F0AAFDC7F808B0CAF80CB0CBF808A068
:10ADF000CBF80C7079E05FEA192108BF002023D05E
:10AE0000B1F5803F28BF1F201ED2A1F58070000C35
:10AE100000F008008140A1F58052120C02F00402FB
:10AE20009140A1F580431B0CC0F10E0003F002031A
:10AE3000801AC01A994000EBD130C11D29FA01F2E5
:10AE400002F0010101EB4000CBF81C000022CBF81E
:10AE50001420CBF8102006EB8001726822FA00F370
:10AE6000DB0701F5987107D4012303FA00F01043C2
:10AE70007060C1F800B01DE01F2809680EBF0020F7
:10AE80004008C0F1190009FA00F000E011464A68D4
:10AE9000D208D2004A4514D0C20F01EB820202F15F
:10AEA000100340001A68002AF0D1306983421AD397
:10AEB000C3F800B0CBF81810CBF80CB0CBF808B042
:10AEC00013E032698868914228BF90420BD3C0F8E2
:10AED0000CB0C1F808B0CBF80800CBF80C1000207B
:10AEE000CBF8180001E004F027FD08F1080000F09D
:10AEF00005BE2DE9FA4D0546DFF88403006884B0ED
:10AF000008B9FFF70CFEDFF8780304998068411850
:10AF10002F31401E21EA00000499814280F0AB816C
:10AF200005F5D876B16841B1D5F8B02180188242D4
:10AF300080F0A1818142C0F09E8104F001FD0028D3
:10AF40001EBF0446D0F8008014F1010F00F0938179
:10AF5000D5F8B0014044C5F8B0017168814238BFEE
:10AF600001467160A86980BB286908B1844200D29B
:10AF70002C613461C6F814800020F06105F12801CD
:10AF8000BF48006868624FF0FF3028620020C96047
:10AF9000896001F10802801C1031D2602028926083
:10AFA000F5D3B848854203D1A8F12802214629E00B
:10AFB00055F8040CC00805EBC000A0F1080108EB2F
:10AFC0000400401AA0F128021CE005F5E0710846D3
:10AFD00000E08068D0B1026843689A189442F8D1C2
:10AFE000027B120712D4AA6903689A420ED34768FB
:10AFF0003B449A420AD208EB07014160E868A9691C
:10B0000008EB00022846FFF7A3FD1EE128698442F1
:10B01000084638BF2C6108EB040100E0806880B16D
:10B0200002688A42FAD1017B09070AD404604168A8
:10B03000414441602146049B284606B0BDE8F04DDE
:10B04000A0E5AF6939462846FFF75CFD0168406816
:10B05000401802902F3800F1080111F0070105D0C7
:10B0600000F10801C1F1080101F00701081807F11A
:10B070001001884234BF009700900098083001907A
:10B0800004F10801009800F1180A11F007014FF0CF
:10B09000000BA8F1280005D004F10801C1F1080156
:10B0A00001F007010A19401AAA61E86040F00101A5
:10B0B000516080182821416071480069E861019859
:10B0C00010F0070018BF04F037FC00991B204860FF
:10B0D00005F5E071B1E80C500198A0E80C5034611E
:10B0E000C6F81480C6F81CB00198B061029800E060
:10B0F0008A460722CAF804200AF104010A1D824286
:10B100000BF1010BF4D3BBF1020FB8BF04F014FC38
:10B110000098B84200F09980C01BC119C4084A6861
:10B12000520852004A6040F001017960C051202C61
:10B1300020D205EBC40101F12806102838BF04F025
:10B14000FBFB286820FA04F1C907B04604D40121AA
:10B15000A1400843286006E0B068296988422CBFF6
:10B16000804604F0E9FBB760C8F80C70C7F80880A7
:10B17000FE606AE0010A08BF002223D0B1F5803FDB
:10B1800028BF1F221ED2A1F58072120C02F0080205
:10B190009140A1F580531B0C03F004039940A1F5E5
:10B1A0008044240CC2F10E0204F00204D21A121BD5
:10B1B000A14002EBD131CA1D20FA02F303F00102D3
:10B1C00002EB4102FA6100237B613B6105EB8201E6
:10B1D0006B6823FA02F4E40701F5987105D40120A5
:10B1E0009040184368600F601CE01F2A09680EBF7A
:10B1F00000225208C2F1190200FA02F200E01946D8
:10B200004B68DB08DB00834210D0D30F01EB8303D4
:10B2100003F1100452002368002BF0D12869844206
:10B2200011D32760B961FF60BF600EE02A698868AA
:10B23000914228BF904206D3C7608F60B860F96022
:10B240000020B86101E004F077FBE86804998142CE
:10B2500011D2401AE860A969049A5218AA6140F014
:10B2600001005060049840F00300486006B001F10E
:10B270000800BDE8F08D002006B0BDE8F08D0000AC
:10B2800080C10300ECA603006859883C2DE9F04D0D
:10B290000446884600265FEA1820C8F1000B08BF64
:10B2A000002123D0B0F5803F28BF1F211ED2A0F57A
:10B2B0008071090C01F008018840A0F58052120C41
:10B2C00002F004029040A0F580431B0CC1F10E0176
:10B2D00003F00203891AC91A984001EBD030C11D4E
:10B2E00028FA01F202F0010101EB400104EB8100B8
:10B2F000D0F8300128B31F290EBF00224A08C2F13E
:10B30000190208FA02F2002300E052004768FF0821
:10B31000FF00A7EB08075F4503D25FEA070B06466D
:10B320000BD04769D50F00EB8500002F00691CBFCB
:10B3300087423B460028E8D1184600283CD1002E21
:10B340003CD10120884040004142084361680840E8
:10B3500000F0678141420840411E080B00F01000D8
:10B3600021FA00F2510901F0080122FA01F39A08CA
:10B3700002F00407FB405A0802F00205081823FAFD
:10B3800005F23844C2F340032818181822FA03F1D2
:10B39000081804EB8000D0F830010DE00846416841
:10B3A000C908C900A1EB080159453CBF8B460646B8
:10B3B00001690029F2D140690028F0D1002E00F087
:10B3C0003081A068A0EB0800834580F02A812069C5
:10B3D0008642C0F024817068C008C00008EB0B01F1
:10B3E000884208EB060518BF04F0A6FAAE4280F0CA
:10B3F0001681F768D6F818A0B7420CD0B06821695A
:10B40000884223D3C168B14204BFB968B1421DD19B
:10B41000C760B8601CE006F11400076837B906F190
:10B4200010000768A7B101E00846076807F114019A
:10B430000A68002A02BF07F110010A68002AF3D146
:10B440002169884202D30021016001E004F074FA0E
:10B45000BAF1000F38D0F06904EB800000F5987065
:10B4600001688E4209D10760380014D1F269606822
:10B47000012191408843606026E02069824508D31D
:10B48000DAF81000B04214BFCAF81470CAF810708D
:10B4900001E004F051FABFB12069874212D3C7F826
:10B4A00018A0306930B12169884226BF38618761B0
:10B4B00004F042FA706938B12169884202D3786198
:10B4C000876101E004F038FABBF1100F0CD208EBF1
:10B4D0000B0040F00300706008EB0B00801941681E
:10B4E00041F00101416096E048F0030070604BF0CC
:10B4F000010068604FEADB004BF805B020281DD240
:10B5000004EBC00101F12807216821FA00F2D207FB
:10B51000BB4605D4012202FA00F00843206006E091
:10B52000B868216988422CBF834604F005FABD60E3
:10B53000CBF80C50C5F808B0EF606CE05FEA1B2157
:10B5400008BF002023D0B1F5803F28BF1F201ED2A6
:10B55000A1F58070000C00F008008140A1F5805238
:10B56000120C02F004029140A1F580431B0CC0F1C3
:10B570000E0003F00203801AC01A994000EBD1308C
:10B58000C11D2BFA01F202F0010101EB4000E8615C
:10B5900000226A612A6104EB8001626822FA00F3EA
:10B5A000DB0701F5987106D4012303FA00F010437C
:10B5B00060600D601CE01F2809680EBF0020400875
:10B5C000C0F119000BFA00F000E011464A68D208F9
:10B5D000D2005A4510D0C20F01EB820202F11003D3
:10B5E00040001A68002AF0D12069834211D31D60FF
:10B5F000A961ED60AD600EE022698868914228BFC4
:10B60000904206D3C5608D60A860E9600020A86103
:10B6100001E004F091F906F10800BDE8F08D04F0B6
:10B620008BF90020BDE8F08D2DE9F84F04468846DF
:10B63000606841420840411E080B00F0100021FAEA
:10B6400000F2510901F0080122FA01F39A0802F010
:10B65000040223FA02F56B0803F00203081825FA26
:10B6600003F61018C6F340051818284426FA05F109
:10B67000081804EB8000D0F830014168C908C900FF
:10B680000646A1EB080A09E008464168C908C90056
:10B69000A1EB080151453CBF8A46064601690029D5
:10B6A000F2D140690028F0D120698642C0F0C48000
:10B6B0007068C00808EB0A09C000484508EB060B93
:10B6C00018BF04F039F95E4580F0B680F768B569B7
:10B6D000B7420CD0B0682169884223D3C168B14217
:10B6E00004BFB968B1421DD1C760B8601CE006F163
:10B6F0001400076837B906F110000768A7B101E028
:10B700000846076807F114010A68002A02BF07F11A
:10B7100010010A68002AF3D12169884202D300216E
:10B72000016001E004F008F9002D34D0F06904EB69
:10B73000800000F5987001688E4209D107603800DA
:10B7400011D1F2696068012191408843606022E074
:10B750002069854205D32869B04214BF6F612F610B
:10B7600001E004F0E9F8B7B12069874211D3BD6167
:10B77000306930B12169884226BF3861876104F0A1
:10B78000DBF8706938B12169884202D3786187613A
:10B7900001E004F0D1F8BAF1100F09D249F003002A
:10B7A000706009EB0600416841F0010141603FE033
:10B7B00048F0030070604AF00100CBF804004AF83A
:10B7C0000BA0D4F808804FEAD805202D28BF04F03C
:10B7D000B3F8B8F1000F27D0D4F81490009504EB1B
:10B7E000C50000F12805B8F1100F38BF04F0A4F827
:10B7F0002068009920FA01F2D1072F4605D4009A5B
:10B80000012191400843206006E0A8682169884230
:10B810002CBF074604F090F8C5F80890C7F80C90C4
:10B82000C9F80870C9F80C50C4F808A0C4F814B0DE
:10B8300006F10800BDE8F28F04F07EF80020BDE8B4
:10B84000F28F2DE9F04F83B00546C046C046F52D76
:10B85000DFF8C04780F007810B2D31BF102705F1BD
:10B860000B00C008C7002168FE0821FA06F010F09E
:10B87000030F42D0C04300F00100861904EBC6005C
:10B8800000F12808F700D8F808506868C008C00020
:10B89000B84218BF04F050F8D5F80890454508BFE5
:10B8A00004F04AF84D4508BF04F046F86868C0083F
:10B8B000C000B84218BF04F03FF8C84505D1206861
:10B8C0000121B140884320600DE02069814508D303
:10B8D000D9F80C00A84204D1C8F80890C9F80C8027
:10B8E00001E004F029F847F0030068607819083592
:10B8F000416841F001014160FDE0A168B94280F07A
:10B90000C480002800F0A680012505FA06F1490050
:10B910004A42B0401143084041420840411E080BD2
:10B9200000F0100021FA00F2510901F0080322FA98
:10B9300003F18A0802F0040221FA02F6710801F00C
:10B940000208181826FA08F11018C1F340064044FE
:10B95000301821FA06F202EB000804EBC80000F1EF
:10B9600028094FEAC80AD9F808607068C008C00002
:10B97000504518BF03F0E0FFD6F808B04E4508BFA9
:10B9800003F0DAFF5E4508BF03F0D6FF7068C00819
:10B99000C000504518BF03F0CFFFD94505D120683E
:10B9A00005FA08F1884320600DE02069834508D33B
:10B9B000DBF80C00B04204D1C9F808B0CBF80C9009
:10B9C00001E003F0B9FF47F003007060AAEB07083D
:10B9D000B819019048F0010001994860019848F8B1
:10B9E0000080A7684FEAD70ABAF1200F28BF03F0FA
:10B9F000A3FF47B3CDF800A004EBCA00D4F814901D
:10BA000000F1280A102F38BF03F096FF2068009934
:10BA100020FA01F2D107D34605D4009905FA01F1C5
:10BA20000843206007E0DAF80800216988422CBF4B
:10BA3000834603F081FFCAF80890CBF80C90C9F850
:10BA400008B0C9F80CA0C4F8088006F108050198F0
:10BA5000606150E06068C0B339462046FFF7E4FDFE
:10BA6000050012D047E015F1400F28BF4FF0FF3717
:10BA70000BD205F10B00C008C700606828B1394639
:10BA80002046FFF703FC050035D1A068B8421CD35F
:10BA9000C11B626910290AD3B8186061A16041F026
:10BAA00001034360095047F0030050600AE00021A1
:10BAB000A160616140F0030151608018416841F06C
:10BAC0000101416002F1080515E0E06887420DD2EE
:10BAD000C01BA169E0607A18A26140F001005060CB
:10BAE00001F1080547F00300486004E039462046AC
:10BAF000FFF7FFF90546C046C046284603B0BDE83B
:10BB0000F08F00B970472DE9F047A0F10804C04656
:10BB1000C046DFF8005528698442C0F0748261682D
:10BB200001F00302012A00F06E82CA084FEAC2083F
:10BB3000CA0708EB040936D4226811F0030F00F09D
:10BB40006482A41A84429044C0F05D8269698C4288
:10BB500000F0D880D608202E70D2D4F80CA0A768A8
:10BB6000544508BF03F0E8FEBC4208BF03F0E4FE02
:10BB70006068C008C000B0EBC60F18BF03F0DCFE61
:10BB800005EBC60000F128018F4205D029698F42DC
:10BB900051D3F968A1424ED1BA453DD1286801215F
:10BBA000B140884328604C4580F02D82D9F80400CC
:10BBB000C10740F12882810700F17A81A96989458E
:10BBC00040F0B580E868AC614044E86040F00101B5
:10BBD000616069698C4202D100216961A960E969EB
:10BBE000814280F01282DFF83004006808B9FEF765
:10BBF00096FFA969002900F00882E868292824BF77
:10BC00002846FEF77FFFE869E968884280F0FD81F9
:10BC10004FF0FF30E861F8E12830824506D028690E
:10BC2000824508D3DAF80800A04204D1C7F80CA076
:10BC3000CAF80870B7E703F07FFEB4E7E768A669C3
:10BC4000A7420BD0A168814222D3C868A04204BF9A
:10BC5000B868A0421CD1CF60B9601BE004F11401A8
:10BC60000F6837B904F110010F689FB101E0114668
:10BC70000F6807F114021368002B02BF07F11002CE
:10BC80001368002BF3D1814202D30020086001E049
:10BC900003F052FE002E86D0E06905EB800000F52F
:10BCA000987001688C4209D10760380011D1E269AF
:10BCB0006868012191408843686074E7286986427A
:10BCC00005D33069A04214BF7761376101E003F00A
:10BCD00033FE002F3FF467AF28698742ABD3BE61C4
:10BCE000216929B1814226BF39618F6103F024FEA9
:10BCF000606900283FF457AF296988429BD3786177
:10BD0000876150E799F8040000F0030003287FF4EE
:10BD10004AAFC5F80880D9F8040040084000C9F8C7
:10BD2000040048F00100606048F804806DE1696932
:10BD3000894508D1A8686C614044A86040F00101C1
:10BD40006160005161E1C008C0004FEAD00ABAF159
:10BD5000200F804436D2D9F80C70D9F80860B94564
:10BD600008BF03F0E9FDB14508BF03F0E5FDD9F8D0
:10BD70000400C008C000B0EBCA0F18BF03F0DCFD20
:10BD800005EBCA0000F128018E4206D029698E42D7
:10BD9000C0F08180F16849457DD1B74206D128685D
:10BDA000012101FA0AF18843286076E028308742B1
:10BDB00005D0286987426ED3B86848456BD1F760D3
:10BDC000BE606AE0D9F80C70D9F818604F450DD004
:10BDD000D9F808002969884223D3C168494504BFBE
:10BDE000B96849451DD1C760B8601CE009F114006D
:10BDF000076837B909F110000768A7B101E00846E4
:10BE0000076807F114010A68002A02BF07F1100150
:10BE10000A68002AF3D12969884202D3002101600F
:10BE200001E003F089FD002E37D0D9F81C0005EBA6
:10BE3000800000F59870016889450AD107603800D4
:10BE400012D1D9F81C2068680121914088436860AC
:10BE500023E02869864205D33069484514BF7761DD
:10BE6000376101E003F068FDBFB12869874212D352
:10BE7000BE61D9F8101029B1814226BF39618F61A6
:10BE800003F05AFDD9F8140038B12969884202D369
:10BE90007861876101E003F04FFD48F001006060C8
:10BEA00048F80480686984420BD1C5F80880ACE08A
:10BEB00040084000C9F8040048F00100606048F8FC
:10BEC00004804FEAD807202F22D205EBC70000F1EB
:10BED0002809B8F1100F38BF03F02EFD286820FAAA
:10BEE00007F1C9074E4604D40121B9400843286030
:10BEF00007E0D9F80800296988422CBF064603F0FC
:10BF00001BFDC9F80840F460A660C4F80C907CE002
:10BF10005FEA182008BF002123D0B0F5803F28BF7A
:10BF20001F211ED2A0F58071090C01F00801884084
:10BF3000A0F58052120C02F004029040A0F580435C
:10BF40001B0CC1F10E0103F00203891AC91A9840B3
:10BF500001EBD030C11D28FA01F202F0010101EB22
:10BF60004001E16100226261226105EB81006A68A3
:10BF700022FA01F3DB0700F5987006D4012303FAD7
:10BF800001F11143696004601CE01F2900680EBFC5
:10BF900000214908C1F1190108FA01F100E0104639
:10BFA0004268D208D200424510D0CA0F00EB82028C
:10BFB00002F1100349001A68002AF0D129698B4266
:10BFC00011D31C60A061E460A4600EE02A6981685E
:10BFD000904228BF914206D3CC608460A160E060AB
:10BFE0000020A06101E003F0A7FC286A401E28623F
:10BFF0000BD1D5F8C80100E080680028FCD14FF0D3
:10C00000FF30286201E003F097FCC046C046BDE85F
:10C01000F0870000ECA6030080C10300802282F3B9
:10C02000118800BF00BFC1600248407808B980F3A2
:10C0300011887047C063030000B581B0802282F38D
:10C04000118800BF00BF8368094A33B9507808B926
:10C0500080F31188012001B000BD13785B1C1370C0
:10C0600003F0A7FCFAF744FB002001B000BD00BFBD
:10C07000C063030010B50F4C2178491C217080214A
:10C0800081F3118800BF00BFA1688A69024205D10F
:10C09000C861082008742046FEF76BFCA168886917
:10C0A00000228A612178491E2170617809B981F3E3
:10C0B000118810BDC063030070B40024002526461B
:10C0C00070C070C018384360C260818270BC704715
:10C0D0002DE9F0470E46089F099DDDF8289004469B
:10C0E000924698463421F6F739FA1049C4F814A05C
:10C0F000207C09780843207484F8299006B1666290
:10C10000E819C008C000002140F8501D4FF08071B0
:10C11000416407490164C0F84C806FF0020141623C
:10C1200060602046BDE8F047FAF73ABBB0C20300B2
:10C130003FB9000030B50D4D2A78521C2A7081B0ED
:10C140000124802282F3118800BF00BF8268C36887
:10C150009A4202D203F00AFC0024687808B980F3FE
:10C160001188FAF7C5FA204601B030BDC06303005C
:10C1700000B581B0802282F3118800BF00BF8A69B8
:10C18000104388610A7C02F0F802082A05D1CA69C6
:10C1900002421CBF0846FAF7C7FA0348407808B9BC
:10C1A00080F3118801B000BDC0630300B5EEC00A82
:10C1B000F1EE10FA02D4B1EEC00A70476FF0004CF5
:10C1C00000EE10CA03F022BC10EE101A04204FF04B
:10C1D0007E5C01EE90CA49004FEA510100EE101A50
:10C1E00088BF0820B1F17E5F13D871EEC00ADFF876
:10C1F00038C031EE801A61EE200AF1EEE00A6145A6
:10C2000086BF80F0040080EE800A80EE200A03F0F2
:10C2100003BC490011F1807F9CBF6FF0004100EE2C
:10C22000101A43F2F3837047F404353FF0B540F23F
:10C23000FF7581EA030C0CF0004C15EA11541DBF88
:10C2400015EA1357AC42AF42E5E0BC41C1F313011C
:10C25000C3F31303801A994143F4801304D2641E7C
:10C260004000494180185941C90241EA5051B1FB8F
:10C27000F3F603FB1611A2FB0675D7EBC020A9410C
:10C2800002D2761E80185941C90241EA5051B1FBD1
:10C29000F3FE03FB1E11A2FB0E75D7EBC020A941D4
:10C2A00003D2AEF1010E80185941890241EA905142
:10C2B000760546EA8E2EB1FBF3F603FB1611A2FBC0
:10C2C0000675D7EB8020A94102D2761E801859410D
:10C2D000C90241EA50514EEA060EB1FBF3F603FBE8
:10C2E0001611A2FB0675D7EBC020A94102D2761E1B
:10C2F00080185941C90241EA5051B1FBF3F703FBE1
:10C300001711A2FB0735D3EBC020A94167F1000745
:10C310000CBF004247F0010766F3D5274FEA1E31F4
:10C32000B80814F5806412DDBD0775F1004250EBCA
:10C330000E5051EB045111F5801F5CBF41EA0C0116
:10C34000F0BD4CF07F6141F0E0410020F0BDBD0741
:10C350006D0840EA0E5041F48011D4F10104B4F1AB
:10C3600020060ADAC4F120060200E04001FA06F3D2
:10C37000E1401843B24015430EE0342C13DCC6F103
:10C38000200445EA40056D0820FA06F2154321FA1B
:10C3900006F0A1400D43002175F1004250F100006C
:10C3A00051EB0C01F0BD00205FEA0C01F0BDCFB9EC
:10C3B00092185B41B3FA83F704BFB2FA82F6BF1951
:10C3C0000B3FB7F120062FBF02FA06F3BB40C7F1BF
:10C3D000200622FA06F638BF3343BA401CB1E419EE
:10C3E000641E33E77F4231F00041B1FA81F404BFAB
:10C3F000B0FA80F6A4190B3CB4F120062FBF00FA66
:10C4000006F1A140C4F1200620FA06F638BF3143F8
:10C41000A0403C1B1AE7AC421ABF05EA1357AF42D3
:10C4200012E050EA41061CBF52EA4306BFE750EA59
:10C430004107304661461CBF41EA0551F0BD52EA52
:10C44000430C08BFC143F0BD00204FF4001616EBAB
:10C45000410F98BF16EB430F08BF16EB410F24BFE7
:10C46000C14305E016EB430F0CBF61464CEA055192
:10C47000F0BD0000DFF8D0120A68002803D042F0B7
:10C480000100086070475008400008607047DFF8FE
:10C49000B8024FF0FF314160092101604FF4807113
:10C4A00001600020E6E7F0B4DFF8A4120A6E086825
:10C4B00010F00103DFF894020CD00A6ED0E90245B7
:10C4C0004FF0144647F23577A4197D41C0E9024583
:10C4D00001230B60DFF87C12A1FB0223D20B42EA9E
:10C4E0004342D0E90245121955EBD333D0E9004558
:10C4F000101943EB0501F0BC7047F8B505460E4630
:10C500001746DFF844422068400403D50FF2482064
:10C51000FCF786FA6FF00040854201D30F20EEE071
:10C52000B5F1804F0CD30E2079004FF47A72B1FB35
:10C53000F2F101EB4601B1FBF2F101EB4505DEE062
:10C54000B5F1005F0CD30D20B9004FF47A72B1FB46
:10C55000F2F101EB8601B1FBF2F101EB8505CEE0D2
:10C56000B5F1805F0CD30C20F9004FF47A72B1FB67
:10C57000F2F101EBC601B1FBF2F101EBC505BEE042
:10C58000B5F1006F0CD30B2039014FF47A72B1FB77
:10C59000F2F101EB0611B1FBF2F101EB0515AEE092
:10C5A000B5F1806F0CD30A2079014FF47A72B1FB98
:10C5B000F2F101EB4611B1FBF2F101EB45159EE002
:10C5C000B5F1007F0CD30920B9014FF47A72B1FBA9
:10C5D000F2F101EB8611B1FBF2F101EB85158EE072
:10C5E000B5F1807F0CD30820F9014FF47A72B1FBCA
:10C5F000F2F101EBC611B1FBF2F101EBC5157EE0E2
:10C60000B5F5000F0CD3072039024FF47A72B1FB55
:10C61000F2F101EB0621B1FBF2F101EB05256EE031
:10C62000B5F5800F0CD3062079024FF47A72B1FB76
:10C63000F2F101EB4621B1FBF2F101EB45255EE0A1
:10C64000B5F5001F0CD30520B9024FF47A72B1FB87
:10C65000F2F101EB8621B1FBF2F101EB85254EE011
:10C66000B5F5801F0CD30420F9024FF47A72B1FBA8
:10C67000F2F101EBC621B1FBF2F101EBC5253EE081
:10C68000B5F5002F0FD3032040F6FE7101FB07F232
:10C690004FF47A73B2FBF3F201FB0622B2FBF3F222
:10C6A00001FB05252BE0B5F5802F0CD30220790383
:10C6B0004FF47A72B1FBF2F101EB4631B1FBF2F1CA
:10C6C00001EB45351BE0B5F5003F0CD30120B90364
:10C6D0004FF47A72B1FBF2F101EB8631B1FBF2F16A
:10C6E00001EB85350BE00020F9034FF47A72B1FBC2
:10C6F000F2F101EBC631B1FBF2F101EBC535A560FA
:10C70000216821F4705141EA80202060F1BD0E497A
:10C710000A68002803D042F480400860704722F481
:10C720008040086070470A490A6802F0040210431A
:10C7300008607047002006490A6812F004020A6087
:10C7400000D001207047000040004240E8C10300D3
:10C750003000424000CA9A3B5B495D52544320542A
:10C7600069636B2069732072756E6E696E67200A4B
:10C7700000000000F0B492B213460246B1FBF3F49D
:10C7800003FB1410110C01EB0041B1FBF3F0254643
:10C7900000240646274647EA164714EB06447D4127
:10C7A00003FB1010000410FA82F0B0FBF3F000213C
:10C7B00020186941F0BC7047DFF8401908607047E5
:10C7C000DFF8381951F830007047DFF8301901EB05
:10C7D000C0004068704780B50120FFF7F1FF406C52
:10C7E00002BD10B504460120FFF7EAFFA0F84A4059
:10C7F00010BD2DE9F04F93B00020FFF7E1FF074691
:10C8000007F580760FF674140FF634150B223146B7
:10C81000284603F053F900280BD0019600953346C3
:10C820000FF6081221460FF62410FCF7F9F8002045
:10C83000F7E03069DFF8C838984209D000900FF669
:10C84000EC0221460FF64010FCF7EAF80020E8E081
:10C85000DFF8A858AE60F069C0192861706BC01984
:10C860002865706AC019A861F16AC919A965F16BD8
:10C87000C9192967B1697269891A6960316AF269EF
:10C88000891A6961B16B726B891A6965B16A726ADA
:10C890008A1AEA61316BF36AC91AE965316CF36B84
:10C8A000C91A6967A86746F22C41DFF858389A1808
:10C8B0000A50A86F00F5C4429C322A624FF4BE723F
:10C8C0006A6200F5C8431B1DAB620023EB6200F5F2
:10C8D000C24320332B636A6300F5C4428832AA63E3
:10C8E0000022EA63A86443F2900213182B64EA64FE
:10C8F0006A6400F5C84238322A66085868668318A8
:10C90000AB666020E866A869E969081803F1600170
:10C9100088420AD2B06A0190602000900FF60C02A3
:10C9200021460FF69C00FCF77BF8686F0A90286F91
:10C930000990686D0890286D0790E86D0690A86DC5
:10C940000590E8690490A8690390686902902869D5
:10C950000190686800902B68326921460FF69800B4
:10C96000FCF75EF80D20FFF730FF12900D20FFF767
:10C9700027FF11900C20FFF728FF10900C20FFF7E5
:10C980001FFF0F900420FFF720FF0E900420FFF7F9
:10C9900017FF0D900620FFF718FF0C900620FFF7F9
:10C9A0000FFF06460820FFF710FF07460820FFF795
:10C9B00007FF80460920FFF708FF81460920FFF79F
:10C9C000FFFE82460320FFF700FF83460320FFF7A8
:10C9D000F7FE12990B9111990A91109909910F99EB
:10C9E00008910E9907910D9906910C99059104965D
:10C9F0000397CDF80880CDF80490CDF800A05B46F1
:10CA0000024621460FF66400FCF70AF81E2000904B
:10CA1000102340F2013221460FF6DC00FCF700F84B
:10CA2000A86F13B0BDE8F08F02F0CCBA016840687F
:10CA3000814201D1012070470020704701684068A1
:10CA4000491C01F00F01814201D1012070470020F3
:10CA500070472DE9F04182B004460E461746002586
:10CA6000002C01D1092000E00820FFF7A9FE804634
:10CA700040F20230874226DA72B64046FFF7DEFF08
:10CA8000002814D1D8F800004FF4427101FB008057
:10CA9000103007603A463146001DF5F717FDD8F80B
:10CAA0000000401C00F00F00C8F8000009E00FF67D
:10CAB00084020FF2C8610FF68C00FBF7B1FF6FF034
:10CAC000150562B60AE03B460FF668020FF2AC614C
:10CAD0000FF68400FBF7A4FF6FF01505002D12D1AF
:10CAE0002046401E8041C043C00F002100F007F9DE
:10CAF000050017D00FF63C020FF280610FF67400AC
:10CB0000FBF78EFF0EE0D8F80030D8F80400009054
:10CB10000FF620020FF264610FF67400FBF780FF3E
:10CB200000F00FFA2846BDE8F68170B50C460028E3
:10CB300001D1092000E00820FFF742FE054600264B
:10CB400072B6FFF773FF00280DD168684FF4427189
:10CB500001FB00501030016821606968491C01F038
:10CB60000F016960061D62B6304670BD1CB5082015
:10CB7000FFF726FE026843688168C0680FF2FC5424
:10CB80000190009121460FF62800FBF749FF09208C
:10CB9000FFF716FE026843688168C0680190009143
:10CBA00021460FF63800FBF73BFF13BD00B583B0FD
:10CBB000DFF84805806F00F5C84024308168019196
:10CBC000416800910368C2680FF2B0510FF6380057
:10CBD000FBF726FF07BDF8B5DFF82045A06F00285A
:10CBE00005D10FF64C010FF65400FBF719FF00209A
:10CBF00010E043F2900141430022A36FCA50A36F9B
:10CC0000CB185A60A36FCB189A600122A36FC91882
:10CC1000CA60401C0228ECDB002000F02FFA002143
:10CC200046F2201711E000EB4003A66F961916EBB1
:10CC30008306BD51A66F961916EB830346F22416A0
:10CC4000F550401C1E28EEDB491C022921DA4FF466
:10CC5000BE7000FB01F20020A36FD31846F28C25B2
:10CC6000E850A36FD31846F28825E850A36FD31875
:10CC700046F29025E8500120A36FD31846F2942580
:10CC8000E8500020A36FD31846F29825E850FF25FE
:10CC9000D8E7F1BD10B4DFF86414896F4FF4BE72A9
:10CCA00012FB001000F5C2422032002072B602F5DD
:10CCB000B4714B68D2F86841A3420CD003EB430037
:10CCC00002EB8000002282604A68521C1E2A00D1BA
:10CCD00000224A6010E08C68002C0DD003EB43006A
:10CCE00002EB8000002282604A68521C1E2A00D19A
:10CCF00000224A6000228A6062B610BC70472DE9AB
:10CD0000FE4F0E46DFF8F413896F4FF4BE7212FB2C
:10CD1000001101F5C2472037022802DA4FF000085F
:10CD200001E04FF004084FF00009002F06D0B8F1E1
:10CD3000000F0FF248440FF2207515D043460FF252
:10CD400018720FF238410FF21C70FBF769FE4FF0BA
:10CD5000FF309DE009EB8900009033462A462146CA
:10CD60000FF2D470FBF75CFE72B607F5B47ADAF80E
:10CD70000800002840F08E80D7F8680100EB4001E1
:10CD800017EB810B08D129460FF20070FBF748FE24
:10CD900062B64FF0FF307BE0DAF81010002000F0B0
:10CDA00028F90290002844D0002000F04AF90190B0
:10CDB00002980090DAF810302A4621460FF2E4601B
:10CDC000FBF72EFE0520FFF72FFEDAF810100020EB
:10CDD00000F00FF9002804D0484600F101090528A9
:10CDE000F0DBDAF81010002000F003F90346CDF86C
:10CDF0000490DAF8100000902A4621460FF2CC6029
:10CE0000FBF70EFEDAF81010002000F0F2F8002810
:10CE10000FD0DAF81010002000F0EBF803462A4695
:10CE200021460FF2E860FBF7FBFD62B64FF0FF30E2
:10CE30002EE0CBF800600120CBF80800DAF81000F3
:10CE4000CBF80400D7F86801401C1E2800D1002050
:10CE5000C7F86801DAF81000401C0F2800D1032041
:10CE6000CAF81000D7F86801DAF80410884202D135
:10CE70000120CAF8080062B6B8F1040F07D0BBF170
:10CE8000000F24D0DBF80410404600F00CF900201D
:10CE9000BDE8FE8F62B60520FFF7C6FDDAF8080090
:10CEA000002804D0484600F101090528F3DBDAF830
:10CEB000080000283FF44EAF2A4621460FF2A0603A
:10CEC000FBF7AEFD00F03DF84FF0FF30E0E74FF02C
:10CED000FF30DDE77FB58949896F4FF4BE7212FBE1
:10CEE000001101F5C2442034012801D181A300E0E2
:10CEF00081A304F5B4700FF2842501690391816860
:10CF0000029140680190D4F86801009022462946B9
:10CF10000FF27060FBF784FD00260FE006EB460081
:10CF2000800001198A6801924968009103593246CC
:10CF300029460FF28060FBF773FD761C1E2EEDDB99
:10CF40007FBD38B50FF234240FF28C652A46214696
:10CF50000FF29060FBF764FD0120FFF7BBFF2A464C
:10CF600021460FF29860FBF75BFD0020FFF7B2FF50
:10CF70002A4621460FF29C60FBF752FDFFF7F6FDB3
:10CF80002A4621460FF2A460FBF74AFDBDE8314076
:10CF90000CE630B4594B9C6F002C16D046F224415D
:10CFA0000A59521C0C19E5686D1CE5609C6F0D59FF
:10CFB0002C1946F238452855986F0B189B689A42F1
:10CFC00002D100220A5000E00A5030BC704710B471
:10CFD0004D4B03EBC004616003F8302010BC704778
:10CFE000494911F83000002801D010207047002076
:10CFF000704710B4444A02EBC003012412F8300019
:10D000000028586804D0806A04FA01F1084004E05E
:10D010004069103104FA01F1084010BC70473A4BE6
:10D0200003EBC000406800EB8200C0F8801070473E
:10D03000354A02EBC000406800EB8100D0F8800068
:10D040007047314901EBC00211F8300000285068E8
:10D0500001D040697047806A704710B42A4A02EBD9
:10D06000C003012404FA01F112F8300000285868C6
:10D0700001D0C16000E0016210BC704738B50446C1
:10D080004FF6FF750020FFF7ABFF05FA00F01E49D1
:10D0900001EBC40211F834100029516801D0C860B6
:10D0A00031BD086231BD38B504460D46002C01D1B2
:10D0B00000F06EFF144800EBC401012210F83400A8
:10D0C000002804D002FA05F04968C86131BD05F1B5
:10D0D000100002FA00F04968886031BD0A4A02EB8C
:10D0E000C0004068016070470448806F46F21841F4
:10D0F00008587047413243004332410084B803006E
:10D1000020C30200689BFFFFFCBF030038B5054643
:10D110000121FFF78DFF044602212846FFF788FF13
:10D12000224601460020104334BD00006970635F51
:10D130006765745F636875625F6D61700000000011
:10D140004E616E6F687562204F5300005B455D2530
:10D15000733A2025733A2025702068617320777216
:10D160006F6E67206D61676963206B65793A202572
:10D1700073202D3E2025730A000000006E616E6F43
:10D180006875622D697063005B455D25733A2025E3
:10D19000733A206970635F76657273696F6E20649D
:10D1A0006F65736E2774206D617463683A20415017
:10D1B0002025642C20436875623A2025640A00000B
:10D1C0005B495D25733A2025733A2077726F6E674D
:10D1D000207065727369737462756620616464722D
:10D1E0003A25702C2025642C206970635F656E647D
:10D1F0003A307825780A00005B495D25733A206350
:10D200006F6E74657874687562206D617020696EE8
:10D21000666F726D6174696F6E28762575290A20B4
:10D22000626C282570202564290A206F73282570D8
:10D23000202564290A206970632825702025642927
:10D240000A2072616D282570202564290A207368E0
:10D2500061726564282570202564290A2064756D33
:10D2600070282570202564290A0000005B495D258F
:10D27000733A206970635F6D617020696E666F72CA
:10D280006D6174696F6E0A206970632825702025AE
:10D2900064290A20646174615F633261282570200B
:10D2A0002564290A20646174615F613263282570F6
:10D2B000202564290A206576745F63326128257011
:10D2C000202564290A206576745F61326328257001
:10D2D000202564290A206C6F672825702025642981
:10D2E0000A207065727369737462756628257020F0
:10D2F0002564290A000000005B495D25733A206916
:10D3000070635F6D617020646174615F63683A731C
:10D31000697A653A2564206F6E2025642063686110
:10D320006E6E656C2E206576745F63683A25640ABC
:10D33000000000006970635F77726974655F646103
:10D34000746100005B495D25733A2025733A2069BA
:10D35000732066756C6C0A005B495D25733A202565
:10D36000733A20696E76616C69642073697A653AF4
:10D3700025640A005B495D25733A2025733A2066CF
:10D3800061696C206279206164645F6576740A006B
:10D390005B495D25733A2025733A206572726F727E
:10D3A0003A2065713A25642C2064713A25640A009C
:10D3B0005B495D25733A206132633A2065713A25F5
:10D3C000642064713A25642066756C6C3A2564208B
:10D3D000656D7074793A25640A0000005B495D252B
:10D3E000733A206332613A2065713A256420647192
:10D3F0003A25642066756C6C3A256420656D7074FE
:10D40000793A25640A0000005B495D25733A20746F
:10D410006F6B656E3A25642C2065713A25642C206B
:10D4200064713A25642C2073697A653A25640A0090
:10D430006970635F696E6974000000005B455D257B
:10D44000733A206970635F6D6170206973204E5577
:10D450004C4C2E0A000000006970635F6164645FD9
:10D46000657674005B455D25733A2025733A206923
:10D470006E76616C6964206970635F6576742C20D8
:10D480006F776E65723A25640A0000005B455D2582
:10D49000733A20696E76616C6964206375725F65AA
:10D4A00076740A005B455D25733A2025733A20693E
:10D4B00072713A25642070656E64696E673A3078DF
:10D4C00025782D3E307825780A0000005B495D25DF
:10D4D000733A2025733A2070656E64696E6720691F
:10D4E000727120776169743A2070656E643A2564C0
:10D4F0002069727120256420647572696E67202529
:10D50000642074696D65730A000000005B455D2549
:10D51000733A2025733A206661696C20746F20612C
:10D520006464206576742062792070656E64696E2B
:10D53000673A307825780A005B495D25733A2025E3
:10D54000733A2065767420256420647572696E676D
:10D55000202564206D732069732066756C6C0A0049
:10D560005B455D25733A2025733A206661696C201E
:10D57000746F20616464206576742062792066751A
:10D580006C6C0A005B495D25733A2065767428252A
:10D5900070292D25733A2065713A25642064713A0B
:10D5A00025642066756C6C3A2564206972713A2591
:10D5B000640A00005B495D25733A20657674256432
:10D5C000286576743A25642C6972713A25642C6654
:10D5D0003A2564290A0000006970635F64756D7004
:10D5E000000000005B495D25733A2025733A2061F5
:10D5F0003278206576656E740A0000005B495D250F
:10D60000733A2025733A20633261206576656E7423
:10D610000A0000005B495D25733A2025733A2064B7
:10D62000617461206275666665720A005B495D25FA
:10D63000733A2025733A206C6F67206275666665C1
:10D64000720A000002F050BA80B50F280BDB2322CB
:10D650000FF240010FF23000FBF7E2F90020C04664
:10D66000C046002002BDBDE8024002F07DBB0F288D
:10D6700001DB00207047102901D30020704702F021
:10D68000B9BB02F0F4BB00005B455D25732C20257F
:10D69000640A0000443A5C576F726B737061636593
:10D6A0005C4445565C53656E736F724875625C4DA1
:10D6B0004153535F50524F4A4543545C50524F447C
:10D6C0005C47544134584C5C525C706C6174666FBA
:10D6D000726D5C6578796E6F73393631305C66696E
:10D6E000726D776172655C6F735C706C6174666F8C
:10D6F000726D5C6578796E6F735C7372635C636D79
:10D70000755C636D752E630002F056BC80B52128F0
:10D710000BDB25220FF234110FF22410FBF780F9F6
:10D720000020BDE8024001F05FBCBDE8044002F00B
:10D7300053BC80B521280CDB2E220FF210110FF202
:10D740000010FBF76DF90020C046C0464FF0FF30D7
:10D7500002BDBDE8024002F05DBC80B521280BDBB4
:10D7600039220FF2E8010FF2D800FBF759F9002037
:10D77000BDE8024001F038BCBDE8044002F067BCDF
:10D7800080B521280CDB45220FF2C0010FF2B0005A
:10D79000FBF746F90020C046C0464FF0FF3002BDFF
:10D7A000BDE8024002F071BC80B521280BDB51229C
:10D7B0000FF298010FF28800FBF732F90020BDE864
:10D7C000024001F011BCBDE8044002F07DBC80B510
:10D7D00021280BDB5E220FF274010FF26400FBF7CD
:10D7E0001FF90020BDE8024001F0FEBBBDE8044087
:10D7F00002F088BC80B521280BDB6A220FF24C01B5
:10D800000FF23C00FBF70CF90020BDE8024001F0EC
:10D81000EBBBBDE8044002F093BC80B521280BDBD4
:10D8200076220FF228010FF21800FBF7F9F800201A
:10D83000BDE8024001F0D8BBBDE8044002F09EBC48
:10D840005B455D25732C2025640A0000443A5C5733
:10D850006F726B73706163655C4445565C53656EB3
:10D86000736F724875625C4D4153535F50524F4A1B
:10D870004543545C50524F445C47544134584C5CCF
:10D88000525C706C6174666F726D5C6578796E6FF6
:10D8900073393631305C6669726D776172655C6FC1
:10D8A000735C706C6174666F726D5C6578796E6FB5
:10D8B000735C7372635C6770696F5C6770696F2E0D
:10D8C00063000000102810D8DFE800F0090B090BF6
:10D8D000090B090B0F0F0F0F0F0F0F0F0D0000207B
:10D8E00070470120704702207047032070470249AB
:10D8F00051F82000704700005C5C030003F074BA2C
:10D9000010B5044603F07DFA20702078FFF7DAFFA7
:10D9100060702078FFF7EBFF606010BD80B503F00A
:10D9200099FA03F0DFFABDE8014003F0EDBA000018
:10D9300030B5044610480D460178491C017081B08D
:10D94000802080F3118800BF00BFA06858B9402133
:10D95000204601F0D3FF802080F3118800BF00BF74
:10D96000A0680028F3D02946204602F022F801B032
:10D97000BDE83040F8F7BCBEC0630300012100F0F1
:10D980001F0291408A4A400942F820107047012145
:10D9900000F01F029140874A400942F8201070476A
:10D9A00080B50020FFF7A0FB0FF210210FF2182026
:10D9B000BDE80440FBF734B880B50246D21E052A04
:10D9C0000BD8DFE802F0030C0C030A070020FFF776
:10D9D00044FB04E0FFF7E4FF01E000F051F9002010
:10D9E000FFF794FBBDE80440FAF7C3BAF0B585B081
:10D9F0000020FFF726FB04460020FFF7F1FA05465A
:10DA000005F10F062046F040C00747D5032100204E
:10DA1000FFF70EFBC7B2022F0AD1032200210846EE
:10DA2000FFF7FDFA0020FEF7DCFE00F0B6FA0BE08F
:10DA3000012F09D100F0ACFA032200210846FFF7BC
:10DA4000EEFA0120FEF7CDFE082F01D100F0A0FA7A
:10DA50000120B040844331460020FFF7FEFA022F38
:10DA600003D00F210020FFF71EFB012F05D0022F4E
:10DA700003D0042F01D0082F10D100A80FF2EC1111
:10DA80001422F4F733FDADF8037000A8FAF763FC35
:10DA9000002803D00FF26410FAF7C2FF002C27D041
:10DAA0000AE0076829460020FFF7D7FA29463846DA
:10DAB000C0B2FFF781FF6D1CB54219DA2046E8407D
:10DAC000C007F8D50120FFF7E5F80028E9D100F0FC
:10DAD00033F90020FFF7B5FA009023462A460FF2EB
:10DAE00004110FF22810FAF79BFF0020FFF7C6FA87
:10DAF00005B0F0BD70B50120FFF7A3FA0446012080
:10DB0000FFF76EFA054621460FF23410FAF788FF48
:10DB10002E460BE02046F040C00706D5304600F008
:10DB200047F931460120FFF798FA761C05F11000FD
:10DB30008642EFD370BD70B50FF21010FAF770FF88
:10DB40000320FFF77EFA04460320FFF749FA054653
:10DB50002E4607E02046F040C00702D5701B00F0BB
:10DB6000A6F9761C05F10F008642F3D370BD80B58F
:10DB70000020FEF721FEFEF73CFE002817D00C2007
:10DB8000FEF71EFE0C4908600E20FFF700FF0E2076
:10DB9000FFF7F4FE1020FFF7FAFE1020FFF7EEFE6D
:10DBA0001120FFF7F4FE1120BDE80240E6E601BDBA
:10DBB00000E100E080E200E08CC2030068616E6476
:10DBC0006C654465627567005B495D25733A206446
:10DBD0006F65736E277420737570706F72746564EF
:10DBE0002E0A00006D61696C626F7841505F495286
:10DBF0005148616E646C6572000000004D5347200F
:10DC0000426F782046756C6C0A0000005B455D250C
:10DC100073282564293A206576656E7471206973CE
:10DC200020656D7074792C207374617475733A304B
:10DC30007825782853523A30782578290A00000050
:10DC40005B495D6841504D3A25780A005B495D4D5E
:10DC500061696C626F78476E737332436875625F97
:10DC600049525148616E646C65720A0003FF3800C6
:10DC700000000000000000000000000000000000A4
:10DC800010B5ADF5427D334C2078002821D000221C
:10DC900040F2013101A8F4F7EBFB00A90120FEF7E7
:10DCA00044FF010003D0009A01A8F4F70FFC00988C
:10DCB00040F20231884204D2014601A800F036F851
:10DCC0002BE002460FF294010FF2AC00FAF7A8FE27
:10DCD00023E0A068002820D000A90120FEF725FF3E
:10DCE000002807D0009A0146A068F4F7EFFB002057
:10DCF000009002E04FF0FF300090A16863681800C8
:10DD000003D0009AE068984707E000230A460FF224
:10DD10004C010FF28000FAF783FE0DF5427D10BD35
:10DD20000C494A60CB608860002070470A4692B276
:10DD300001460020FEF78DBE80B5FEF74CFF0022A5
:10DD400005491046FFF743F901210020BDE80440D2
:10DD5000FFF7C4B9D8C10300000038406D61696C99
:10DD6000626F7844727648616E646C6552784D6576
:10DD700073736167650000005B455D25733A206938
:10DD80006E76616C69642073697A653A2025640A4D
:10DD9000000000005B455D25733A206E6F206361D3
:10DDA0006C6C6261636B3A2025782C2025780A0020
:10DDB00010B5044621460FF2A400FAF731FE002CFC
:10DDC0000AD102210120FFF733F901460FF2A0002A
:10DDD000BDE81040FAF724BE10BD38B51C4C4FF416
:10DDE000803504E00FF29C00FAF71AFE256001204E
:10DDF000FFF727F90028FAD000210120FFF72DF9BD
:10DE000002210120FFF714F90100EBD5256031BD97
:10DE100080B510490A68521C53015B090B6000224F
:10DE200040EA03110120FFF7FAF800210120BDE8C4
:10DE30000440FFF738B980B5002207490120FFF7F9
:10DE4000C6F801210846BDE80440FFF747B90000C5
:10DE500080E200E088C20300000037405B495D209B
:10DE60006841504D3A6972713D25640A0000000016
:10DE70005B495D206841504D3A7372323D25303820
:10DE8000580A00005B495D453A3078253038580A19
:10DE900000000000234A42F820107047014603208A
:10DEA000FFF701B900F110010320FFF7D6B810B554
:10DEB0000446FFF7F7FF1B4850F824100A0008D16A
:10DEC00022460FF274010FF28800BDE81040FAF705
:10DED000A7BD002C01D0012C01D1884703E0022C02
:10DEE00001D180688047002C01D0012C03D120464D
:10DEF000BDE81040D2E710BD80B501220A490320D9
:10DF0000FFF765F803F0D8F908490020FFF7C2FFD2
:10DF100007490120FFF7BEFF06490220BDE8044083
:10DF2000B8E70000A0BD0300000039407DEF00000D
:10DF300087EF0000892001006D61696C626F78478E
:10DF40006E737344727668616E646C6549727100B9
:10DF50005B455D25733A2057726F6E6720696E745A
:10DF60006572727570742068617070656E65642882
:10DF70006576656E743A20256429000041F2100030
:10DF80003C494860704740F201103A494860704788
:10DF900041F2100037490860704740F201103549DE
:10DFA0000860704740F2011032494A68824204D149
:10DFB0000968814201D100207047012070470000AC
:10DFC0002DE9F0412C4E346800254FF0FF302B49ED
:10DFD000086072B62846FAF75BFA03F0B3FA074610
:10DFE000274803F0ABFA274A1068C00203D54FF464
:10DFF000801025490860106829462040294001D139
:10E0000000280CD06FF0604003F09AFA384603F015
:10E0100095FA34600220FAF73BFA62B628E0DFF89E
:10E02000688010686040C8F8000018480160006807
:10E03000C00303D54FF00070154908600120FAF7BE
:10E0400027FA4FF48030306030BF00BFFAF70BF88A
:10E0500029460120FFF701F84FF48810C8F80000A6
:10E060006FF0604003F06CFA384603F067FA3460F2
:10E07000BDE8F0817469030000E100E080E100E0A8
:10E08000FFFFFE1F00E200E080E200E010E000E0A1
:10E0900004ED00E0103003689343002900D01343DF
:10E0A0000360704701680A68437B002B02D122F0AD
:10E0B000100201E042F01002837B002B02D122F01B
:10E0C000080201E042F00802C37B002B02D122F0DB
:10E0D000040201E042F004020A6002F00103016858
:10E0E000096801F001019942F9D1704703689B0862
:10E0F0009B00002901D043F00203002A01D043F025
:10E1000001030360704710B582B004460022114637
:10E11000FFF7ECFF00202062204601680091009983
:10E1200041F0200100910099016004F114010A6896
:10E130000092009A12F4FC3FF9D10A680092009A0A
:10E1400012F4FC6FF9D101680091009921F02001CF
:10E150000091009901600168009100998906FAD444
:10E1600013BD2030036823F48033036062F30F0390
:10E17000002901D043F480330360704710B4016874
:10E1800008310A6890F83030012B02D142F00402C5
:10E1900001E022F0040290F83130012B02D142F06C
:10E1A000020201E022F0020290F84430012B02D179
:10E1B00042F0010201E052085200036ADFF86046B3
:10E1C000002B02D0224042EAC34424F4C02290F83B
:10E1D000243042EA434222F4FC62C36A42EA431218
:10E1E00022F4FC32836A42EAC32290F865000028D8
:10E1F00002D042F0080001E022F00800086010BCE4
:10E20000704708300268002902D042F0080101E09E
:10E2100022F008010160704701680C310A6890F82B
:10E220004C30002B02D042F0040201E022F0040244
:10E2300022F47C72806C42EA00100860704790F80B
:10E240005C1090F85D2042EA01110068816270471D
:10E2500090F85E100068C16270471030016841F0AC
:10E260000301016070471F21416270470C30026852
:10E27000002902D05108490001E042F0010101608B
:10E280000020704770B504460FF2AC550FF2A0564F
:10E290002368002231462846FAF7C2FBA368082209
:10E2A00031462846FAF7BCFBE3680C223146284683
:10E2B000FAF7B6FB2369102231462846FAF7B0FB7D
:10E2C0006369142231462846FAF7AAFBA36918228B
:10E2D00031462846FAF7A4FBE3691C22314628465A
:10E2E000FAF79EFB236A202231462846FAF798FB6C
:10E2F000636A242231462846FAF792FBA36A282251
:10E3000031462846FAF78CFBE36A2C223146284630
:10E31000BDE87040FAF784BBF0B583B0064600272D
:10E32000F9F7BAFE04460D467069800121D43846DB
:10E33000471C42F211718842F6DB00200146001BA7
:10E34000A941DFF8E02400239942EDD301D890429F
:10E35000EAD300200146CDE9000122462B460FF208
:10E36000F4410FF20850FAF75BFB3046BDE8FE407F
:10E3700088E7F7BD10B4DFF8B024E42303FB0020E6
:10E380004A68426091F84C2080F84C20021D0B1D19
:10E390005C6954615C7A54729C7A9472DC7AD472AF
:10E3A0001C6914611B7E137691F8242080F82420C8
:10E3B00000F1240201F124031C7B14735B7B537373
:10E3C00091F85E1080F85E1010BC704710B5DFF851
:10E3D0005814E42202FB00140120E0622046FFF7FB
:10E3E00061FE2046FFF7CAFE2046FFF715FF2046D4
:10E3F000FFF725FF2046FFF72BFF94F83100042894
:10E4000003D094F83000042802D12068FFF725FFDC
:10E410002068FFF728FF94F83100042803D094F80F
:10E420003000042810D10020C4F89000C4F8A000E7
:10E43000C4F89800C4F8A800C4F8B000C4F8B80044
:10E44000C4F8C800C4F8C0002068FFF75CFE0020D4
:10E4500010BD80B5E4214143DFF8CC230FF23C43EB
:10E4600053F820308B5089184860FFF7AFFF002821
:10E4700002D04FF0FF3002BD002002BDF8B50F46BC
:10E480001D46DFF8A413E42303FB001696F82400CE
:10E49000002841D196F84C000028144614D0294693
:10E4A00003E017F8012B0276491E30680029F8D1E5
:10E4B00001221146FFF71AFE002D25D03068007F9B
:10E4C00004F8010B6D1EF7E7002211463068FFF7D4
:10E4D00048FE012211463068FFF708FE012130682E
:10E4E000FFF7C4FE0AE017F8011B01763068FFF75A
:10E4F00013FF3068007F04F8010B6D1E3068002D9B
:10E50000F1D10021FFF7B2FE3068FFF705FF306858
:10E51000FFF7F9FD0020F2BD012843D196F84C0029
:10E520000028144614D0294603E037F8022B028352
:10E53000491E30680029F8D101221146FFF7D6FDA7
:10E54000002DE1D03068808B24F8020B6D1EF7E7B8
:10E55000002211463068FFF704FE012211463068A0
:10E56000FFF7C4FD002D0EE0401EFDD100213068F4
:10E57000FFF77CFE3068808B24F8020B3068808BBC
:10E5800024F8020B6D1EBFD001213068FFF76EFE2C
:10E5900037F8020B3168088337F8020B31680883BB
:10E5A0009620E2E70228AFD196F84C0000281446E6
:10E5B00014D0294603E057F8042B8261491E3068C5
:10E5C0000029F8D101221146FFF790FD002D9BD0C4
:10E5D0003068C06944F8040B6D1EF7E7002211464D
:10E5E0003068FFF7BEFD012211463068FFF77EFD5F
:10E5F000002D0EE0401EFDD100213068FFF736FEF1
:10E600003068C06944F8040B3068C06944F8040BF2
:10E610006D1E3FF479AF01213068FFF727FE57F8F0
:10E62000040B3168886157F8040B316888619620C3
:10E63000E1E738B57C4CE42505FB0044C4F8CC1078
:10E64000C4F8D0300020C4F8D400C4F8D820C4F8EE
:10E65000DC30C4F8E000022201212068FFF71AFD37
:10E66000012211462068FFF715FD002032BD2DE97B
:10E67000F84304460D4616461F464FF000086A4808
:10E68000E42101FB040999F86400002803D0D9F8BB
:10E690000000FFF738FD99F86500002804D001213B
:10E6A000D9F80000FFF7ADFD99F83100002807D137
:10E6B0003B46324629462046FFF7E0FE804608E00A
:10E6C000042806D13B46324629462046FFF7B1FFD3
:10E6D000804699F86500002804D00021D9F8000090
:10E6E000FFF78FFD4046BDE8F2832DE9F84F044661
:10E6F0008A4615461E464C48E42101FB04074FF0AC
:10E700000009FF2E02D94FF0FF080FE0B0460DE0E0
:10E710000BF1040105EB8900F3F7D8FE08EB0900C3
:10E72000864201D2A6EB0908C144CA44B14532D29F
:10E73000DFF8F8B0584697F82410002903D14AF0C2
:10E740008001017008E0012903D14AF400410180F1
:10E7500002E04AF00041016008F101035A465946BF
:10E760002046FFF784FF002816D197F824000028E0
:10E7700007D142460BF1010109EB0500F3F7A6FEB4
:10E78000CCE701284246C3D10BF1020105EB490059
:10E79000F3F79CFEC2E70020BDE8F28F2DE9F84FA9
:10E7A00004468A4615461E461F48E42101FB04071D
:10E7B0004FF00009FF2E02D94FF0FF0809E0B046E4
:10E7C00007E008EB0900864201D2A6EB0908C14424
:10E7D000CA44B14520D2DFF854B05846014697F8F4
:10E7E0002420002A07D181F800A032462946401C87
:10E7F000F3F76CFE06E0C1F800A0B2002946001D48
:10E80000F3F764FE08F10103002259462046FFF7A2
:10E810002EFF0028D5D000E00020BDE8F28F0000D8
:10E820000000F81F81969800C08B0300C895030074
:10E8300064756D70537069005B4C4F475F494E467D
:10E840004F5D25733A202B25643A20307825780ACD
:10E85000000000005F5F776169745F756E74696CBA
:10E860005F74785F646F6E65000000005B4C4F471B
:10E870005F4552524F525D25733A206F75742120C7
:10E88000696E54696D653A256C6C752C206F7574D2
:10E8900054696D653A256C6C750A000000001C40D7
:10E8A00000007040000070400000724000007440A2
:10E8B0000000764000EB40010801DFF8E814425800
:10E8C000136843F000431360405801684900490849
:10E8D0000160704770B4022802D2DFF8CC4401E036
:10E8E000DFF8C84400EB40021001DFF8B8248318B9
:10E8F0005B6886581B01B4FBF3F3DDB24FF0FF33C6
:10E9000001292DD106F15C010E6826F47F0646EA46
:10E9100005460E60691CC4EBC404DFF89454B4FBD4
:10E92000F5F4642515FB01F1B4FBF1F1845858347A
:10E9300025682D0A1E46CE408E40F6B256EA0525C1
:10E940002560491E80585430026822F47F021C461C
:10E95000CC4004FA01F1C9B242EA014101602CE065
:10E9600006F168010E6826F47F0646EA05460E6049
:10E97000691C04EBC404DFF83854B4FBF5F401EB74
:10E9800081056900B4FBF1F18458643425682D0ACF
:10E990001E46CE408E40F6B256EA05252560491E39
:10E9A00080586030026822F47F021C46CC4004FA92
:10E9B00001F1C9B242EA01410160002070BC704718
:10E9C00010B504460021FFF785FF002810D1DFF8BD
:10E9D000D40304EB440100EB01104068DFF8D413CA
:10E9E000884208D301212046FFF774FF002802D097
:10E9F000DFF8C40310BD002010BD38B500EB4001A6
:10EA00000C01DFF8A053605901680FF2C030FAF72B
:10EA100007F8605941680FF2C830FAF701F86059F9
:10EA200081680FF2D430F9F7FBFF6059016A0FF2E9
:10EA3000E430F9F7F5FF6059416A0FF2EC30F9F76D
:10EA4000EFFF6059016B0FF2F830F9F7E9FF6059F9
:10EA5000016C0FF20440F9F7E3FF6059416C0FF2CB
:10EA60000C40F9F7DDFF6059016D0FF21440F9F722
:10EA7000D7FF6059416D0FF22440F9F7D1FF60597B
:10EA8000816D0FF23040F9F7CBFF6059C16D0FF285
:10EA90003C40F9F7C5FF6059016F0FF24840BDE8EF
:10EAA0003440F9F7BDBF2DE9F8430746884607EB28
:10EAB00047000401BB4D6619307BC00701D500201B
:10EAC0002BE00FF2A84050F827006051C6F80480F0
:10EAD0000020B060F06030613846FFF7EBFE60590F
:10EAE000016841F00809C0F800903846FFF768FF58
:10EAF0000F2061598860AF48804506D36059403087
:10EB0000016841F00059C0F8009049F00040615997
:10EB1000086401203061F0600020BDE8F283A14963
:10EB200000EB400201EB02100021C16001610846C8
:10EB3000704780B59B4900EB400210014058016DC1
:10EB400001F00F00012805D00FF2AC30F9F768FF93
:10EB5000002002BD012002BD2DE9F84F04460D46FC
:10EB6000002604EB44000701DFF8388257F808302C
:10EB70001968586C4833D3F800C04FEA4C0C4FEA80
:10EB80005C0CC3F800C08D4B57F808C0CCF80430BB
:10EB90002B79DB0704D541F0400140F4803003E0DD
:10EBA00021F0400120F48030012A02D140F40030ED
:10EBB00001E020F4003057F808207032136803F4A5
:10EBC000700395F800C00CF07F0C43EA8C231360AF
:10EBD00057F808201160000C2979C90703D5A968E6
:10EBE00051EA004002E0E96851EA004057F8081095
:10EBF000486457F808004430016841F00041016062
:10EC0000DFF8BC91CA4607EB080BDBF8080029794E
:10EC1000C9072BD5002862D102F094FC40F02100F6
:10EC200002F08CFC802057F80810086265490846FD
:10EC30000246501E002A4BD057F80820136BDB0108
:10EC400004D4926B28693254761C0846AA6896420E
:10EC5000EED308460146481E002939D057F808105F
:10EC600024310A680A60110630D4F3E700281DD168
:10EC700002F068FC40F0210002F060FC802057F8B0
:10EC8000081008624F480AE057F808100A6B02F0B3
:10EC90007F02102A03D26A69B25C761C4A6301467D
:10ECA000481E002902D0E9688E42EDD3DBF8080047
:10ECB000002814D143480146481E002908D057F8BF
:10ECC000081024310A680A601106F4D54FF0000AD2
:10ECD000CA4504D12046FFF790FE484600E0504662
:10ECE000BDE8F28F2DE9F04104460D4601260027CC
:10ECF000002D02D16FF4004046E02A4804EB4401A5
:10ED000000EB011898F80C00C00701D42E483BE036
:10ED10002046FFF70EFF002807D12046FFF7FFFE31
:10ED2000D8F804102046FFF7BEFE38466860A86891
:10ED3000002800D03E46E868002824D04FF48040E8
:10ED40006860324629462046FFF706FF070006D0D6
:10ED500039460FF2D010F9F763FE384614E0002E62
:10ED600011D1686840F00100686001222946204600
:10ED7000FFF7F2FE070006D039460FF2CC10F9F784
:10ED80004FFE384600E03846BDE8F0810C2801D33C
:10ED900000207047034900EB400201EB021040687D
:10EDA00070470000ACA2030000EA32060080BB00FE
:10EDB00040420F00811A0600FE7FFFFF830008001B
:10EDC000FD7FFFFFA0860100FC7FFFFF5B495D49DF
:10EDD00032432043544C203A2025780A000000009A
:10EDE0005B495D493243204649464F5F43544C20BE
:10EDF0003A2025580A0000005B495D4932432054FF
:10EE00005241494C494E475F43544C203A202558C3
:10EE10000A0000005B495D49324320494E545F457A
:10EE20004E203A2025580A005B495D49324320496B
:10EE30004E545F53544154203A2025580A00000094
:10EE40005B495D493243204649464F5F5354415424
:10EE5000203A2025580A00005B495D49324320438F
:10EE60004F4E46203A2025580A0000005B495D4974
:10EE7000324320434F4E4632203A2025580A0000A4
:10EE80005B495D493243205452414E532053544113
:10EE9000545553203A2025580A0000005B495D492B
:10EEA00032432054494D494E4720485331203A209F
:10EEB00025580A005B495D4932432054494D494E6B
:10EEC0004720485332203A2025580A005B495D49C3
:10EED00032432054494D494E4720485333203A206D
:10EEE00025580A005B495D49324320414444522081
:10EEF0003A2025580A0000005B455D493243204214
:10EF00007573206973206E6F742049444C45203A14
:10EF1000205452414E535F535441545553203D2089
:10EF200025780A005B455D6932634472764D6173F2
:10EF3000746572205472616E736D697420466169E4
:10EF40006C203A2025640A005B455D693263447297
:10EF5000764D6173746572205265636569766520CC
:10EF60004661696C203A2025640A000000001C40BC
:10EF700000001D4000007040000071400000724021
:10EF800000007340000074400000754000007640AF
:10EF900000007740000078400000794010B582B052
:10EFA00004460320FEF750FB0549B0FBF1F0604337
:10EFB00000900098411E00910028FAD113BD000076
:10EFC000404B4C0010B582B004460320FEF73CFBDA
:10EFD00041F28831B0FBF1F0604300900098411E8F
:10EFE00000910028FAD113BD704710B504460846B9
:10EFF00011461A46029BA04710BD00002DE9F84CAF
:10F000002DED068B154603B4C1F30A5040F2FF7193
:10F0100088420CD101980024000304BF0098002806
:10F0200002D1019800281BD4DDE9000113E1012879
:10F030000FDA00A800F092F901280ADB00F0FEF9CF
:10F040002221016002B00020BDEC068BA249BDE880
:10F05000F48C019A40F2FE3161F31E520192441A7F
:10F06000019800280CD500F0E9F92121016002B0D7
:10F070004FF0FF30BDEC068B6FF00041BDE8F48C23
:10F08000DDE90001954A964BF7F7C0F909D2DDE9B1
:10F09000002300204FF08041F6F7E6FFCDE90001A4
:10F0A000641EDDE9002300208E49F7F7DBF8DDE977
:10F0B000002341EC180B00208B49F7F7D3F80246E8
:10F0C0000B4651EC180BFDF7B1F841EC190B53EC62
:10F0D000192BF6F7C9FF41EC1A0B53EC1A2B834896
:10F0E0008349F6F7C1FF834A834BF7F7BBF853EC2C
:10F0F0001A2BF6F7B9FF814A814BF7F7B3F853ECB7
:10F100001A2BF6F7B1FF7F4A7F4BF7F7ABF853ECBA
:10F110001A2BF6F7A9FF7D4A7D4BF7F7A3F853ECBE
:10F120001A2BF6F7A1FF7B4A7B4BF7F79BF853ECC2
:10F130001A2BF6F799FF794A794BF7F793F853ECC6
:10F140001A2BF6F791FF02460B4651EC180BFAF713
:10F150002FFC53EC192BF6F787FF41EC190B20B26B
:10F16000F9F770FC41EC1A0BCDB953EC1A2B6D4832
:10F170006D49F6F779FF53EC192BFAF719FC53ECAC
:10F18000182BF7F76FF804460D4653EC1A2B4FF087
:10F1900040406649F6F768FF22462B4659E0012DAC
:10F1A00053EC182B34DB00206149F6F75DFF8246F3
:10F1B0008B4653EC182B5F485F49F6F755FF064620
:10F1C0000F4653EC1A2B5D485D49F6F74DFF044698
:10F1D0000D4653EC192B5B485549F6F745FF02469F
:10F1E0000B4620462946FAF7E3FB32463B46F7F743
:10F1F00039F852465B46F7F735F804460D4653ECAE
:10F200001A2B00205049F6F72FFF22462B4620E00C
:10F210004FF0C0404D49F6F727FF04460D4653EC2A
:10F22000182B4B484B49F6F71FFF06460F4653EC89
:10F23000192B49484549F6F717FF02460B46304659
:10F240003946FAF7B5FB22462B46F7F70BF853EC95
:10F250001A2BF7F707F802B0BDEC068BBDE8F48C6B
:10F2600080B52DED028B41EC180B53EC182B1F4889
:10F270001F49F6F7F9FE1F4A1F4BF6F7F3FF53EC51
:10F28000182BF6F7F1FE1D4A1D4BF6F7EBFF53EC7A
:10F29000182BF6F7E9FE1B4A1B4BF6F7E3FF53EC7E
:10F2A000182BF6F7E1FE194A194BF6F7DBFF53EC82
:10F2B000182BF6F7D9FE174A174BF6F7D3FF53EC86
:10F2C000182BF6F7D1FE154A154BBDEC028BBDE8A5
:10F2D0000050F6F7C7BF00000000F0FFCD3B7F668F
:10F2E0009EA0E63F0000F0BF0000F03FF7DE29BF20
:10F2F000D8F8C23FF4B3FECC1A99C33F62CB68D9A9
:10F300006F46C73FC6C912DAC471CC3F4AE98A9436
:10F310002449D23FF75F97999999D93FBC555555E4
:10F320005555E53F9EBC9AF71C7D7F3E422EE63F39
:10F330007BCBDB3FABA6320EE526553E7CC4BC7FC3
:10F34000DE27743E0EE526151344D33F4715F73FDD
:10F3500044DF5DF80BAE543EFE822B6530B443684B
:10F3600003F0004201211B031B0B436004BF036831
:10F37000002B08D10DE00368DD0F45EA440444602A
:10F380005B000360491E4468E302F4D523031B0BB2
:10F39000436043681A434260084630BC7047426885
:10F3A000C2F30A5240F2FF739A4209D1416809033D
:10F3B00004BF0068002801D1012070470220704777
:10F3C00043685B0004BF0368002B25D040F2334341
:10F3D0009A1A521A012A1FDB352A06DB416801F00E
:10F3E000004141600021016013E0012102F01F0390
:10F3F0009940491E920607D5426811404A40426032
:10F4000002681143002202E0026811404A40026093
:10F4100011B14FF0FF3070470020704790420CD17F
:10F4200041EA030C50EA4C0C07D0994205D14FF445
:10F43000001C1CEB410F38BF89427047014802F0A5
:10F4400085B80000000003002DE9704C04462DED46
:10F45000088B94ED009B43EC182B51EC190B02F038
:10F4600081F8064651EC180B02F07CF831000E9D35
:10F4700006D500284DD4022805D184ED008B42E149
:10F48000022EF8D121E050B951EC190B0022344B77
:10F49000FFF7C4FF0FD084ED008B002033E101287B
:10F4A00018D151EC190B00222E4BFFF7B7FF18BFF4
:10F4B00084ED008B51D1FFF7C1FF212101604FF096
:10F4C000FF306FF00041C4E90001BDEC088B022061
:10F4D000BDE8708C7EB984ED008B2946204600F093
:10F4E0004FF9040018BF012C40F00C81FFF7A6FF74
:10F4F0002221016006E151EC190B0022184BFFF7A5
:10F500008DFF0DD151EC180BF6F7AEFDC4E90001EB
:10F5100023E051EC190B0022134BF6F777FF0BD2C7
:10F5200051EC180B0023F6F79FFDC4E90001BDEC78
:10F53000088B0020BDE8708C01220C4BF6F74EFFC3
:10F5400016D851EC180B0022054BF6F78DFDC4E9D7
:10F550000001FFF773FF222101600120D3E000BF0B
:10F560000000F07F0000F0FF00C89CC000C89C4075
:10F57000384A394BF6F778FD00220023F6F746FFAC
:10F5800034BF9FED360B9FED370B53EC102BF6F786
:10F5900069FEF6F73BFE0646F9F754FA41EC1A0B02
:10F5A0004FF07842314BF6F75FFD02460B4651ECC7
:10F5B000190BFAF7FDF982468B4653EC1A2B2C48AF
:10F5C0002C49F6F751FD02460B4650465946FAF7CC
:10F5D000EFF96FF00102284BF6F700FF41EC190B31
:10F5E00005D80022254BF6F711FFC0F07D8053ECC3
:10F5F000192BF6F739FD41EC1A0B214A214BF6F78E
:10F6000033FD214A214BF6F72DFE53EC1A2BF6F76A
:10F610002BFD1F4A1F4B41EC1B0B51EC1A0BF6F74D
:10F6200023FD1D4A1D4BF6F71DFE53EC1A2BF6F772
:10F630001BFD1B4B0022F6F715FE53EC192BF6F7BA
:10F6400013FD41EC190B9FED01AB2BE00000000016
:10F650000000F03FFE822B654715F73F00000000D9
:10F660000000E0BF000000000000E03F422EE63F47
:10F67000F2E4D5BCE7E84B3EFFFF8FBC0000903CB6
:10F68000112E5781A03F503F5843128C8F71BC3FC1
:10F690004BE8A541B752013F0BBDF3DAE8708C3F50
:10F6A0000000E03F51EC1B0B53EC192BF6F7DAFD91
:10F6B00053EC1A2BF6F7D6FD82468B4651EC1B0B0A
:10F6C00053EC192BFAF774F953EC1A2BF6F7CAFD21
:10F6D00002460B4650465946FCF7A8FD53EC182B42
:10F6E000F6F7C2FC41EC180B84ED008BA9192046FB
:10F6F00000F046F8040018BF012C03D1FFF79EFE6E
:10F70000222101602046BDEC088BBDE8708C000012
:10F710000278C9B28A421AB11CBF10F8012FF9E76A
:10F7200018BF002070470000C9B2830706D0521EE0
:10F7300022D310F8013B9942F7D11FE0083A13D3C6
:10F7400002F1040241EA012141EA014150F8043B7F
:10F75000121F21BF4B40A3F1013C2CEA030C1CF00B
:10F76000803FF3D0C9B2001F083210F8013B521E8F
:10F7700028BF91EA030FF8D818BF0120401E704738
:10F7800070B504460D466068C0F30A5040F2FF7140
:10F79000884207D16068000304BF2068002817D0A2
:10F7A000022070BD20B92046FFF7D8FD012868DA95
:10F7B000012D0FDB40F2FF71091A8D420AD36068F8
:10F7C00000284CBF9FED300B9FED310B84ED000BFB
:10F7D000012070BD4142A942616806DA6FF31E51F3
:10F7E000401941EA0050606042E0401E63684519DC
:10F7F000012205F1350062F31F53352801F0004165
:10F80000636003D361600020206070BD002215F1A9
:10F810001F0F04DA226823600020203560606842F0
:10F8200014D0521E25689241C0F12003D2439D405E
:10F8300045EAD272256825FA00F6656805FA03F3F1
:10F8400033432360636823FA00F56560606808430A
:10F85000B2F1004F606003D80DD12078C0070AD5FF
:10F860002068401C2060206828B96068401C6060E7
:10F870004FF0FF3070BD6068884204BF20680028E8
:10F88000F6D1002070BD00BF000000000000F0FFB6
:10F89000000000000000F07F91FBF2F303FB121167
:10F8A000C0E900317047000007490A78521C0A700D
:10F8B00000224A70114681F31188044908700878C3
:10F8C0000028FCD1704700BFC0630300AEC2030034
:10F8D00010B5044602E0C068F6F726FF802080F3EA
:10F8E000118800BF00BF20680028F4D1024840788A
:10F8F00008B980F3118810BDC063030000B50D4A3C
:10F90000936885B0039302900190802383F311885C
:10F9100000BF00BF0368009300AB0360009800B114
:10F920004360906800AA82600174F6F779FF05B021
:10F9300000BD00BFC0630300012001F033BE000022
:10F940000749086808B1002070470648C008C00091
:10F9500008600549C908C900091A0160704700BF5D
:10F96000A4C203000F2003000840030030B482B09B
:10F9700083680469828AE318C468A34228BF1B1BFA
:10F980005343446811F8015B1D555B1C521EF8D1AE
:10F990008168491C8160012903D102B030BCFFF7A6
:10F9A00097BF1948407808B980F3118802B030BC7D
:10F9B000704710B481B0828A0369534344681C5D68
:10F9C00001F8014B5B1C521EF8D10169491C016111
:10F9D000C268914224BF0021016181684B1E83608F
:10F9E0009142094B5B7807D113B9002181F311884B
:10F9F00001B010BCFFF76CBF13B9002080F3118871
:10FA000001B010BC70470000C06303001FB5FFF7D2
:10FA100015FD212101601FBD1AA210EE101ADFF89A
:10FA200060C0F2EC060A614509DB00EE803A70EE38
:10FA3000800A83EE200A40F0020010EE101A21F036
:10FA4000004CDCF1665C0BD860EE000A20EE203A38
:10FA500003EE010A01EEA02A42EE202A80EE220ADD
:10FA6000400810F0020F18BFB1EE400A02EB80020E
:10FA7000D2ED000A30EE200A28BFB1EE400A7047EE
:10FA8000A430893ED7B3DD3F6AD5033F2B94A93D0F
:10FA9000B82A593F0000803F000080BF00000000EE
:10FAA000920A063FDB0FC93F920A863FDB0FC93F30
:10FAB000920A0640DB0F4940368D274001E0491C81
:10FAC000521E72B10B7890F800C09C4505D002D24E
:10FAD0004FF0FF3070470120704710F8013B002BBA
:10FAE000EDD1002070470000DFF8C8130860DFF890
:10FAF000C8031021016001680906FCD4DFF8BC03CB
:10FB0000012101600168C903FCD401214160416801
:10FB1000C903FCD4DFF8A803012101600168C9030F
:10FB2000FCD4002141604168C903FCD47047DFF870
:10FB300094037047DFF880030068C00603D5DFF840
:10FB4000740300687047DFF87C037047F2E7F1E761
:10FB500080B5DFF868030068C00702D5FFF7F6FF3D
:10FB600001E0DFF86003DFF85813096801F00F01C6
:10FB7000491CB0FBF1F002BD7047DFF844130A687E
:10FB8000120900F00F0050EA021008600868C00374
:10FB9000FCD4704780B5DFF830030068C00702D599
:10FBA000FFF7D4FF01E0DFF81C03DFF8201309683A
:10FBB00001F00F01491CB0FBF1F002BDDFF80C139E
:10FBC0000A68120900F00F0050EA02100860086885
:10FBD000C003FCD47047DFF8F802704780B5DFF847
:10FBE000F4020068C00702D5FFF7F5FF01E0DFF877
:10FBF000D402DFF8E412096801F00F01491CB0FBE0
:10FC0000F1F002BD80B5DFF8D4020068C00702D56C
:10FC1000FFF7E1FF01E0DFF8AC02DFF8C41209688A
:10FC200001F00F01491CB0FBF1F002BD80B5DFF817
:10FC3000B4020068C00702D5FFF7CDFF01E0DFF88E
:10FC40008402DFF8A412096801F00F01491CB0FB1F
:10FC5000F1F002BD80B5DFF894020068C00702D55C
:10FC6000FFF7B9FF01E0DFF85C02DFF884120968F2
:10FC700001F00F01491CB0FBF1F002BD80B5DFF8C7
:10FC800074020068C00702D5FFF7A5FF01E0DFF8A6
:10FC90003402DFF86412096801F00F01491CB0FB5F
:10FCA000F1F002BD80B5DFF854020068C00702D54C
:10FCB000FFF791FF01E0DFF80C02DFF8441209685A
:10FCC00001F00F01491CB0FBF1F002BDDFF8081292
:10FCD0000A68120900F00F0050EA02100860086874
:10FCE000C003FCD47047DFF8F8110A68120900F06D
:10FCF0000F0050EA021008600868C003FCD4704787
:10FD0000DFF8E4110A68120900F00F0050EA02104F
:10FD100008600868C003FCD47047DFF8D4110A6893
:10FD2000120900F00F0050EA021008600868C003D2
:10FD3000FCD47047DFF8C0110A68120900F00F0008
:10FD400050EA021008600868C003FCD47047DFF86E
:10FD5000B0110A68120900F00F0050EA02100860A2
:10FD60000868C003FCD4704780B50E2834D8DFE89B
:10FD700000F01E080B0F1215181B1E2124272A2D18
:10FD800030004FF4004002BDDFF82801006802BDDA
:10FD9000BDE80140DBE6BDE80140C8E6BDE8014042
:10FDA000D4E6BDE80140D3E6BDE80140F2E6DFF865
:10FDB000140102BDBDE8014010E7BDE8014021E7A4
:10FDC000BDE8014032E7BDE8014043E7BDE801403E
:10FDD00054E7BDE8014065E740F261120FF23811C7
:10FDE0000FF22810F8F71CFE0020C046C046002085
:10FDF00002BD000080B5401F09282BD8DFE800F0C5
:10FE0000050A0E2A12161A1E22260846FFF7B4FE0D
:10FE1000012002BD0846FFF7B0FEF9E70846FFF7EC
:10FE2000CDFEF5E70846FFF751FFF1E70846FFF77B
:10FE30005AFFEDE70846FFF763FFE9E70846FFF7DB
:10FE40006CFFE5E70846FFF775FFE1E70846FFF7B7
:10FE50007EFFDDE74FF4C9720FF2BC010FF2AC0078
:10FE6000F8F7DEFD0020C046C046002002BD10B5F8
:10FE7000DFF89040217800290CD040F2A1120FF257
:10FE800098010FF28800F8F7CBFD0020C046C0466D
:10FE9000002010BDDFF87010002803D04FF0405252
:10FEA0000A6001E000220A6001F082FB012020705C
:10FEB00010BD00007C6903000001104000101040DC
:10FEC0000018104000007701041010400418104082
:10FED00000EA3206041060400418604008106040D8
:10FEE000081860400C1060400C1860401010604012
:10FEF00010186040141060401418604018106040E2
:10FF000018186040A9C20300000810405B455D2539
:10FF1000732C2025640A0000443A5C576F726B739F
:10FF2000706163655C4445565C53656E736F7248DF
:10FF300075625C4D4153535F50524F4A4543545C88
:10FF400050524F445C47544134584C5C525C706C86
:10FF50006174666F726D5C6578796E6F7339363176
:10FF6000305C6669726D776172655C6F735C706C32
:10FF70006174666F726D5C6578796E6F735C7372B5
:10FF8000635C636D755C636D7544727639363130D0
:10FF90002E630000012100F01F029140874A4009B2
:10FFA00042F820107047012100F01F029140844A5E
:10FFB000400942F82010704710B5002403E02046A5
:10FFC00000F002F9641C072CF9DB0420FFF7EBFFBB
:10FFD0000420BDE81040DDE718B4342212FB00F025
:10FFE0000FF2882283185C68002C11D0805C00F02E
:10FFF0000F00DA690092009A12686043714B53F85F
:020000021000EC
:10000000243083409A4301FA00F0104300990860BD
:1000100011BC704781B0342111FB00F00FF24C216C
:1000200042185368002B02D14FF0FF300DE0D26927
:100030000092009A1268405C00F00F00584311468D
:10004000C140604850F82300084001B0704718B420
:10005000342212FB00F00FF2142283189C68002C4B
:1000600011D0805C00F00F001A6A0092009A1268AA
:100070006043544B53F8243083409A4301FA00F014
:1000800010430099086011BC704781B0342111FB06
:1000900000F00FF2D81142189368002B02D14FF0F4
:1000A000FF300FE0405C00F00F00116A00910099F2
:1000B000096803FB00F2434850F8230090400140D8
:1000C0000846D04001B0704718B4342212FB00F04B
:1000D0000FF298128318DC68002C11D0805C00F0BD
:1000E0000F005A6A0092009A12686043354B53F829
:1000F000243083409A4301FA00F0104300990860CD
:1001000011BC704718B4342212FB00F00FF25C12DD
:1001100083181C69002C11D0805C00F00F009A6AD3
:100120000092009A12686043264B53F824308340B3
:100130009A4301FA00F010430099086011BC70471F
:1001400018B4342212FB00F00FF2201283185C69FD
:10015000002C11D0805C00F00F00DA6A0092009A47
:1001600012686043174B53F8243083409A4301FAD6
:1001700000F010430099086011BC704718B4342295
:1001800012FB00F00FF2E40283189C69002C11D0DE
:10019000805C00F00F001A6B0092009A12686043B6
:1001A000084B53F8243083409A4301FA00F010437F
:1001B0000099086011BC70470000000000E100E0F9
:1001C00080E200E0A068030010B582B00FF2507129
:1001D00000EBC00201EB82040021207CFFF7FCFE53
:1001E000E0690090009800680121A26801FA02F21B
:1001F0001043009A1060206A0090E06801FA00F055
:100200000099086013BD0FF2187100EBC00201EBFA
:100210008200007C39E781B00FF2047100EBC0026C
:1002200001EB8200C168006A0090009800680246F5
:10023000CA40D00703D5012088400099086001B06A
:10024000704781B00FF2D86100EBC00201EB820071
:10025000016A009100990968C0680A46C240D00747
:1002600001D5012000E0002001B07047000000002F
:100270000400000001000000040000000400000071
:1002800002000000040000000000184004001840B4
:10029000080018400C0018401000184014001840C6
:1002A0000100000004000000010000000400000044
:1002B00004000000020000000400000000001840DC
:1002C00004001840080018400C00184010001840A6
:1002D00014001840020000000400000001000000AB
:1002E0000400000004000000020000000400000000
:1002F0000000184004001840080018400C00184086
:100300001000184014001840030000000400000012
:1003100001000000040000000400000002000000D2
:1003200004000000000018400400184008001840B5
:100330000C00184010001840140018400000000085
:1003400004000000010000000400000004000000A0
:1003500002000000040000002000184024001840A3
:10036000280018402C001840300018403400184075
:100370000100000004000000010000000400000073
:1003800004000000020000000400000020001840EB
:1003900024001840280018402C0018403000184055
:1003A00034001840020000000400000001000000BA
:1003B000040000000400000002000000040000002F
:1003C0002000184024001840280018402C00184035
:1003D0003000184034001840000000000400000005
:1003E0000100000004000000040000000000000004
:1003F000000000000000624004006240080062400B
:100400000C0062401C0062401C00624000000000C2
:1004100004000000010000000400000004000000CF
:100420000000000000000000200062402400624044
:10043000280062402C0062403C0062403C00624068
:1004400000000000040000000100000004000000A3
:1004500004000000000000000000000040006240B6
:1004600044006240480062404C0062405C006240D0
:100470005C00624000000000040000000100000079
:100480000400000004000000000000000000000064
:100490006000624064006240680062406C0062403C
:1004A0007C0062407C00624000000000040000000C
:1004B0000100000004000000040000000000000033
:1004C00000000000800062408400624088006240BA
:1004D0008C0062409C0062409C0062400000000072
:1004E00004000000010000000400000004000000FF
:1004F0000000000000000000A0006240A400624074
:10050000A8006240AC006240BC006240BC00624097
:1005100000000000040000000100000004000000D2
:10052000040000000000000000000000C000624065
:10053000C4006240C8006240CC006240DC006240FF
:10054000DC00624000000000040000000100000028
:100550000400000004000000000000000000000093
:10056000E0006240E4006240E8006240EC0062406B
:10057000FC006240FC00624000000000040000003B
:100580000100000004000000040000000000000062
:100590000000000000016240040162400801624066
:1005A0000C0162401C0162401C016240000000001E
:1005B000040000000100000004000000040000002E
:1005C00000000000000000002001624024016240A1
:1005D000280162402C0162403C0162403C016240C3
:1005E0000000000004000000010000000400000002
:1005F0000400000000000000000000004001624014
:1006000044016240480162404C0162405C0162402A
:100610005C016240000000000400000001000000D6
:1006200004000000040000000000000000000000C2
:100630006001624064016240680162406C01624096
:100640007C0162407C016240000000000400000068
:100650000100000004000000040000000000000091
:100660000000000080016240840162408801624015
:100670008C0162409C0162409C01624000000000CD
:10068000040000000100000004000000040000005D
:100690000000000000000000A0016240A4016240D0
:1006A000A8016240AC016240BC016240BC016240F2
:1006B0000000000004000000010000000400000031
:1006C000040000000000000000000000C0016240C3
:1006D000C4016240C8016240CC016240DC0162405A
:1006E000DC01624000000000040000000100000086
:1006F00004000000040000000000000000000000F2
:10070000E0016240E4016240E8016240EC016240C5
:10071000FC016240FC016240000000000400000097
:1007200001000000040000000400000000000000C0
:1007300000000000000262400402624008026240C1
:100740000C0262401C0262401C0262400000000079
:10075000040000000100000004000000040000008C
:1007600000000000000000002002624024026240FD
:10077000280262402C0262403C0262403C0262401D
:100780000000000004000000010000000400000060
:100790000400000000000000000000004002624071
:1007A00044026240480262404C0262405C02624085
:1007B0005C02624000000000040000000100000034
:1007C0000400000004000000000000000000000021
:1007D0006002624064026240680262406C026240F1
:1007E0007C0262407C0262400000000004000000C5
:1007F00001000000040000000400000000000000F0
:100800000000000080026240840262408802624070
:100810008C0262409C0262409C0262400000000028
:1008200004000000010000000400000004000000BB
:100830000000000000000000A0026240A40262402C
:10084000A8026240AC026240BC026240BC0262404C
:10085000000000000400000001000000040000008F
:10086000040000000000000000000000C002624020
:10087000C4026240C8026240CC026240DC026240B4
:10088000DC026240000000000400000001000000E3
:100890000400000004000000000000000000000050
:1008A000E0026240E4026240E8026240EC02624020
:1008B000FC026240FC0262400000000004000000F4
:1008C000010000000400000004000000000000001F
:1008D000000000000003624004036240080362401D
:1008E0000C0362401C0362401C03624000000000D5
:1008F00004000000010000000400000004000000EB
:100900000000000000000000200362402403624059
:10091000280362402C0362403C0362403C03624077
:1009200000000000000000000000000000000000C7
:100930000000000000071840000818400009184097
:10094000000A184004000000080000000100000038
:1009500001000000010000000007184000081840D6
:1009600000091840000A18400800000010000000AC
:100970000200000002000000020000000007184012
:100980000008184000091840000A18400C00000038
:100990001800000003000000030000000300000036
:1009A000000718400008184000091840000A1840C5
:1009B0000000000000000000000000000000000037
:1009C00004000000040718400408184004091840F7
:1009D000040A1840040000000800000001000000A4
:1009E000010000000500000004071840040818403A
:1009F00004091840040A1840080000001000000014
:100A00000200000002000000060000000407184079
:100A10000408184004091840040A184000000000A7
:100A200000000000000000000000000007000000BF
:100A3000000762400008624000096240000A62400C
:100A400000000000000000000000000000000000A6
:100A50000800000004076240040862400409624084
:100A6000040A6240000000000000000000000000D6
:100A7000000000000900000008076240080862400A
:100A800008096240080A62400000000000000000FF
:100A900000000000000000000A0000000C07624097
:100AA0000C0862400C0962400C0A62400000000021
:100AB0000000000000000000000000000B0000002B
:100AC000100762401008624010096240100A62403C
:100AD0000000000000000000000000000000000016
:100AE0000C000000140762401408624014096240C0
:100AF000140A624000000000000000000000000036
:100B0000000000000D000000180762401808624055
:100B100018096240180A624000000000000000004E
:100B200000000000000000000E0000001C076240F2
:100B30001C0862401C0962401C0A62400000000060
:100B40000000000000000000000000000F00000096
:100B5000200762402008624020096240200A62406B
:100B60000000000000000000000000000000000085
:100B700010000000240762402408624024096240FB
:100B8000240A624000000000000000000000000095
:100B900000000000110000002807624028086240A1
:100BA00028096240280A624000000000000000009E
:100BB0000000000000000000120000002C0762404E
:100BC0002C0862402C0962402C0A624000000000A0
:100BD0000000000000000000000000001300000002
:100BE000300762403008624030096240300A62409B
:100BF00000000000000000000000000000000000F5
:100C00001400000034076240340862403409624036
:100C1000340A6240000000000000000000000000F4
:100C200000000000150000003807624038086240EC
:100C300038096240380A62400000000000000000ED
:100C40000000000000000000160000003C076240A9
:100C50003C0862403C0962403C0A624000000000DF
:100C6000000000000000000000000000170000006D
:100C7000400762404008624040096240400A6240CA
:100C80000000000000000000000000000000000064
:100C90001800000044076240440862404409624072
:100CA000440A624000000000000000000000000054
:100CB0000000000019000000480762404808624038
:100CC00048096240480A624000000000000000003D
:100CD00000000000000000001A0000004C07624005
:100CE0004C0862404C0962404C0A6240000000001F
:100CF0000000000000000000000000001B000000D9
:100D0000500762405008624050096240500A6240F9
:100D100000000000000000000000000000000000D3
:100D20001C000000540762405408624054096240AD
:100D3000540A6240000000000000000000000000B3
:100D4000000000001D000000580762405808624083
:100D500058096240580A624000000000000000008C
:100D600000000000000000001E0000005C07624060
:100D70005C0862405C0962405C0A6240000000005E
:100D80000000000000000000000000001F00000044
:100D9000600762406008624060096240600A624029
:100DA0000000000000000000000000000000000043
:100DB00020000000640762406408624064096240E9
:100DC000640A6240012100F01F0291401D4A40095F
:100DD00042F820107047012100F01F0291401A4A8A
:100DE000400942F82010704780B518484FF0FF3195
:100DF000016001631320FFF7EEFF1320BDE80240FE
:100E0000E0E730B400210846114A1368044606E0C2
:100E10001D46E540ED0701D520460121641C202C2C
:100E2000F6D300290BD1136B002406E01946E140EC
:100E3000C90701D504F12000641C202CF6D330BC76
:100E40007047000000E100E080E200E05C026740E3
:100E50007C026740F8B500240FF240061BE0C4EBAB
:100E6000C405AF197978A85DFCF750FCB978A85D86
:100E7000FCF773FCF978A85DFCF796FC3979A85D5E
:100E8000FCF7B8FC7979A85DFCF7C7FCB979A85DD7
:100E9000FCF79DFC641C0A2CE1D3F1BD0B020100A0
:100EA0000300000C02010003000011030100030015
:100EB000001203010003000000020103030300010C
:100EC0000201030303000202010103010003020106
:100ED00003030300050F0000020000040F000002DE
:100EE0000000000010B5002409E0064800EBC40132
:100EF0004A79097950F8340000F07EFB641C032C19
:100F0000F3D310BD58680300F8B5002510E0052E96
:100F100000D10E242046C0B2FCF796FB7969890007
:100F2000B0FBF1F0411E2046C0B2FCF7A0FB6D1CE7
:100F3000012D28DA0FF26C00E42101FB05077E6821
:100F400001220221304600F057FB002803D00FF2A7
:100F50003800F7F765FD39462846F7F74FFB002EB6
:100F600001D10724D6E7012E01D10A24D2E7022EAF
:100F700001D10B24CEE7032E01D10C24CAE7042EA5
:100F8000C5D10D24C6E7F1BD5B455D0A4552524F00
:100F90005220737069426F617264496E69742121D5
:100FA000210A000000000000000000000000000016
:100FB000000001010000000000127A0000127A0017
:100FC0000000000000000000000000000000000021
:100FD0000000000000000000000000000000000011
:100FE0000000000000000000000000000000000001
:100FF00000000000000000000000000000000000F1
:1010000000000100000000000000000000000000DF
:1010100000000000000000000000000000000000D0
:1010200000000000000000000000000000000000C0
:1010300000000000000000000000000000000000B0
:1010400000000000000000000000000000000000A0
:101050000000000000000000000000000000000090
:101060000000000000000000000000000000000080
:101070000000000000000000000000000000000070
:10108000000000000000000000B5ADF2D47D00A813
:101090004FF4FA61F1F762FA06E04FF4FA6300AA3E
:1010A000DFF8640300F04FF94FF4FA6100A800F094
:1010B000C9FD01281BDB40F245318842EDD040F2EA
:1010C000454188420BD047F20A118842ECD14FF4D7
:1010D000FA6300AADFF8300300F0ACF9E4E74FF45C
:1010E000FA6300AADFF8200300F0FAF9DCE70DF25A
:1010F000D47D00BD2DE9D0030446DFF81083DFF86E
:101100001093A8FB046709FB0477DFF80803E0FBF2
:101110000167DFF80403DFF8041330187941DFF8C2
:101120000033A3FB0223801A9941BDE8D003704726
:101130002DE9F04186B004460D4616461F460020B4
:101140008DF8150001208DF814000020ADF8100076
:10115000002F06D01820ADF80E0000208DF80C00EE
:1011600005E00220ADF80E0001208DF80C004FF4D0
:101170007A70684302908DF8124070008DF8130069
:10118000102202A940F2654000F0EBFC8046019776
:1011900000962B4622460FF264310FF27030F7F7BB
:1011A0003FFCB8F1010F01DB012000E0002006B098
:1011B000BDE8F08194494860704793498860704762
:1011C0009149086070479049C860704700208E4977
:1011D0004860704700208C498860704700208A4929
:1011E0000860704700208849C860704786494A688F
:1011F000002A01D0002801D5002070470246521E67
:101200009241D20F8A7501220A750861887D0028F3
:1012100004D000231A460121104689E700231A460C
:101220000969104684E778480021817501750161DC
:10123000417D00230A4618467AE701460020724A9B
:101240001368002B07D05175117D002903D1517D02
:1012500003460A466CE7704738B504466A4DE868AD
:10126000002801D1002032BD23462246214601201C
:10127000FFF75EFF002800D0EC7532BD38B504469C
:10128000614DE87D044202D00120FFF7E5FF2046D2
:10129000401E8041C00F8DF80000012200A94FF4CC
:1012A000A26000F05EFC012800DB2C76012801DB47
:1012B000012032BD002032BD534800210160416051
:1012C0008160C16081754175012101760021C17580
:1012D00000F069BD70B400229FED4A0A134690F9F0
:1012E000044002E041F82220521CA242FADB012C09
:1012F00027DB1A461FE051F8245005EB850600EB6A
:101300008605D5ED030AB4EE600AF1EE10FA02D5B7
:10131000B0EE600A2346641C90F90450AC42EADB4C
:1013200051F8224051F8235041F8225041F823400F
:101330009FED340A521C90F90440A24201DA14468F
:10134000EAE770BC704730B58FB004461546002CF4
:1013500054D0002D52D0287900F03F003F284DD1C5
:10136000E868F7F76FFB4FF403722E4BF4F77CFE3F
:10137000CDE900012869F7F765FB6FF0E7022A4B1A
:10138000F4F772FECDE902016869F7F75BFB002212
:10139000264BFAF74BFFCDE90401688BF7F75CFBAE
:1013A0000022234BFAF742FFCDE90601A88BF7F79D
:1013B00053FB00221D4BFAF739FFCDE90801288BBA
:1013C0000C906A79A968E888FFF794FECDE90A01D4
:1013D000207D002805D0616808000AD000A8884751
:1013E00007E0607D002804D02168080001D000A833
:1013F0008847A07D002801D0FFF715FF0FB030BD52
:101400000000000000000000F4BE0300000029F905
:101410000F26020040420F00000087C14F8862047F
:1014200000CA9A3B0080663EFF7F763E0000244063
:101430000000594070B5ADF5A16D04461546A06891
:1014400000284AD0002D48D00026FFA908312846A0
:10145000FFF740FF3046009036E0FFA8083050F814
:10146000260000EB800105EB810090ED030AB5EE4C
:10147000400AF1EE10FA26DD00A9009A01EB0211F4
:1014800081ED020A017A00AA009B02EB031211719E
:10149000417A00AA009B02EB0312517100A9009A45
:1014A00001EB021102690A6100A9009A01EB021125
:1014B0004269CA60807A00A9009A01EB0211887122
:1014C0000098401C0090761C95F904008642C4DB0D
:1014D000A168080001D000A888470DF5A16D70BD76
:1014E000C168080009D0002A07D0080005D012788A
:1014F000501E8041C043C00F0847704773656E643B
:101500004C6F636174696F6E526571005B495D5B1E
:10151000202573205D2069643A2575207261746509
:101520003A256C6920706173736976653A25752078
:10153000617661696C3A25750A00000000F041B8D7
:1015400000F046B800F04EB8000000000349044A1D
:10155000096801B91146801A40187047A0C20300FB
:101560000000030003B4DDE90023C3F30A5140F295
:10157000FF72914206D001B10CE0190350EA11301C
:1015800006D00BE0190350EA113014BF02200120ED
:1015900002B070474FF0FF3002B070476FF00100AB
:1015A00002B070472021090326311820ABBEF9E7AD
:1015B0000F49002802D07F20086070470020086093
:1015C00070470C490A68C00052EAD00008607047B2
:1015D00008490A6802F06042C043C00052EAD000E5
:1015E0000860704703480068C000C00870470000EA
:1015F000040111402804114038B504460D462B461D
:101600000C2C03D2052B01DA022A0ADB00922246B7
:101610000FF224010FF22800F7F702FA6FF015001D
:1016200032BD00F0DAFD002802D102482554002026
:1016300032BD00002CC203007573694F70656E00E7
:101640005B455D25732C20696E76616C6964207042
:101650006172616D65746572202825642C20256493
:101660002C202564290A0000F0B591B004460D46EF
:10167000002600AF17E0DFF8C405335D1B111B5CCB
:101680003B70335D03F00F03185C07F8010F761C05
:10169000002007F8010F491C9142ECDB00A90FF272
:1016A0007860F7F7BDF9AE4205DAAA1B212A00DB04
:1016B00020220021F0E711B0F0BD01684A1C026051
:1016C0000878704701688A1C02600878497840EA07
:1016D0000120704701680A1D026008784A7840EAD4
:1016E00002208A7840EA0240C97840EA01607047E7
:1016F00081B001680A1D026008784A7840EA022039
:101700008A7840EA0240C97840EA016000909DED85
:10171000000A01B0704713B50446012201A92068F0
:10172000F0F7D4FE2068401C2060012016BD13B5E0
:101730000446022201A92068F0F7C8FE2068801C38
:101740002060022016BD13B50446042201A92068BA
:10175000F0F7BCFE2068001D2060042016BD38B5DF
:1017600004460D460094297800A8FFF7D4FF697855
:1017700000A8FFF7D0FFA97800A8FFF7CCFFE97811
:1017800000A8FFF7C8FF297900A8FFF7C4FF69790F
:1017900000A8FFF7C0FFA97900A8FFF7BCFFE9790F
:1017A00000A8FFF7B8FF297A00A8FFF7B4FF697A0D
:1017B00000A8FFF7B0FFA97A00A8FFF7ACFFE97A0D
:1017C00000A8FFF7A8FF297B00A8FFF7A4FF697B0B
:1017D00000A8FFF7A0FFA97B00A8FFF79CFFE97B0B
:1017E00000A8FFF798FF297C00A8FFF794FF697C09
:1017F00000A8FFF790FFA97C00A8FFF78CFFE97C09
:1018000000A8FFF788FF297D00A8FFF784FF697D06
:1018100000A8FFF780FFA97D00A8FFF77CFFE97D06
:1018200000A8FFF778FF297E00A8FFF774FF697E04
:1018300000A8FFF770FFA97E00A8FFF76CFFE97E04
:1018400000A8FFF768FF297F00A8FFF764FF697F02
:1018500000A8FFF760FFA97F00A8FFF75CFFE97F02
:1018600000A8FFF758FF95F8201000A8FFF753FFD6
:1018700095F8211000A8FFF74EFF95F8221000A858
:10188000FFF749FF95F8231000A8FFF744FF95F8EC
:10189000241000A8FFF73FFF95F8251000A8FFF7D8
:1018A0003AFF95F8261000A8FFF735FF95F82710A6
:1018B00000A8FFF730FF95F8281000A8FFF72BFFCE
:1018C00095F8291000A8FFF726FF95F82A1000A820
:1018D000FFF721FF95F82B1000A8FFF71CFF95F8E4
:1018E0002C1000A8FFF717FF95F82D1000A8FFF7A0
:1018F00012FF95F82E1000A8FFF70DFF95F82F1096
:1019000000A8FFF708FF95F8301000A8FFF703FFC5
:1019100095F8311000A8FFF7FEFE95F8321000A8E8
:10192000FFF7F9FE95F8331000A8FFF7F4FE0098D2
:10193000001B32BD38B504460D460094296800A846
:10194000FFF701FF297900A8FFF7E5FEE98800A865
:10195000FFF7EDFE298900A8FFF7E9FEA97A00A8A4
:10196000FFF7D9FEE97A00A8FFF7D5FE297B00A88A
:10197000FFF7D1FE697B00A8FFF7CDFE0098001BA2
:1019800032BD10B582B004460094097800A8FFF774
:10199000C2FE0098001B16BD38B504460D460094E3
:1019A000297800A8FFF7B7FE697800A8FFF7B3FE13
:1019B0000098001B32BD10B582B00446009409782F
:1019C00000A8FFF7A8FE0098001B16BD38B5044616
:1019D0000D46009500A8FFF770FE207000A8FFF7E5
:1019E0006CFE607000A8FFF768FEA07000A8FFF70B
:1019F00064FEE07000A8FFF760FE207100A8FFF70A
:101A00005CFE607100A8FFF75DFEE08000A8FFF7B4
:101A100061FEA06000A8FFF75DFEE06000A8FFF790
:101A200059FE206100A8FFF755FE606100A8FFF78E
:101A300049FE208300A8FFF745FE608300A8FFF75A
:101A400041FEA08300A8FFF738FEA0770098401B56
:101A500032BD38B504460D46009500A8FFF72DFEAF
:101A6000207000A8FFF729FE607000A8FFF725FE90
:101A7000A07000A8FFF73CFE84ED010A00A8FFF764
:101A800037FE84ED020A00A8FFF732FE84ED030A58
:101A900000A8FFF72DFE84ED040A0098401B32BD1C
:101AA000F8B505460C4600263746009400A8FFF717
:101AB00004FE287000A8FFF700FE687000A8FFF77A
:101AC000FCFDA87000A8FFF7F8FDE87000A8FFF77C
:101AD000F4FD287195F90400412810DBA0F14007BE
:101AE000402028710BE0009906EB860005EB800092
:101AF0000830FFF7AEFF009940180090761C95F96A
:101B000004008642EFDB002F03D0009800EB0710A3
:101B100000900098001BF2BD38B504460D460095B4
:101B200000A8FFF7CAFD20700098401B32BD38B5F1
:101B300004460D46009500A8FFF7BFFD207000A8E1
:101B4000FFF7BBFD60700098401B32BD38B50446FE
:101B50000D46009500A8FFF7B0FD20700098401BCF
:101B600032BD70B59CB004460E4602A86421F0F761
:101B7000F5FC00250FF21820D0E90023CDE9002361
:101B80002046ADF80400E4380CD040F26131401A30
:101B900020D020380CD0AB3810D040F2C711401AFA
:101BA00012D01DE0314604A8FFF7D9FD05461EE01E
:101BB000314604A8FFF7BEFE054618E0314604A8EA
:101BC000FFF7DFFE054612E0314604A8FFF7E4FE0A
:101BD00005460CE0314604A8FFF7EDFE054606E099
:101BE00022460FF24C110FF25410F6F719FF284657
:101BF000ADF80000A0208DF8080002ACA3206070B2
:101C0000062200A90DF10A00F0F760FC05F10800BA
